:020000040000FA
:0600000025EF74F0120070
:0610000025EF74F0120060
:06100800F5EF63F0120099
:06101800FDEF59F012008B
:101080000A00E8E80000CB02000032000000E5E8BA
:101090000000FA04000003000000E3E80000680319
:1010A000000002000000D9E800005E0300000A0012
:1010B0000000D6E80000FD0E00000300000089E6F5
:1010C00000006A03000001000000BDE800004503C5
:1010D000000019000000B5E80000380F000008000B
:1010E0000000A8E80000F00E00000D000000D7E4AA
:0A10F0000000FF04000001000000F2
:0610FA00D9CFE6FFDACFBA
:10110000E6FFE1CFD9FFE2CFDAFF110EE12402E3DF
:10111000E168E652E16E840EDF6EDE52880EDD6E0F
:101120008B0EF36E020EF3CFDBFF8E0EF36E030E0B
:10113000F3CFDBFF010EE76EFC0EDBCF14F0FD0EEC
:10114000DBCF15F0E7501426000E1522060E14C052
:10115000DBFF070E15C0DBFF080EDB6A090EDB6A3A
:101160000A0EDB6A0B0EDB6A0201010ED96FFC0E60
:10117000DBCFE9FFFD0EDBCFEAFF030ED890E936A7
:10118000EA36E806FBE1FD0EE926020EEA22EFCF81
:1011900014F0156A14BE15680C0E14C0DBFF0D0E9A
:1011A00015C0DBFFFC0EDBCFE9FFFD0EDBCFEAFF56
:1011B000030ED890E936EA36E806FBE1FD0EE92693
:1011C000020EEA22020EE926000EEA220E0EEFCFF0
:1011D000DBFFFC0EDBCFE9FFFD0EDBCFEAFF030EEA
:1011E000D890E936EA36E806FBE1FD0EE926020E64
:1011F000EA22020EE926000EEA22EE520F0EEFCF8F
:10120000DBFFFC0EDBCFE9FFFD0EDBCFEAFF030EB9
:10121000D890E936EA36E806FBE1FD0EE926020E33
:10122000EA22020EE926000EEA22020EE926000E4C
:10123000EA22100EEFCFDBFF250E0CC2E9FF0DC234
:10124000EAFFEF6E010E0201EA6A0C25E96E0D510C
:10125000EA220E0EEF6EE66AE668E6680CC2E6FF6A
:101260000DC2E6FF0FC2E6FF10C2E6FFAEEC43F090
:10127000146E070EE15C02E2E16AE552E16E145081
:10128000100EE66EE66A200EE66E0CC2E6FF0DC298
:10129000E6FFA8EC6EF0146E050EE15C02E2E16A76
:1012A000E552E16E1450210E0CC2E9FF0DC2EAFFB7
:1012B000EF6E7F0EE66EDA0EE66E000EE66E010E43
:1012C0000201156A0C25146E0D51152214C0E6FF9B
:1012D00015C0E6FFF4EC6EF0166E050EE15C02E25E
:1012E000E16AE552E16E16500F0EE76E060EDBCF97
:1012F00014F0070EE7501416156A300E1412000E83
:101300001512030E0201EA6A0C25E96E0D51EA225C
:1013100014C0EFFFD9500C0FE96E000EDA20EA6E10
:10132000EE50ED1017E17B0EE66EDA0EE66E000E63
:10133000E66E050E156A0C25146E0D51152214C0AB
:10134000E6FF15C0E6FFF4EC6EF0166E050EE15CEC
:1013500046E243D0D9500C0FE96E000EDA20EA6E57
:10136000010EEE1819E1ED5017E1770EE66EDA0E78
:10137000E66E000EE66E050E156A0C25146E0D5114
:10138000152214C0E6FF15C0E6FFF4EC6EF0166EF1
:10139000050EE15C24E221D0D9500C0FE96E000E5D
:1013A000DA20EA6E020EEE181CE1ED501AE1730E1F
:1013B000E66EDA0EE66E000EE66E050E156A0C2578
:1013C000146E0D51152214C0E6FF15C0E6FFF4ECB3
:1013D0006EF0166E050EE15C02E2E16AE552E16E26
:1013E0001650080E0201EA6A0C25E96E0D51EA2238
:1013F000200EEF6E0A0E146E0E6E0E0EDBCF09F08D
:1014000009EC71F009503009E66E090E0201EA6A32
:101410000C25E96E0D51EA22E552E750EF6E0E0EF3
:10142000DBCF14F014C009F00A0E0E6E09EC71F057
:1014300005503009E66E0A0E0201EA6A0C25E96ED3
:101440000D51EA22E552E750EF6E0B0EEA6A0C25C9
:10145000E96E0D51EA223A0EEF6E0A0E146E0E6E10
:101460000F0EDBCF09F009EC71F009503009E66E80
:101470000C0E0201EA6A0C25E96E0D51EA22E552D2
:10148000E750EF6E0F0EDBCF14F014C009F00A0E18
:101490000E6E09EC71F005503009E66E0D0E02017A
:1014A000EA6A0C25E96E0D51EA22E552E750EF6E2B
:1014B0000E0EEA6A0C25E96E0D51EA223A0EEF6E25
:1014C0000A0E146E0E6E100EDBCF09F009EC71F0EF
:1014D00009503009E66E0F0E0201EA6A0C25E96E2A
:1014E0000D51EA22E552E750EF6E100EDBCF14F0FB
:1014F00014C009F00A0E0E6E09EC71F005503009A7
:10150000E66E100E0201EA6A0C25E96E0D51EA2220
:10151000E552E750EF6EE66AE668E6680CC2E6FF61
:101520000DC2E6FF0FC2E6FF10C2E6FFAEEC43F0CD
:10153000146E070EE15C02E2E16AE552E16E1450BE
:10154000100EE66EE66A200EE66E0CC2E6FF0DC2D5
:10155000E6FFA8EC6EF0146E050EE15C02E2E16AB3
:10156000E552E16E1450400E0CC2E9FF0DC2EAFFD5
:10157000EF6E630EE66EDA0EE66E000EE66E010E9C
:101580000201156A0C25146E0D51152214C0E6FFD8
:1015900015C0E6FFF4EC6EF0166E050EE15C02E29B
:1015A000E16AE552E16E1650E66AE668E6680CC24A
:1015B000E6FF0DC2E6FF0FC2E6FF10C2E6FFAEEC8B
:1015C00043F0146E070EE15C02E2E16AE552E16E5F
:1015D0001450250E0CC2E9FF0DC2EAFFEF6ED9CF01
:1015E00014F0DACF15F0080EDB50D924E96E090E9D
:1015F000DB50DA20EA6EEF50E66E010E0201EA6A75
:101600000C25E96E0D51EA22E552E750EF6EE66ACD
:10161000E668E6680CC2E6FF0DC2E6FF0FC2E6FF11
:1016200010C2E6FFAEEC43F0146E070EE15C02E27E
:10163000E16AE552E16E1450E66AE668E668D95060
:10164000040FE66E000EDA20E66E11C2E6FF12C24B
:10165000E6FF93EC47F0146E070EE15C02E2E16AEC
:10166000E552E16E1450000901E125D3040EDB5070
:10167000040A01E1B7D2010A01E162D2060A01E1DE
:1016800017D2010A01E1D3D1040A01E11AD3070AF2
:1016900001E00CD3D9500C0FE96E000EDA20EA6E8F
:1016A000EE50ED1001E032D1250E0CC2E9FF0DC263
:1016B000EAFFEF6E010E0201EA6A0C25E96E0D5198
:1016C000EA220C0EEF6EE66AE668E6680CC2E6FFF8
:1016D0000DC2E6FF0FC2E6FF10C2E6FFAEEC43F01C
:1016E000146E070EE15C02E2E16AE552E16E14500D
:1016F000230E0CC2E9FF0DC2EAFFEF6EE66AE66850
:10170000E6680CC2E6FF0DC2E6FF0FC2E6FF10C29C
:10171000E6FFAEEC43F0146E070EE15C02E2E16A14
:10172000E552E16E1450240E0CC2E9FF0DC2EAFF2F
:10173000EF6EE66AE668E6680CC2E6FF0DC2E6FFF9
:101740000FC2E6FF10C2E6FFAEEC43F0146E070EC8
:10175000E15C02E2E16AE552E16E1450210E0CC236
:10176000E9FF0DC2EAFFEF6E520EE66EDA0EE66E8C
:10177000000EE66E010E0201156A0C25146E0D5165
:10178000152214C0E6FF15C0E6FFF4EC6EF0166EED
:10179000050EE15C02E2E16AE552E16E1650E66A8E
:1017A000E668E6680CC2E6FF0DC2E6FF0FC2E6FF80
:1017B00010C2E6FFAEEC43F0146E070EE15C02E2ED
:1017C000E16AE552E16E1450400E0CC2E9FF0DC211
:1017D000EAFFEF6E460EE66EDA0EE66E000EE66E7D
:1017E000010E0201156A0C25146E0D51152214C04C
:1017F000E6FF15C0E6FFF4EC6EF0166E050EE15C38
:1018000002E2E16AE552E16E1650010EE76EFC0E4F
:10181000DBCF14F0FD0EDBCF15F0E7501426000EE1
:101820001522300E1412000E1512070E0201EA6A7C
:101830000C25E96E0D51EA2214C0EFFFE66AE66856
:10184000E6680CC2E6FF0DC2E6FF0FC2E6FF10C25B
:10185000E6FFAEEC43F0146E070EE15C02E2E16AD3
:10186000E552E16E1450E66AE668E668D950040F66
:10187000E66E000EDA20E66E11C2E6FF12C2E6FF47
:1018800093EC47F0146E070EE15C02E2E16AE55268
:10189000E16E1450000903E123EC59F0E4D7040E83
:1018A000DB50060864E1FC0EDBCFE9FFFD0EDBCF69
:1018B000EAFF030ED890E936EA36E806FBE1FD0EB2
:1018C000E926020EEA22EE52EF6AFC0EDBCF08F0A8
:1018D000FD0EDBCF09F0030E081801E1095014E0FA
:1018E000020E081801E109500DE0010E081801E18F
:1018F000095006E008503BE1095039E18D9037D09E
:101900008D9235D08D9433D08D9631D0FC0EDBCFB7
:10191000E9FFFD0EDBCFEAFF030ED890E936EA3689
:10192000E806FBE1FD0EE926020EEA22EE52EFCFB9
:1019300014F0010EE76E1418E8AE02D0143403D090
:10194000E750D880145413E3FC0EDBCFE9FFFD0E03
:10195000DBCFEAFF030ED890E936EA36E806FBE172
:10196000FD0EE926020EEA22EE52010EEF6EFC0E8B
:10197000DBCFE9FFFD0EDBCFEAFF030ED890E9369F
:10198000EA36E806FBE1FD0EE926020EEA220C0E1D
:10199000DBCFEFFFFC0EDBCFE9FFFD0EDBCFEAFF75
:1019A000030ED890E936EA36E806FBE1FD0EE9269B
:1019B000020EEA22020EE926000EEA220E0EDBCF0C
:1019C000EFFFFC0EDBCFE9FFFD0EDBCFEAFF030EDE
:1019D000D890E936EA36E806FBE1FD0EE926020E6C
:1019E000EA22020EE926000EEA22EE520F0EDBCFAB
:1019F000EFFFFC0EDBCFE9FFFD0EDBCFEAFF030EAE
:101A0000D890E936EA36E806FBE1FD0EE926020E3B
:101A1000EA22020EE926000EEA22020EE926000E54
:101A2000EA22100EDBCFEFFF8FEC36F04AD1080E22
:101A3000DB06090E01E2DB06DBCF15F0800E151484
:101A400007E0030EF36E080EF3CFDBFF090EDB6A2F
:101A5000250E0CC2E9FF0DC2EAFFEF6ED9CF14F0DC
:101A6000DACF15F0080EDB50D924E96E090EDB50F1
:101A7000DA20EA6EEF50E66E010E0201EA6A0C25EA
:101A8000E96E0D51EA22E552E750EF6EE66AE6682C
:101A9000E6680CC2E6FF0DC2E6FF0FC2E6FF10C209
:101AA000E6FFAEEC43F0146E070EE15C46E243D075
:101AB000080EDB2ADBCF14F0090E01E3DB2ADBCFB3
:101AC00015F0153409E214500308000E155404E211
:101AD000080EDB6A090EDB6A250E0CC2E9FF0DC297
:101AE000EAFFEF6ED9CF14F0DACF15F0080EDB5015
:101AF000D924E96E090EDB50DA20EA6EEF50E66E6B
:101B0000010E0201EA6A0C25E96E0D51EA22E55246
:101B1000E750EF6EE66AE668E6680CC2E6FF0DC2C3
:101B2000E6FF0FC2E6FF10C2E6FFAEEC43F0146E14
:101B3000070EE15C02E2E16AE552E16E1450B6D0B4
:101B4000080EDBCF08F0090EDBCF09F0030E0818F2
:101B500001E109503BE0020E081801E109502CE0B8
:101B6000010E081801E109501CE0085001E09BD06B
:101B7000095001E098D00C0EDB06DBCF14F00D0EFF
:101B800001E2DB06DBCF15F00001800E151401E148
:101B90008AD0020EF36E0C0EF3CFDBFF0D0EDB6A64
:101BA00082D00E0EDB06DBCF14F0143401E27BD0C2
:101BB000170EF36E0E0E13D00F0EDB06DBCF14F0F4
:101BC000143471E33B0EF36E0F0E09D0100EDB06DA
:101BD000DBCF14F0143467E33B0EF36E100EF3CF3B
:101BE000DBFF61D0080EDBCF08F0090EDBCF09F078
:101BF000030E081801E1095045E0020E081801E142
:101C000009502FE0010E081801E1095019E00850B1
:101C10004AE1095048E10C0EDB2ADBCF14F00D0E2F
:101C200001E3DB2ADBCF15F0D890155004E6030E54
:101C3000145C000E155837E30C0EDB6A0D0E32D023
:101C40000E0EDB2ADBCF14F0170EE76E1418E8AE89
:101C500002D0143403D0E750D880145424E20E0E7E
:101C600021D00F0EDB2ADBCF14F03B0EE76E1418E9
:101C7000E8AE02D0143403D0E750D880145413E2F5
:101C80000F0E10D0100EDB2ADBCF14F03B0EE76EE8
:101C90001418E8AE02D0143403D0E750D88014549E
:101CA00002E2100EDB6A050EDB6A05D0010EF36E50
:101CB000050EF3CFDBFF050EDB5001E0BDD440EF96
:101CC00009F0250E0CC2E9FF0DC2EAFFEF6E010E0E
:101CD0000201EA6A0C25E96E0D51EA220C0EEF6E44
:101CE000E66AE668E6680CC2E6FF0DC2E6FF0FC2D0
:101CF000E6FF10C2E6FFAEEC43F0146E070EE15CA7
:101D000002E2E16AE552E16E14500201010ED86F61
:101D10000201D96B040EDB50146E110EE15C02E27D
:101D2000E16AE552E16E1450E552E5CFDAFFE7CF04
:101D3000D9FF1200D9CFE6FFDACFE6FFE1CFD9FF16
:101D4000E2CFDAFF0E0EE12402E3E168E652E16E33
:101D5000880EDF6EDE528B0EDD6E8E0EF36E020E7F
:101D6000F3CFDBFF010EE76EFC0EDBCF14F0FD0EB0
:101D7000DBCF15F0E7501426000E1522050E14C017
:101D8000DBFF060E15C0DBFF070EDB6A080EDB6A01
:101D9000090EDB6A0A0EDB6A0201010ED96FFC0E26
:101DA000DBCFE9FFFD0EDBCFEAFF030ED890E9366B
:101DB000EA36E806FBE1FD0EE926020EEA22050EF0
:101DC000E926000EEA220B0EEFCFDBFFFC0EDBCF85
:101DD000E9FFFD0EDBCFEAFF030ED890E936EA36C5
:101DE000E806FBE1FD0EE926020EEA22050EE926D1
:101DF000000EEA22EE520C0EEFCFDBFFFC0EDBCF23
:101E0000E9FFFD0EDBCFEAFF030ED890E936EA3694
:101E1000E806FBE1FD0EE926020EEA22050EE926A0
:101E2000000EEA22020EE926000EEA220D0EEFCF86
:101E3000DBFF250E0CC2E9FF0DC2EAFFEF6E010EBB
:101E40000201EA6A0C25E96E0D51EA220E0EEF6ED0
:101E5000E66AE668E6680CC2E6FF0DC2E6FF0FC25E
:101E6000E6FF10C2E6FFAEEC43F0146E070EE15C35
:101E700002E2E16AE552E16E1450100EE66EE66A87
:101E8000200EE66E0CC2E6FF0DC2E6FFA8EC6EF077
:101E9000146E050EE15C02E2E16AE552E16E145057
:101EA000210E0CC2E9FF0DC2EAFFEF6E7F0EE66E57
:101EB000DA0EE66E000EE66E010E0201156A0C25C2
:101EC000146E0D51152214C0E6FF15C0E6FFF4ECA8
:101ED0006EF0166E050EE15C02E2E16AE552E16E1B
:101EE00016500F0EE76E050EDBCF14F0060EE7500E
:101EF0001416156A300E1412000E1512030E02018C
:101F0000EA6A0C25E96E0D51EA2214C0EFFF0A0EB1
:101F1000146E0E6E0B0EDBCF09F009EC71F0095058
:101F20003009E66E090E0201EA6A0C25E96E0D51D0
:101F3000EA22E552E750EF6E0B0EDBCF14F014C02F
:101F400009F00A0E0E6E09EC71F005503009E66ECC
:101F50000A0E0201EA6A0C25E96E0D51EA22E552E9
:101F6000E750EF6E0B0EEA6A0C25E96E0D51EA227E
:101F70003A0EEF6E0A0E146E0E6E0C0EDBCF09F0E9
:101F800009EC71F009503009E66E0C0E0201EA6AA4
:101F90000C25E96E0D51EA22E552E750EF6E0C0E6A
:101FA000DBCF14F014C009F00A0E0E6E09EC71F0CC
:101FB00005503009E66E0D0E0201EA6A0C25E96E45
:101FC0000D51EA22E552E750EF6E0E0EEA6A0C253B
:101FD000E96E0D51EA223A0EEF6E0A0E146E0E6E85
:101FE0000D0EDBCF09F009EC71F009503009E66EF7
:101FF0000F0E0201EA6A0C25E96E0D51EA22E55244
:10200000E750EF6E0D0EDBCF14F014C009F00A0E8E
:102010000E6E09EC71F005503009E66E100E0201EB
:10202000EA6A0C25E96E0D51EA22E552E750EF6E9F
:10203000E66AE668E6680CC2E6FF0DC2E6FF0FC27C
:10204000E6FF10C2E6FFAEEC43F0146E070EE15C53
:1020500002E2E16AE552E16E1450100EE66EE66AA5
:10206000200EE66E0CC2E6FF0DC2E6FFA8EC6EF095
:10207000146E050EE15C02E2E16AE552E16E145075
:10208000400E0CC2E9FF0DC2EAFFEF6E630EE66E72
:10209000DA0EE66E000EE66E010E0201156A0C25E0
:1020A000146E0D51152214C0E6FF15C0E6FFF4ECC6
:1020B0006EF0166E050EE15C02E2E16AE552E16E39
:1020C0001650E66AE668E6680CC2E6FF0DC2E6FF57
:1020D0000FC2E6FF10C2E6FFAEEC43F0146E070E2F
:1020E000E15C02E2E16AE552E16E1450250E0CC299
:1020F000E9FF0DC2EAFFEF6ED9CF14F0DACF15F089
:10210000070EDB50D924E96E080EDB50DA20EA6EA8
:10211000EF50E66E010E0201EA6A0C25E96E0D51E0
:10212000EA22E552E750EF6EE66AE668E6680CC21E
:10213000E6FF0DC2E6FF0FC2E6FF10C2E6FFAEECFF
:1021400043F0146E070EE15C02E2E16AE552E16ED3
:102150001450E66AE668E668D950030FE66E000E92
:10216000DA20E66E11C2E6FF12C2E6FF93EC47F0FA
:10217000146E070EE15C02E2E16AE552E16E145072
:10218000000901E16CD1030EDB50040A01E118D112
:10219000010A01E1E1D0060A01E196D0010A53E00B
:1021A000040A01E161D1070A01E054D1FC0EDBCF42
:1021B000E9FFFD0EDBCFEAFF030ED890E936EA36E1
:1021C000E806FBE1FD0EE926020EEA22050EE926ED
:1021D000000EEA220B0EDBCFEFFFFC0EDBCFE9FF98
:1021E000FD0EDBCFEAFF030ED890E936EA36E806AB
:1021F000FBE1FD0EE926020EEA22050EE926000E9D
:10220000EA22EE520C0EDBCFEFFFFC0EDBCFE9FF34
:10221000FD0EDBCFEAFF030ED890E936EA36E8067A
:10222000FBE1FD0EE926020EEA22050EE926000E6C
:10223000EA22020EE926000EEA220D0EDBCFEFFFA6
:102240008FEC36F011D1070EDB06080E01E2DB063B
:10225000DBCF15F0800E151407E0020EF36E070EAB
:10226000F3CFDBFF080EDB6A250E0CC2E9FF0DC2BF
:10227000EAFFEF6ED9CF14F0DACF15F0070EDB507E
:10228000D924E96E080EDB50DA20EA6EEF50E66ED4
:10229000010E0201EA6A0C25E96E0D51EA22E552AF
:1022A000E750EF6EE66AE668E6680CC2E6FF0DC22C
:1022B000E6FF0FC2E6FF10C2E6FFAEEC43F0146E7D
:1022C000070EE15C46E243D0070EDB2ADBCF14F0B9
:1022D000080E01E3DB2ADBCF15F0153409E21450B8
:1022E0000208000E155404E2070EDB6A080EDB6AD2
:1022F000250E0CC2E9FF0DC2EAFFEF6ED9CF14F034
:10230000DACF15F0070EDB50D924E96E080EDB504A
:10231000DA20EA6EEF50E66E010E0201EA6A0C2541
:10232000E96E0D51EA22E552E750EF6EE66AE66883
:10233000E6680CC2E6FF0DC2E6FF0FC2E6FF10C260
:10234000E6FFAEEC43F0146E070EE15C02E2E16AD8
:10235000E552E16E14507ED0070EDBCF08F0080E78
:10236000DBCF09F0020E081801E109501DE0010E53
:10237000081801E109500EE0085069E1095067E1D1
:102380000B0EDB06DBCF14F0143461E3170EF36E93
:102390000B0E13D00C0EDB06DBCF14F0143457E316
:1023A0003B0EF36E0C0E09D00D0EDB06DBCF14F0E6
:1023B00014344DE33B0EF36E0D0EF3CFDBFF47D02D
:1023C000070EDBCF08F0080EDBCF09F0020E08186D
:1023D00001E109502BE0010E081801E1095015E058
:1023E000085035E1095033E10B0EDB2ADBCF14F046
:1023F000170EE76E1418E8AE02D0143403D0E7507D
:10240000D880145424E20B0E21D00C0EDB2ADBCF33
:1024100014F03B0EE76E1418E8AE02D0143403D06B
:10242000E750D880145413E20C0E10D00D0EDB2AA6
:10243000DBCF14F03B0EE76E1418E8AE02D0143474
:1024400003D0E750D880145402E20D0EDB6A040E6C
:10245000DB6A05D0010EF36E040EF3CFDBFF040E32
:10246000DB5001E076D609D5250E0CC2E9FF0DC27E
:10247000EAFFEF6E010E0201EA6A0C25E96E0D51CA
:10248000EA220C0EEF6EE66AE668E6680CC2E6FF2A
:102490000DC2E6FF0FC2E6FF10C2E6FFAEEC43F04E
:1024A000146E070EE15C02E2E16AE552E16E14503F
:1024B0000201010ED86F0201D96B030EDB50146EBE
:1024C0000E0EE15C02E2E16AE552E16E1450E55263
:1024D000E5CFDAFFE7CFD9FF1200D9CFE6FFDACF99
:1024E000E6FFE1CFD9FFE2CFDAFFE652E652FC0E7B
:1024F000DBCF14F0FD0EDBCF15F0010E1424DF6EE0
:102500000201010ED96F230E0CC2E9FF0DC2EAFFD2
:10251000EF6EE66AE668E6680CC2E6FF0DC2E6FF0B
:102520000FC2E6FF10C2E6FFAEEC43F0146E070EDA
:10253000E15C02E2E16AE552E16E1450240E0CC245
:10254000E9FF0DC2EAFFEF6EE66AE668E6680CC2D4
:10255000E6FF0DC2E6FF0FC2E6FF10C2E6FFAEECDB
:1025600043F0146E070EE15C02E2E16AE552E16EAF
:102570001450210E0CC2E9FF0DC2EAFFEF6E010EEE
:102580000201EA6A0C25E96E0D51EA223A0EEF6E5D
:10259000360EE66EDA0EE66E000EE66E020E156A76
:1025A0000C25146E0D51152214C0E6FF15C0E6FF70
:1025B000F4EC6EF0166E050EE15C02E2E16AE552A3
:1025C000E16E16500F0EDF143009E66E0E0E02019A
:1025D000EA6A0C25E96E0D51EA22E552E750EF6EEA
:1025E000E66AE668E6680CC2E6FF0DC2E6FF0FC2C7
:1025F000E6FF10C2E6FFAEEC43F0146E070EE15C9E
:1026000002E2E16AE552E16E1450400E0CC2E9FFAD
:102610000DC2EAFFEF6E2D0EE66EDA0EE66E000ECC
:10262000E66E010E0201156A0C25146E0D5115227D
:1026300014C0E6FF15C0E6FFF4EC6EF0166E050E52
:10264000E15C02E2E16AE552E16E1650E66AE66894
:10265000E6680CC2E6FF0DC2E6FF0FC2E6FF10C23D
:10266000E6FFAEEC43F0146E070EE15C02E2E16AB5
:10267000E552E16E1450E66AE668E668D950010F4B
:10268000E66E000EDA20E66E11C2E6FF12C2E6FF29
:1026900093EC47F0146E070EE15C02E2E16AE5524A
:1026A000E16E1450000901E164D7010EDB50030A0A
:1026B00007E0010A05E0030A03E0070A01E059D731
:1026C0000201010ED86F0201D96BDB50E552E552D1
:1026D000E552E5CFDAFFE7CFD9FF1200D9CFE6FF09
:1026E000DACFE6FFE1CFD9FFE2CFDAFFE65202010F
:1026F000010ED96F230E0CC2E9FF0DC2EAFFEF6E87
:10270000E66AE668E6680CC2E6FF0DC2E6FF0FC2A5
:10271000E6FF10C2E6FFAEEC43F0146E070EE15C7C
:1027200002E2E16AE552E16E1450210E0CC2E9FFAB
:102730000DC2EAFFEF6E010E0201EA6A0C25E96E96
:102740000D51EA223A0EEF6E61C3E6FF62C3E6FF67
:1027500063C3E6FF020E156A0C25146E0D51152297
:1027600014C0E6FF15C0E6FFF4EC6EF0166E050E21
:10277000E15C02E2E16AE552E16E1650E66AE66863
:10278000E6680CC2E6FF0DC2E6FF0FC2E6FF10C20C
:10279000E6FFAEEC43F0146E070EE15C02E2E16A84
:1027A000E552E16E1450240E0CC2E9FF0DC2EAFF9F
:1027B000EF6EE66AE668E6680CC2E6FF0DC2E6FF69
:1027C0000FC2E6FF10C2E6FFAEEC43F0146E070E38
:1027D000E15C02E2E16AE552E16E1450400E0CC287
:1027E000E9FF0DC2EAFFEF6E1C0EE66EDA0EE66E32
:1027F000000EE66E010E0201156A0C25146E0D51D5
:10280000152214C0E6FF15C0E6FFF4EC6EF0166E5C
:10281000050EE15C02E2E16AE552E16E1650E66AFD
:10282000E668E6680CC2E6FF0DC2E6FF0FC2E6FFEF
:1028300010C2E6FFAEEC43F0146E070EE15C02E25C
:10284000E16AE552E16E1450E66AE668E668D9CFBF
:10285000E6FFDACFE6FF11C2E6FF12C2E6FF93EC15
:1028600047F0146E070EE15C02E2E16AE552E16EA8
:102870001450000998E0DF50050A0AE0010A08E058
:10288000070A06E0010A04E0030A02E0070A8BE1F6
:102890000201010ED86F0201D96BDF50E552E552FB
:1028A000E5CFDAFFE7CFD9FF1200D9CFE6FFDACFC5
:1028B000E6FFE1CFD9FFE2CFDAFFE652E652E65279
:1028C000E652E652C20EF36E030EF3CFDBFFC60EE6
:1028D000F36E040EF3CFDBFF0201010ED96F250E5C
:1028E0000CC2E9FF0DC2EAFFEF6E010E0201EA6AB7
:1028F0000C25E96E0D51EA220E0EEF6EE66AE668CF
:10290000E6680CC2E6FF0DC2E6FF0FC2E6FF10C28A
:10291000E6FFAEEC43F0146E070EE15C02E2E16A02
:10292000E552E16E1450230E0CC2E9FF0DC2EAFF1E
:10293000EF6EE66AE668E6680CC2E6FF0DC2E6FFE7
:102940000FC2E6FF10C2E6FFAEEC43F0146E070EB6
:10295000E15C02E2E16AE552E16E1450210E0CC224
:10296000E9FF0DC2EAFFEF6E010E0201EA6A0C25D3
:10297000E96E0D51EA223A0EEF6E64C3E6FF65C3BD
:10298000E6FF66C3E6FF020E156A0C25146E0D51B4
:10299000152214C0E6FF15C0E6FFF4EC6EF0166ECB
:1029A000050EE15C02E2E16AE552E16E1650E66A6C
:1029B000E668E6680CC2E6FF0DC2E6FF0FC2E6FF5E
:1029C00010C2E6FFAEEC43F0146E070EE15C02E2CB
:1029D000E16AE552E16E1450240E0CC2E9FF0DC20B
:1029E000EAFFEF6EE66AE668E6680CC2E6FF0DC233
:1029F000E6FF0FC2E6FF10C2E6FFAEEC43F0146E36
:102A0000070EE15C02E2E16AE552E16E1450400E0D
:102A10000CC2E9FF0DC2EAFFEF6E130EE66EDA0E8E
:102A2000E66E000EE66E010E0201156A0C25146EAC
:102A30000D51152214C0E6FF15C0E6FFF4EC6EF050
:102A4000166E050EE15C02E2E16AE552E16E165097
:102A5000E66AE668E6680CC2E6FF0DC2E6FF0FC252
:102A6000E6FF10C2E6FFAEEC43F0146E070EE15C29
:102A700002E2E16AE552E16E1450FC0EDBCFE9FFA1
:102A8000FD0EDBCFEAFF020EEFCFDBFF250E0CC2FF
:102A9000E9FF0DC2EAFFEF6ED950030F146E000E6E
:102AA000DA20156E020EDBCF16F0176A16BE176815
:102AB00014501624E96E15501720EA6EEF50E66E9A
:102AC000010E0201EA6A0C25E96E0D51EA22E55277
:102AD000E750EF6EE66AE668E6680CC2E6FF0DC2F4
:102AE000E6FF0FC2E6FF10C2E6FFAEEC43F0146E45
:102AF000070EE15C02E2E16AE552E16E1450E66A1B
:102B0000E668E668D9CFE6FFDACFE6FF11C2E6FF56
:102B100012C2E6FF93EC47F0146E070EE15C02E28E
:102B2000E16AE552E16E1450000936E0DF50030A15
:102B30001CE0010A0EE0040A33E0070A2AE1FC0E59
:102B4000DBCFE9FFFD0EDBCFEAFF020EDBCFEFFFAD
:102B500027D0020EDB06DBCF14F0143417E3010E8E
:102B6000F36E020EF3CFDBFF11D0020EDB2ADBCFB8
:102B700014F0010EE76E1418E8AE02D0143403D03E
:102B8000E750D880145402E2020EDB6A010EDB6AC1
:102B900003D0DE52010EDD6E010EDB50B0E176D7C0
:102BA000250E0CC2E9FF0DC2EAFFEF6E010E020115
:102BB000EA6A0C25E96E0D51EA220C0EEF6EE66A08
:102BC000E668E6680CC2E6FF0DC2E6FF0FC2E6FF4C
:102BD00010C2E6FFAEEC43F0146E070EE15C02E2B9
:102BE000E16AE552E16E14500201010ED86F020154
:102BF000D96BDF50146E050EE15C02E2E16AE5522A
:102C0000E16E1450E552E5CFDAFFE7CFD9FF1200AD
:102C1000D9CFE6FFDACFE6FFE1CFD9FFE2CFDAFF87
:102C2000E652E652E652E652E652010EF36E020E0C
:102C3000F3CFDBFFC20EF36E030EF3CFDBFFC60E46
:102C4000F36E040EF3CFDBFF0201010ED96F250EE8
:102C50000CC2E9FF0DC2EAFFEF6E010E0201EA6A43
:102C60000C25E96E0D51EA220E0EEF6EE66AE6685B
:102C7000E6680CC2E6FF0DC2E6FF0FC2E6FF10C217
:102C8000E6FFAEEC43F0146E070EE15C02E2E16A8F
:102C9000E552E16E1450230E0CC2E9FF0DC2EAFFAB
:102CA000EF6EE66AE668E6680CC2E6FF0DC2E6FF74
:102CB0000FC2E6FF10C2E6FFAEEC43F0146E070E43
:102CC000E15C02E2E16AE552E16E1450240E0CC2AE
:102CD000E9FF0DC2EAFFEF6EE66AE668E6680CC23D
:102CE000E6FF0DC2E6FF0FC2E6FF10C2E6FFAEEC44
:102CF00043F0146E070EE15C02E2E16AE552E16E18
:102D00001450210E0CC2E9FF0DC2EAFFEF6E030E54
:102D1000E66EDA0EE66E000EE66E010E0201156A30
:102D20000C25146E0D51152214C0E6FF15C0E6FFE8
:102D3000F4EC6EF0166E050EE15C02E2E16AE5521B
:102D4000E16E1650E66AE668E6680CC2E6FF0DC260
:102D5000E6FF0FC2E6FF10C2E6FFAEEC43F0146ED2
:102D6000070EE15C02E2E16AE552E16E1450400EAA
:102D70000CC2E9FF0DC2EAFFEF6EFA0EE66ED90E45
:102D8000E66E000EE66E010E0201156A0C25146E49
:102D90000D51152214C0E6FF15C0E6FFF4EC6EF0ED
:102DA000166E050EE15C02E2E16AE552E16E165034
:102DB000E66AE668E6680CC2E6FF0DC2E6FF0FC2EF
:102DC000E6FF10C2E6FFAEEC43F0146E070EE15CC6
:102DD00002E2E16AE552E16E1450250E0CC2E9FFF1
:102DE0000DC2EAFFEF6ED950030F146E000EDA2009
:102DF000156E020EDBCF16F0176A16BE1768145058
:102E00001624E96E15501720EA6EEF50E66E010E9B
:102E10000201EA6A0C25E96E0D51EA22E552E750FB
:102E2000EF6EE66AE668E6680CC2E6FF0DC2E6FFF2
:102E30000FC2E6FF10C2E6FFAEEC43F0146E070EC1
:102E4000E15C02E2E16AE552E16E1450E66AE6688E
:102E5000E668D9CFE6FFDACFE6FF11C2E6FF12C27D
:102E6000E6FF93EC47F0146E070EE15C02E2E16AC4
:102E7000E552E16E1450000933E0DF50030A19E017
:102E8000010A0BE0040A03E0070A2EE026D0010E37
:102E9000F36E020EF3CFDBFF27D0020EDB06DBCF93
:102EA00014F0143417E3010EF36E020EF3CFDBFFC0
:102EB00011D0020EDB2ADBCF14F0010EE76E1418DE
:102EC000E8AE02D0143403D0E750D880145402E2A4
:102ED000020EDB6A010EDB6A03D0DE52010EDD6EEC
:102EE000010EDB50B3E179D7250E0CC2E9FF0DC20C
:102EF000EAFFEF6E010E0201EA6A0C25E96E0D5140
:102F0000EA220C0EEF6EE66AE668E6680CC2E6FF9F
:102F10000DC2E6FF0FC2E6FF10C2E6FFAEEC43F0C3
:102F2000146E070EE15C02E2E16AE552E16E1450B4
:102F30000201010ED86F0201D96B020EDB5002E1D3
:102F4000010E01D0000E146E050EE15C02E2E16A92
:102F5000E552E16E1450E552E5CFDAFFE7CFD9FF35
:102F60001200D9CFE6FFDACFE6FFE1CFD9FFE2CFFB
:102F7000DAFF070EE12402E3E168E652E16EFC0E9F
:102F8000DBCFE9FFFD0EDBCFEAFF040EEFCFDBFF67
:102F90000201010ED96F250E0CC2E9FF0DC2EAFF36
:102FA000EF6E010E0201EA6A0C25E96E0D51EA226C
:102FB0000C0EEF6EE66AE668E6680CC2E6FF0DC22C
:102FC000E6FF0FC2E6FF10C2E6FFAEEC43F0146E60
:102FD000070EE15C02E2E16AE552E16E1450230E55
:102FE0000CC2E9FF0DC2EAFFEF6EE66AE668E6682A
:102FF0000CC2E6FF0DC2E6FF0FC2E6FF10C2E6FFFD
:10300000AEEC43F0146E070EE15C02E2E16AE552B9
:10301000E16E1450210E0CC2E9FF0DC2EAFFEF6E03
:10302000010E0201EA6A0C25E96E0D51EA223A0E00
:10303000EF6E5EC3E6FF5FC3E6FF60C3E6FF020E0E
:10304000156A0C25146E0D51152214C0E6FF15C02B
:10305000E6FFF4EC6EF0166E050EE15C02E2E16A4A
:10306000E552E16E1650E66AE668E6680CC2E6FFD5
:103070000DC2E6FF0FC2E6FF10C2E6FFAEEC43F062
:10308000146E070EE15C02E2E16AE552E16E145053
:103090007E0E176EE30E186E000E196E040EDBCF57
:1030A0001AF01B6A1C6A1AAE02D01B681C68050E57
:1030B0000C6E0D6A0E6A1AC007F01BC008F01CC027
:1030C00009F076EC71F004C01AF005C01BF006C0E0
:1030D0001CF017500424146E18500520156E19505A
:1030E0000620166E010E14C0DBFF020E15C0DBFFBA
:1030F000030E16C0DBFF240E0CC2E9FF0DC2EAFF6F
:10310000EF6EE66AE668E6680CC2E6FF0DC2E6FF0F
:103110000FC2E6FF10C2E6FFAEEC43F0146E070EDE
:10312000E15C02E2E16AE552E16E1450070EE66EE0
:10313000E66A200EE66E020E0201156A0C25146E78
:103140000D51152214C0E6FF15C0E6FFA8EC6EF085
:10315000166E050EE15C02E2E16AE552E16E165080
:10316000400E0CC2E9FF0DC2EAFFEF6E010E020134
:10317000EA6A0C25E96E0D51EA223E0EEF6E010E51
:10318000DBCFF6FF020EDBCFF7FF030EDBCFF8FF3E
:103190000900F5CFE6FF0900F5CFE6FF0800F5CFFF
:1031A000E6FF020E156A0C25146E0D51152214C08F
:1031B000E6FF15C0E6FFF4EC6EF0166E050EE15C5E
:1031C00002E2E16AE552E16E1650010EDBCFF6FF36
:1031D000020EDBCFF7FF030EDBCFF8FF0900F5CFC0
:1031E000E6FF0900F5CFE6FF0800F5CFE6FF1BEC90
:1031F0006FF0E552E552E552060E07C0DBFFDB50EB
:10320000020F146E156A14BE156802010C511424C5
:10321000E96E0D511520EA6E200EEF6EF30EE66E8C
:10322000D90EE66E000EE66E090E156A0C25146EB8
:103230000D51152214C0E6FF15C0E6FFF4EC6EF048
:10324000166E050EE15C02E2E16AE552E16E16508F
:10325000010EDBCFF6FF020EDBCFF7FF030EDBCF55
:10326000F8FFF626000EF722F8220800050EF5CF2B
:10327000DBFFDBCF14F014340FE3050EDB50FF0D42
:10328000050EF3CFDBFF090E0201EA6A0C25E96E99
:103290000D51EA222D0EEF6E0A0E146E0E6E050E03
:1032A000DBCF09F009EC71F009503009E66E0A0E27
:1032B0000201EA6A0C25E96E0D51EA22E552E75057
:1032C000EF6E050EDBCF14F014C009F00A0E0E6E7F
:1032D00009EC71F005503009E66E0B0E0201EA6A46
:1032E0000C25E96E0D51EA22E552E750EF6E010E12
:1032F000DBCFF6FF020EDBCFF7FF030EDBCFF8FFCD
:10330000040EF626000EF722F8220800F5CF14F07E
:103310000A0E156E0E6E14C009F009EC71F009501A
:103320003009E66E0D0E0201EA6A0C25E96E0D51B8
:10333000EA22E552E750EF6E010EDBCFF6FF020EF8
:10334000DBCFF7FF030EDBCFF8FF040EF626000EEF
:10335000F722F8220800F5CF14F014C009F00A0E85
:103360000E6E09EC71F005503009E66E0E0E02018A
:10337000EA6A0C25E96E0D51EA22E552E750EF6E3C
:10338000E66AE668E6680CC2E6FF0DC2E6FF0FC219
:10339000E6FF10C2E6FFAEEC43F0146E070EE15CF0
:1033A00002E2E16AE552E16E1450E66AE668E66818
:1033B000D9CFE6FFDACFE6FF11C2E6FF12C2E6FF81
:1033C00093EC47F0146E070EE15C02E2E16AE5520D
:1033D000E16E1450000901E15BD6DF50040A54E0AD
:1033E000010A44E0030A5FE0070A01E051D6010E3A
:1033F000DBCFF6FF020EDBCFF7FF030EDBCFF8FFCC
:10340000040EF626000EF722F8220800F5CF14F07D
:10341000156A14BE156814C0E6FF15C0E6FF010E5C
:10342000DBCFF6FF020EDBCFF7FF030EDBCFF8FF9B
:10343000F626000EF722F8220800F5CF16F0176ADC
:1034400016BE176816C0E6FF17C0E6FF8AEC1CF030
:10345000E552E552E552E552FC0EDBCFE9FFFD0EE9
:10346000DBCFEAFF040EDBCFEFFF1DD0040EDB063F
:10347000DBCF14F0143401E20BD603016A05E76ECA
:10348000040EE7CFDBFF04D6040EDB2A03016A51EA
:10349000F36E040EDBCFF4FFF350F45C01E2F8D5D9
:1034A000040EDB6AF5D50201010ED86F0201D96B5B
:1034B000DF50146E070EE15C02E2E16AE552E16E54
:1034C0001450E552E5CFDAFFE7CFD9FF1200D9CF8C
:1034D000E6FFDACFE6FFE1CFD9FFE2CFDAFFE6522F
:1034E000DF6ADFCF14F0040EE76E1418E8AE02D0E6
:1034F000E73402D0E750145C01E3AFD0DFCFE9FF3F
:10350000EA6AE9BEEA68030ED890E936EA36E806C8
:10351000FBE1FD0EE926020EEA22020EE926000E6C
:10352000EA22EFCF14F0DFCFE9FFEA6AE9BEEA68EA
:10353000030ED890E936EA36E806FBE1FD0EE926EF
:10354000020EEA22050EE926000EEA22EF50145C74
:1035500001E081D0DFCFE9FFEA6AE9BEEA68030E45
:10356000D890E936EA36E806FBE1FD0EE926020EC0
:10357000EA22020EE926000EEA22EE52EFCF15F003
:10358000DFCFE9FFEA6AE9BEEA68030ED890E936C0
:10359000EA36E806FBE1FD0EE926020EEA22050EF8
:1035A000E926000EEA22EE52EF50155C54E1DFCF1F
:1035B000E9FFEA6AE9BEEA68030ED890E936EA361E
:1035C000E806FBE1FD0EE926020EEA22020EE926DC
:1035D000000EEA22020EE926000EEA22EFCF16F0D4
:1035E000DFCFE9FFEA6AE9BEEA68030ED890E93660
:1035F000EA36E806FBE1FD0EE926020EEA22050E98
:10360000E926000EEA22020EE926000EEA22EF5019
:10361000165C21E1DFCFE9FFEA6AE9BEEA68030E42
:10362000D890E936EA36E806FBE1FD0EE926020EFF
:10363000EA22EF6ADFCFE9FFEA6AE9BEEA68030E31
:10364000D890E936EA36E806FBE1FD0EE926020EDF
:10365000EA22EE52EF6ADF2A44D7E552E552E5CF7F
:10366000DAFFE7CFD9FF1200D9CFE6FFDACFE6FFC6
:10367000E1CFD9FFE2CFDAFFE652E652E652FC0E86
:10368000DBCFE9FFFD0EDBCFEAFF020EEFCFDBFF62
:103690000201010ED96F250E0CC2E9FF0DC2EAFF2F
:1036A000EF6E010E0201EA6A0C25E96E0D51EA2265
:1036B0000C0EEF6EE66AE668E6680CC2E6FF0DC225
:1036C000E6FF0FC2E6FF10C2E6FFAEEC43F0146E59
:1036D000070EE15C02E2E16AE552E16E1450230E4E
:1036E0000CC2E9FF0DC2EAFFEF6EE66AE668E66823
:1036F0000CC2E6FF0DC2E6FF0FC2E6FF10C2E6FFF6
:10370000AEEC43F0146E070EE15C02E2E16AE552B2
:10371000E16E1450210E0CC2E9FF0DC2EAFFEF6EFC
:10372000E20EE66ED90EE66E000EE66E010E0201A6
:10373000156A0C25146E0D51152214C0E6FF15C034
:10374000E6FFF4EC6EF0166E050EE15C02E2E16A53
:10375000E552E16E1650E66AE668E6680CC2E6FFDE
:103760000DC2E6FF0FC2E6FF10C2E6FFAEEC43F06B
:10377000146E070EE15C02E2E16AE552E16E14505C
:10378000240E0CC2E9FF0DC2EAFFEF6EE66AE6689E
:10379000E6680CC2E6FF0DC2E6FF0FC2E6FF10C2EC
:1037A000E6FFAEEC43F0146E070EE15C02E2E16A64
:1037B000E552E16E1450400E0CC2E9FF0DC2EAFF63
:1037C000EF6E010E0201EA6A0C25E96E0D51EA2244
:1037D0003E0EEF6E020EDBCFE9FFEA6AE9BEEA6851
:1037E000030EEA02F3CFEAFFE902F3CFE9FFF45058
:1037F000EA265E0EE926030EEA22EECFE6FFEECFC2
:10380000E6FFEFCFE6FF020E156A0C25146E0D5190
:10381000152214C0E6FF15C0E6FFF4EC6EF0166E3C
:10382000050EE15C02E2E16AE552E16E1650E66ADD
:10383000E668E6680CC2E6FF0DC2E6FF0FC2E6FFCF
:1038400010C2E6FFAEEC43F0146E070EE15C02E23C
:10385000E16AE552E16E1450E66AE668E668D9CF9F
:10386000E6FFDACFE6FF11C2E6FF12C2E6FF93ECF5
:1038700047F0146E070EE15C02E2E16AE552E16E88
:103880001450000934E0DF50060A24E0030A0FE078
:10389000010A03E0050A28E11DD0020EDB06DBCF9A
:1038A00014F0143414E3020EF36EDB6E10D0020E2B
:1038B000DB2ADBCF14F0030EE76E1418E8AE02D05B
:1038C000E73402D0E750145C02E3020EDB6A010E1B
:1038D000DB6A0DD0FC0EDBCFE9FFFD0EDBCFEAFF8C
:1038E000020EDBCFEFFF07D0DE52010EDD6E010EC0
:1038F000DB50B2E145D70201010ED86F0201D96B4E
:10390000DF50E552E552E552E552E5CFDAFFE7CF69
:04391000D9FF1200C9
:0C391400D9CFE6FFDACFE6FFE1CFD9FF04
:10392000E2CFDAFF190EE12402E3E168E652E16E2C
:10393000B20EE66ED90EE66E000EE66ED9CFE6FF49
:10394000DACFE6FFF4EC6EF0146E050EE15C02E2F5
:10395000E16AE552E16E1450FC0EFD0EDBCF15F06E
:103960000001800E151405E12D0EF36E0B0EF3CF42
:10397000DBFFFC0EDBCF14F0FD0EDBCF15F00A0EE3
:103980000D6E0E6A14C008F015C009F023EC71F03A
:1039900008C014F009C015F0300E1412000E1512F4
:1039A0000C0E14C0DBFFFC0EDBCF14F0FD0EDBCFE2
:1039B00015F00A0E0D6E0E6A14C008F015C009F05D
:1039C00023EC71F004C014F005C015F0300E141291
:1039D000000E15120D0E14C0DBFFFA0EDBCF14F033
:1039E000FB0EDBCF15F00A0E0D6E0E6A14C008F048
:1039F00015C009F023EC71F008C014F009C015F0EF
:103A0000300E1412000E15120F0E14C0DBFFFA0E4A
:103A1000DBCF14F0FB0EDBCF15F00A0E0D6E0E6A35
:103A200014C008F015C009F023EC71F004C014F0C4
:103A300005C015F0300E1412000E1512100E14C031
:103A4000DBFFD9CFE6FFDACFE6FFA2EC70F0E5525C
:103A5000E552190EE15C02E2E16AE552E16EE552DF
:103A6000E5CFDAFFE7CFD9FF1200D9CFE6FFDACFF3
:103A7000E6FFE1CFD9FFE2CFDAFF0A0EE12402E34D
:103A8000E168E652E16E020EDB6A040EDB6A010EAB
:103A9000F36E050EF3CFDBFF7E0E176EE30E186E8E
:103AA000000E196E1FC31AF01B6A1C6A1AAE02D0F0
:103AB0001B681C68050E0C6E0D6A0E6A1AC007F0B2
:103AC0001BC008F01CC009F076EC71F004C01AF0BD
:103AD00005C01BF006C01CF017500424146E1850CB
:103AE0000520156E19500620166E060E14C0DBFF59
:103AF000070E15C0DBFF080E16C0DBFFFC0EDBCF88
:103B0000DEFFDBCFDDFF050EDB5002E1FAEF21F037
:103B1000DECFE9FFDDCFEAFFEF502C0A14E0210AE7
:103B20000FE0070A0DE00A0A0BE0DFCFE9FFDF2A0A
:103B3000010EDBCFEAFF02E2E9EF21F0E8EF21F02E
:103B4000050EDB6AE0D7020EDB50EA6A6A0FE96E07
:103B5000000EEA22EF6A040EDB50080A1FE00B0A8F
:103B600002E1DCEF21F0070A02E1DCEF21F0010ABB
:103B700002E1DCEF21F0030A02E1DCEF21F0010AAF
:103B800002E1DCEF21F0050A02E1DCEF21F0030A9B
:103B900002E1DCEF21F0010ADCEF21F0030EDB6A29
:103BA0000C0EF36E030EDBCFF4FFF350F45C1FE258
:103BB000030EDB50EA6A6A0FE96E000EEA22EFCFCD
:103BC00016F0176A16BE176816C0E6FF17C0E6FFA4
:103BD00094EC73F0E552E552F3CF14F0F4CF15F006
:103BE000F350F41001E1E8D3030EDB2AD9D70F0E0E
:103BF00000016B15166E0F0E6A15E96EEA6AE9BED2
:103C0000EA68F10EE926020EEA22EF501624146E3D
:103C1000156A14BE156814500201D21902E115503C
:103C2000D31902E0010ED86F0F0E00017115146E4A
:103C30000F0E7015E96EEA6AE9BEEA68F10EE92630
:103C4000020EEA22EF501424646F0F0E7315146EE7
:103C50000F0E7215E96EEA6AE9BEEA68F10EE9260E
:103C6000020EEA22EF501424656F0F0E7515146EC4
:103C70000F0E7415E96EEA6AE9BEEA68F10EE926EC
:103C8000020EEA22EF501424666F0201D40507E108
:103C900064C067F065C068F066C069F0D42BD85185
:103CA00006E1000164516511661101E0CAD10F0EF1
:103CB00000016B15146E0F0E6A15E96EEA6AE9BE13
:103CC000EA68F10EE926020EEA22EF5014240201FE
:103CD000D26FD36B800B01E0D3690F0E00016D151D
:103CE000146E0F0E6C15E96EEA6AE9BEEA68F10E11
:103CF000E926020EEA22EF501424606F616B800BFC
:103D000001E061690F0E6F15146E0F0E6E15E96EEE
:103D1000EA6AE9BEEA68F10EE926020EEA22EF50ED
:103D20001424626F636B800B01E06369613504E208
:103D300060510208000E615509E30201D207000E2E
:103D4000D35B0C0E00016027000E61230D0E086E80
:103D5000096A60C00DF061C00EF049EC71F006C058
:103D600018F007C019F0080E1826000E1922050ECB
:103D70000D6E0E6A18C008F019C009F023EC71F03E
:103D800008C018F009C019F0000162510824166E2D
:103D900063510920176ED2C220F0D3C221F0040E65
:103DA0000D6E0E6AD2C208F0D3C209F023EC71F096
:103DB00008C020F009C021F00201D25108241E6E73
:103DC000D35109201F6ED2C222F0D3C223F0640E59
:103DD0000D6E0E6AD2C208F0D3C209F023EC71F066
:103DE00008C022F009C023F008501E5C1C6E095068
:103DF0001F581D6ED2C224F0D3C225F0900E0D6E56
:103E0000010E0E6ED2C208F0D3C209F023EC71F09D
:103E100008C024F009C025F01C5008241A6E1D505B
:103E200009201B6E16501A24146E156A070E0D6EAB
:103E30000E6A14C008F015C009F023EC71F004C03C
:103E400014F005C015F004C0D7F20201D86B0001D0
:103E500061350CE260510C08000E615507E20C0E52
:103E6000605F000E615B0201D22BD3230201D951A6
:103E700001E0E7D0020E0301215D22E0210E0AC21B
:103E8000E9FF0BC2EAFFEF6EA10EE66ED90EE66EF9
:103E9000000EE66E010E0201156A0A25146E0B5122
:103EA000152214C0E6FF15C0E6FFF4EC6EF0166EA6
:103EB000050EE15C02E2E16AE552E16E1650ACD01B
:103EC000210E0AC2E9FF0BC2EAFFEF6E010E0201EA
:103ED000EA6A0A25E96E0B51EA22270EEF6E020EFE
:103EE000EA6A0A25E96E0B51EA226AC0EFFF030E67
:103EF000EA6A0A25E96E0B51EA226BC0EFFF040E55
:103F0000EA6A0A25E96E0B51EA222D0EEF6E050EC4
:103F1000EA6A0A25E96E0B51EA226CC0EFFF060E31
:103F2000EA6A0A25E96E0B51EA226DC0EFFF070E1F
:103F3000EA6A0A25E96E0B51EA222D0EEF6E080E91
:103F4000EA6A0A25E96E0B51EA226EC0EFFF090EFC
:103F5000EA6A0A25E96E0B51EA226FC0EFFF0A0EEA
:103F6000EA6A0A25E96E0B51EA22200EEF6E020181
:103F7000D751030DF3CFE9FFF4CFEAFFDC0EE926BA
:103F8000020EEA22EECFE6FFEECFE6FFEFCFE6FF2E
:103F90000B0E0201156A0A25146E0B51152214C06E
:103FA000E6FF15C0E6FFF4EC6EF0166E050EE15C60
:103FB00002E2E16AE552E16E16500E0E0201EA6A73
:103FC0000A25E96E0B51EA22200EEF6E0201D5514F
:103FD000EA6ACE0FE96E020EEA22EF50E66E0F0E8D
:103FE0000201EA6A0A25E96E0B51EA22E552E7501E
:103FF000EF6E0201D651EA6ACB0FE96E020EEA2299
:10400000EF50E66E100E0201EA6A0A25E96E0B51C6
:10401000EA22E552E750EF6EE66AE668E6680AC211
:10402000E6FF0BC2E6FF0FC2E6FF10C2E6FFAEECF2
:1040300043F0146E070EE15C02E2E16AE552E16EC4
:1040400014500201010EDA6F0001665115E1020100
:10405000DA830001655110E10201DA850001645143
:104060000BE10201DA87010E0001621905E1000E81
:10407000631902E10201DA89E66AE668E668DA0EA7
:10408000E66E020EE66E15C2E6FF16C2E6FFAEEC65
:1040900043F0146E070EE15C02E2E16AE552E16E64
:1040A00014500201D95101E087D1020E0301215DB4
:1040B0001EE0400E0AC2E9FF0BC2EAFFEF6E900E4F
:1040C000E66ED90EE66E000EE66E010E0201156A6E
:1040D0000A25146E0B51152214C0E6FF15C0E6FF29
:1040E000F4EC6EF0166E050EE15C76E273D01D51B5
:1040F00076E0400E0AC2E9FF0BC2EAFFEF6E010E46
:104100000201EA6A0A25E96E0B51EA2270C0EFFF4C
:10411000020EEA6A0A25E96E0B51EA2271C0EFFF2E
:10412000030EEA6A0A25E96E0B51EA223A0EEF6E97
:10413000040EEA6A0A25E96E0B51EA2272C0EFFF0B
:10414000050EEA6A0A25E96E0B51EA2273C0EFFFF9
:10415000060EEA6A0A25E96E0B51EA223A0EEF6E64
:10416000070EEA6A0A25E96E0B51EA2274C0EFFFD6
:10417000080EEA6A0A25E96E0B51EA2275C0EFFFC4
:10418000090EEA6A0A25E96E0B51EA22200EEF6E4B
:10419000060EDBCFF6FF070EDBCFF7FF080EDBCFF7
:1041A000F8FF0900F5CFE6FF0900F5CFE6FF0800AC
:1041B000F5CFE6FF0A0E156A0A25146E0B5115227B
:1041C00014C0E6FF15C0E6FFF4EC6EF0166E050EA7
:1041D000E15C02E2E16AE552E16E1650D8D00C0EC5
:1041E0000001E76E6419E8AE02D0643503D0E750F1
:1041F000D880645503E20C0E645D01D06451E76E13
:10420000090EE7CFDBFF400E0AC2E9FF0BC2EAFF4F
:10421000EF6E0A0E146E0E6E090EDBCF09F009EC7C
:1042200071F009503009E66E010E0201EA6A0A25B2
:10423000E96E0B51EA22E552E750EF6E090EDBCF33
:1042400014F014C009F00A0E0E6E09EC71F005505E
:104250003009E66E020E0201EA6A0A25E96E0B5188
:10426000EA22E552E750EF6E030EEA6A0A25E96E8C
:104270000B51EA223A0EEF6E040EEA6A0A25E96E45
:104280000B51EA2272C0EFFF050EEA6A0A25E96EB9
:104290000B51EA2273C0EFFF060EEA6A0A25E96EA7
:1042A0000B51EA223A0EEF6E070EEA6A0A25E96E12
:1042B0000B51EA2274C0EFFF080EEA6A0A25E96E84
:1042C0000B51EA2275C0EFFF090EEA6A0A25E96E72
:1042D0000B51EA222E0EEF6E0A0EEA6A0A25E96EEB
:1042E0000B51EA22200EEF6E0B0EEA6A0A25E96EE8
:1042F0000B51EA226D0EEF6E0C0EEA6A0A25E96E8A
:104300000B51EA22200EEF6E060EDBCFF6FF070EF2
:10431000DBCFF7FF080EDBCFF8FF0900F5CFE6FF94
:104320000900F5CFE6FF0800F5CFE6FF0D0E156A90
:104330000A25146E0B51152214C0E6FF15C0E6FFC6
:10434000F4EC6EF0166E050EE15C02E2E16AE552F5
:10435000E16E16500C0E0001E76E6419E8AE02D053
:10436000E73402D0E750645D09E20A0E0201EA6A0E
:104370000A25E96E0B51EA22610E08D00A0E0201ED
:10438000EA6A0A25E96E0B51EA22700EEF6EE66AC0
:10439000E668E6680AC2E6FF0BC2E6FF0FC2E6FF68
:1043A00010C2E6FFAEEC43F0146E070EE15C02E2D1
:1043B000E16AE552E16E1450020EDB6A040EDB2A5C
:1043C000DF2A010E02E283EF1DF0DB2A83EF1DF0EE
:1043D000DB2AEF50E66E020EDBCFF3FFDB2AF35051
:1043E000EA6A6A0FE96E000EEA22E552E750EF6EC4
:1043F00083EF1DF00A0EE15C02E2E16AE552E16E34
:10440000E552E5CFDAFFE7CFD9FF1200D9CFE6FFBB
:10441000DACFE6FFE1CFD9FFE2CFDAFFE652E6528C
:10442000E652E652E652020EDB6A030EDB6A010E2A
:10443000F36E040EF3CFDBFFFC0EDBCFDEFFDBCF32
:10444000DDFF040EDB5001E135D1DECFE9FFDDCF2A
:10445000EAFFEF502C0A12E0210A0DE0070A0BE0F8
:104460000A0A09E0DFCFE9FFDF2A010EDBCFEAFF0E
:1044700001E210D10ED1040EDB6AE3D7020EDB504D
:10448000EA6A6A0FE96E000EEA22EF6A030EDB5059
:10449000090A01E1F4D0010A01E1F1D00C0A01E1BD
:1044A000EED0070A01E1ADD0010A38E0030A01E1CC
:1044B000E6D0010A01E0E3D08A0EE66ED90EE66E80
:1044C000000EE66E6A0EE66E000EE66EDEEC6EF034
:1044D000146E050EE15C02E2E16AE552E16E1450F1
:1044E000000901E1CCD0840EE66ED90EE66E000E16
:1044F000E66E6A0EE66E000EE66EDEEC6EF0146E90
:10450000050EE15C02E2E16AE552E16E1450000939
:1045100002E1020ED0D0040EDB6AB1D0820EE66E4C
:10452000D90EE66E000EE66E6A0EE66E000EE66EC0
:10453000DEEC6EF0146E050EE15C02E2E16AE5521B
:10454000E16E1450000904E10201D46BD66B97D0E0
:10455000800EE66ED90EE66E000EE66E6A0EE66E10
:10456000000EE66EDEEC6EF0146E050EE15C02E20B
:10457000E16AE552E16E1450000915E10201D46BC5
:10458000010ED65D0DE2D8510BE1010E0301215D54
:1045900004E2010E216F8FEC36F00201010ED86F9C
:1045A000010ED66F6CD07E0EE66ED90EE66E000E52
:1045B000E66E6A0EE66E000EE66EDEEC6EF0146ECF
:1045C000050EE15C02E2E16AE552E16E1450000979
:1045D00056E1020E0201D65D0DE2D8510BE1020E4A
:1045E0000301215D04E2020E216F8FEC36F002011F
:1045F000010ED86F020ED66FD45141E1010ED46F77
:104600003ED0820EE66ED90EE66E000EE66E6A0EA3
:10461000E66E000EE66EDEEC6EF0146E050EE15CEA
:1046200002E2E16AE552E16E145000090AE102017A
:10463000D50504E0D85102E1010ED86F010ED56F07
:104640001ED07C0EE66ED90EE66E000EE66E6A0E89
:10465000E66E000EE66EDEEC6EF0146E050EE15CAA
:1046600002E2E16AE552E16E1450000908E102013C
:10467000D55104E0D85102E1010ED86FD56B020E7E
:10468000DB6A030EDB2ADF2A010E01E2DAD6DB2A1F
:10469000D8D6DB2AEF50E66E020EDBCFF3FFDB2A23
:1046A000F350EA6A6A0FE96E000EEA22E552E7501B
:1046B000EF6EC7D6030E146E050EE15C02E2E16AEE
:1046C000E552E16E1450E552E5CFDAFFE7CFD9FFAE
:1046D00012000201010EDB6FF0941200D9CFE6FF49
:1046E000DACFE6FFE1CFD9FFE2CFDAFFE652E652BA
:1046F000E652E652E652020EDB6A030EDB6A010E58
:10470000F36E040EF3CFDBFFFC0EDBCFDEFFDBCF5F
:10471000DDFF040EDB5042E0DECFE9FFDDCFEAFF34
:10472000EF502C0A11E0210A0CE0070A0AE00A0AFD
:1047300008E0DFCFE9FFDF2A010EDBCFEAFF1EE34F
:104740001CD0040EDB6AE5D7030EDB50050A0AE035
:10475000010A08E0040A06E0010A04E0030A02E094
:10476000010A1CE100016A6B020EDB6A030EDB2A00
:10477000DF2A010ECEE3DB2ACCD7DB2AEF50E66E30
:10478000020EDBCFF3FFDB2AF350EA6A6A0FE96E11
:10479000000EEA22E552E750EF6EBBD7050EE15C52
:1047A00002E2E16AE552E16EE552E5CFDAFFE7CFDA
:1047B000D9FF1200D9CFE6FFDACFE6FFE1CFD9FF6C
:1047C000E2CFDAFFE652E652DF6ADE52010EDD6E1C
:1047D000FC0EDBCFE9FFFD0EDBCFEAFFEF502C0A2A
:1047E0000FE0260A2CE00A0A09E0FC0EDBCFE9FF05
:1047F000DB2AFD0EDBCFEAFF26E324D0FE0E33D00A
:10480000DF50EA6A6A0FE96E000EEA22EF6A760E5E
:10481000E66ED90EE66E000EE66E6A0EE66E000ECD
:10482000E66EDEEC6EF0146E050EE15C02E2E16A0B
:10483000E552E16E1450000902E1010E14D0010EA0
:10484000DB6A0DD0DB2AEF50E66EDF50DF2AEA6A22
:104850006A0FE96E000EEA22E552E750EF6E010E94
:10486000DB50B6E1FF0EE552E552E552E5CFDAFF47
:10487000E7CFD9FF1200920E146E000E14C0F3FFA2
:10488000F46E1200D9CFE6FFDACFE6FFE1CFD9FF11
:10489000E2CFDAFFE6522C0E0001965D1DE1985141
:1048A0001BE197C016F0176A16BE176816C0E6FF20
:1048B00017C0E6FF94EC73F0E552E552F350F410A4
:1048C00001E1B0D300019751340A08E0070A06E07D
:1048D000010A04E0030A02E0000EA5D30F0E9715AB
:1048E000FF0FDF6EFC0EDBCFE9FFFD0EDBCFEAFF33
:1048F000540EEF6E010EE76EFC0EDBCFE9FFFD0EEE
:10490000DBCFEAFFE750E926000EEA224D0EEF6EFC
:10491000020EE76EFC0EDBCFE9FFFD0EDBCFEAFFF8
:10492000E750E926000EEA22520EEF6E030EE76E04
:10493000FC0EDBCFE9FFFD0EDBCFEAFFE750E926F7
:10494000000EEA2297C0EFFF040EE76EFC0EDBCFED
:10495000E9FFFD0EDBCFEAFFE750E926000EEA2271
:10496000200EEF6EDFCFE9FFEA6AE9BEEA68030EC8
:10497000D890E936EA36E806FBE1FD0EE926020E9C
:10498000EA22EF5044E0020A22E0030A40E1030E6B
:10499000E66EE66A720EE66ED90EE66E000EE66E02
:1049A000050EE76EFC0EDBCF14F0FD0EDBCF15F02D
:1049B000E7501426000E152214C0E6FF15C0E6FFCE
:1049C00085EC6EF0166E070EE15C42E23FD0030EFE
:1049D000E66EE66A6E0EE66ED90EE66E000EE66EC6
:1049E000050EE76EFC0EDBCF14F0FD0EDBCF15F0ED
:1049F000E7501426000E152214C0E6FF15C0E6FF8E
:104A000085EC6EF0166E070EE15C22E21FD0030EFD
:104A1000E66EE66A6A0EE66ED90EE66E000EE66E89
:104A2000050EE76EFC0EDBCF14F0FD0EDBCF15F0AC
:104A3000E7501426000E152214C0E6FF15C0E6FF4D
:104A400085EC6EF0166E070EE15C02E2E16AE5525B
:104A5000E16E1650080EE76EFC0EDBCFE9FFFD0E8F
:104A6000DBCFEAFFE750E926000EEA22200EEF6EC8
:104A7000DFCFE9FFEA6AE9BEEA68030ED890E936BB
:104A8000EA36E806FBE1FD0EE926020EEA22020EF6
:104A9000E926000EEA22EECF14F0EECF15F0EFCFAC
:104AA00016F00A0E176E0E6E14C009F009EC71F0C4
:104AB00009503009E66E090EE76EFC0EDBCFE9FF08
:104AC000FD0EDBCFEAFFE750E926000EEA22E552B1
:104AD000E750EF6EDFCFE9FFEA6AE9BEEA68030E4E
:104AE000D890E936EA36E806FBE1FD0EE926020E2B
:104AF000EA22020EE926000EEA22EECF14F0EECFF3
:104B000015F0EFCF16F014C009F00A0E0E6E09EC86
:104B100071F005503009E66E0A0EE76EFC0EDBCF31
:104B2000E9FFFD0EDBCFEAFFE750E926000EEA229F
:104B3000E552E750EF6E0B0EE76EFC0EDBCFE9FFA0
:104B4000FD0EDBCFEAFFE750E926000EEA223A0E1F
:104B5000EF6EDFCFE9FFEA6AE9BEEA68030ED8909C
:104B6000E936EA36E806FBE1FD0EE926020EEA2206
:104B7000020EE926000EEA22EECF14F0EECF15F079
:104B8000EFCF16F00A0E176E0E6E15C009F009EC85
:104B900071F009503009E66E0C0EE76EFC0EDBCFAB
:104BA000E9FFFD0EDBCFEAFFE750E926000EEA221F
:104BB000E552E750EF6EDFCFE9FFEA6AE9BEEA6847
:104BC000030ED890E936EA36E806FBE1FD0EE92649
:104BD000020EEA22020EE926000EEA22EECF14F0BF
:104BE000EECF15F0EFCF16F015C009F00A0E0E6EDD
:104BF00009EC71F005503009E66E0D0EE76EFC0E03
:104C0000DBCFE9FFFD0EDBCFEAFFE750E926000E20
:104C1000EA22E552E750EF6E0E0EE76EFC0EDBCF98
:104C2000E9FFFD0EDBCFEAFFE750E926000EEA229E
:104C30003A0EEF6EDFCFE9FFEA6AE9BEEA68030EDB
:104C4000D890E936EA36E806FBE1FD0EE926020EC9
:104C5000EA22020EE926000EEA22EECF14F0EECF91
:104C600015F0EFCF16F00A0E176E0E6E16C009F093
:104C700009EC71F009503009E66E0F0EE76EFC0E7C
:104C8000DBCFE9FFFD0EDBCFEAFFE750E926000EA0
:104C9000EA22E552E750EF6EDFCFE9FFEA6AE9BEAC
:104CA000EA68030ED890E936EA36E806FBE1FD0E25
:104CB000E926020EEA22020EE926000EEA22EECFD3
:104CC00014F0EECF15F0EFCF16F016C009F00A0E73
:104CD0000E6E09EC71F005503009E66E100EE76EAD
:104CE000FC0EDBCFE9FFFD0EDBCFEAFFE750E92644
:104CF000000EEA22E552E750EF6E110EE76EFC0E51
:104D0000DBCFE9FFFD0EDBCFEAFFE750E926000E1F
:104D1000EA22200EEF6E120EE76EFC0EDBCFE9FFEB
:104D2000FD0EDBCFEAFFE750E926000EEA222D0E4A
:104D3000EF6E130EE76EFC0EDBCFE9FFFD0EDBCF4F
:104D4000EAFFE750E926000EEA22200EEF6EDFCFE1
:104D5000E9FFEA6AE9BEEA68030ED890E936EA3666
:104D6000E806FBE1FD0EE926020EEA22050EE92621
:104D7000000EEA22EECF14F0EECF15F0EFCF16F0D2
:104D80000A0E176E0E6E14C009F009EC71F009508E
:104D90003009E66E140EE76EFC0EDBCFE9FFFD0E68
:104DA000DBCFEAFFE750E926000EEA22E552E750A2
:104DB000EF6EDFCFE9FFEA6AE9BEEA68030ED8903A
:104DC000E936EA36E806FBE1FD0EE926020EEA22A4
:104DD000050EE926000EEA22EECF14F0EECF15F014
:104DE000EFCF16F014C009F00A0E0E6E09EC71F048
:104DF00005503009E66E150EE76EFC0EDBCFE9FFBD
:104E0000FD0EDBCFEAFFE750E926000EEA22E5526D
:104E1000E750EF6E160EE76EFC0EDBCFE9FFFD0EDE
:104E2000DBCFEAFFE750E926000EEA223A0EEF6EEA
:104E3000DFCFE9FFEA6AE9BEEA68030ED890E936F7
:104E4000EA36E806FBE1FD0EE926020EEA22050E2F
:104E5000E926000EEA22EECF14F0EECF15F0EFCFE8
:104E600016F00A0E176E0E6E15C009F009EC71F0FF
:104E700009503009E66E170EE76EFC0EDBCFE9FF36
:104E8000FD0EDBCFEAFFE750E926000EEA22E552ED
:104E9000E750EF6EDFCFE9FFEA6AE9BEEA68030E8A
:104EA000D890E936EA36E806FBE1FD0EE926020E67
:104EB000EA22050EE926000EEA22EECF14F0EECF2C
:104EC00015F0EFCF16F015C009F00A0E0E6E09ECC2
:104ED00071F005503009E66E180EE76EFC0EDBCF60
:104EE000E9FFFD0EDBCFEAFFE750E926000EEA22DC
:104EF000E552E750EF6E190EE76EFC0EDBCFE9FFCF
:104F0000FD0EDBCFEAFFE750E926000EEA223A0E5B
:104F1000EF6EDFCFE9FFEA6AE9BEEA68030ED890D8
:104F2000E936EA36E806FBE1FD0EE926020EEA2242
:104F3000050EE926000EEA22EECF14F0EECF15F0B2
:104F4000EFCF16F00A0E176E0E6E16C009F009ECC0
:104F500071F009503009E66E1A0EE76EFC0EDBCFD9
:104F6000E9FFFD0EDBCFEAFFE750E926000EEA225B
:104F7000E552E750EF6EDFCFE9FFEA6AE9BEEA6883
:104F8000030ED890E936EA36E806FBE1FD0EE92685
:104F9000020EEA22050EE926000EEA22EECF14F0F8
:104FA000EECF15F0EFCF16F016C009F00A0E0E6E18
:104FB00009EC71F005503009E66E1B0EE76EFC0E31
:104FC000DBCFE9FFFD0EDBCFEAFFE750E926000E5D
:104FD000EA22E552E750EF6E1C0EE76EFC0EDBCFC7
:104FE000E9FFFD0EDBCFEAFFE750E926000EEA22DB
:104FF0000D0EEF6E1D0EE76EFC0EDBCFE9FFFD0E12
:10500000DBCFEAFFE750E926000EEA220A0EEF6E38
:10501000FA0EDBCFE9FFFB0EDBCFEAFF1E0EEF6ED1
:10502000010E01D0000EE552E552E5CFDAFFE7CFE1
:10503000D9FF1200D9CFE6FFDACFE6FFE1CFD9FFE3
:10504000E2CFDAFF2C0E0001965D1CE198511AE1C7
:1050500097C016F0176A16BE176816C0E6FF17C08D
:10506000E6FF94EC73F0E552E552F350F4102AE0B9
:1050700000019751340A1DE0070A14E0010A0BE011
:10508000030A02E0000E31D0FD0EDB5002E08D80FD
:1050900014D08D9015D0FD0EDB5002E08D820DD026
:1050A0008D920ED0FD0EDB5002E08D8406D08D94E3
:1050B00007D0FD0EDB5003E08D86010E13D08D96D8
:1050C000000E10D0410E0001975D0EE1FD0EDB5089
:1050D00005E08D808D828D848D8604D08D908D929B
:1050E0008D948D96010E01D0000EE552E5CFDAFFCA
:1050F000E7CFD9FF1200D9CFE6FFDACFE6FFE1CF45
:10510000D9FFE2CFDAFFE652DF6A0201FB5111E17B
:10511000FB51E76EFC0EDBCFE9FFFD0EDBCFEAFFB4
:10512000E750E926000EEA22EF50240802E1010EC2
:10513000FC6FDF6AFB0EDB50DF5C01E356D1FC51F4
:105140000FE0DF50E76EFC0EDBCFE9FFFD0EDBCF9B
:10515000EAFFE750E926000EEA22EF50E66E1CD087
:10516000DF50E76EFC0EDBCFE9FFFD0EDBCFEAFF81
:10517000E750E926000EEA22EFCF14F0156A14BEBC
:10518000156814C0E6FF15C0E6FFA6EC73F0E55203
:10519000E552F350E66E0201FB51EA6A920FE96EA6
:1051A000000EEA22E552E750EF6E010E146EFB513D
:1051B000145C01E30CD1FB51156E166A630E155C8D
:1051C000000E165801E303D1FB05EA6A920FE96E5F
:1051D000000EEA22EF500D0801E0F9D0FB51EA6A17
:1051E000920FE96E000EEA22EF500A0801E0EFD0BC
:1051F000FB05EA6A920FE96E000EEA22EF6AFB6B8A
:10520000650EE66ED90EE66E000EE66E920EE66E46
:10521000000EE66EDEEC6EF0146E050EE15C02E24E
:10522000E16AE552E16E1450000904E10201FC6BF1
:10523000000EFED0600EE66ED90EE66E000EE66E33
:10524000920EE66E000EE66EDEEC6EF0146E050E4B
:10525000E15C02E2E16AE552E16E1450000904E10A
:105260000201FC6B010EE4D05B0EE66ED90EE66E19
:10527000000EE66E920EE66E000EE66EDEEC6EF04E
:10528000146E050EE15C02E2E16AE552E16E145033
:10529000000904E10201FC6B020ECAD0040EE66EA6
:1052A000E66A560EE66ED90EE66E000EE66E920EB9
:1052B000E66E000EE66E3BEC6EF0146E070EE15CDF
:1052C00002E2E16AE552E16E1450000904E10201D4
:1052D000FC6B030EADD0040EE66EE66A510EE66E70
:1052E000D90EE66E000EE66E920EE66E000EE66ECB
:1052F0003BEC6EF0146E070EE15C02E2E16AE552EF
:10530000E16E1450000904E10201FC6B040E90D020
:10531000040EE66EE66A4C0EE66ED90EE66E000EE0
:10532000E66E920EE66E000EE66E3BEC6EF0146ECC
:10533000070EE15C02E2E16AE552E16E14500009F9
:1053400004E10201FC6B050E73D0040EE66EE66A02
:10535000470EE66ED90EE66E000EE66E920EE66E13
:10536000000EE66E3BEC6EF0146E070EE15C02E29E
:10537000E16AE552E16E1450000904E10201FC6BA0
:10538000060E56D00201FC511FE0FC6B440EE66E87
:10539000D90EE66E000EE66E920EE66E000EE66E1A
:1053A000C2EC6EF0146E050EE15C02E2E16AE552B9
:1053B000E16E1450920EE66E000EE66EA2EC70F0F6
:1053C000E552E552080E34D0FC6B090E31D0FB2BB0
:1053D000FB51146E156A630E145C000E155803E33E
:1053E000FC6BFB6B02D0DF2AA5D6FB51EA6A920F59
:1053F000E96E000EEA22EF6A440EE66ED90EE66E02
:10540000000EE66E920EE66E000EE66EDEEC6EF0BC
:10541000146E050EE15C02E2E16AE552E16E1450A1
:10542000000905E10201FB6BFC6B070E01D0FF0ECA
:0E543000E552E552E5CFDAFFE7CFD9FF1200D3
:02543E006EEC12
:105440006FF05EEC56F0CCEC72F0500EE66E800E13
:10545000E66E250EE66EE66AE66A6DEC62F0146EA4
:10546000050EE15C02E2E16AE552E16E14500401CE
:10547000D86B4B0ED96FDA6BDB6B080EDC6FDD6B14
:10548000DE6B140EE66E040EE66E8DEC42F0E55215
:10549000E552F3CF0FF2F4CF10F2010EE66E060ED6
:1054A000E66E8DEC42F0E552E552F3CF15F2F4CF03
:1054B00016F2010EE66E080EE66E8DEC42F0E55235
:1054C000E552F3CF11F2F4CF12F2020EE66E010EA6
:1054D000E66E8DEC42F0E552E552F3CF13F2F4CFD5
:1054E00014F2020EE66E010EE66E8DEC42F0E5520D
:1054F000E552F3CF17F2F4CF18F2000EE66EE66A2B
:10550000E66EE66A000EE66E020EE66E010EE66ECE
:10551000000EE66EE66AF00EE66EE66A000EE66ED5
:10552000E66ACE0EE66E560EE66E000EE66ECEEC27
:1055300036F0146E100EE15C02E2E16AE552E16EB3
:105540001450000EE66EE66AE66EE66A080EE66E37
:10555000020EE66E010EE66E000EE66EE66AF00ED4
:10556000E66EE66A000EE66EE66A000EE66E600E15
:10557000E66E000EE66ECEEC36F0146E100EE15CB8
:1055800002E2E16AE552E16E1450000EE66EE66A50
:10559000E66EE66A040EE66E020EE66E010EE66E3A
:1055A000000EE66EE66AC80EE66EE66A000EE66E6D
:1055B000E66A960EE66E620EE66E000EE66ECEECC3
:1055C00036F0146E100EE15C02E2E16AE552E16E23
:1055D0001450000EE66EE66AE66EE66A060EE66EA9
:1055E000020EE66E010EE66E000EE66EE66AAA0E8A
:1055F000E66EE66A000EE66EE66AE80EE66E680E95
:10560000E66E000EE66ECEEC36F0146E100EE15C27
:1056100002E2E16AE552E16E145004C2E6FF05C2FF
:10562000E6FF43EC39F0E552E55208C2E6FF09C255
:10563000E6FF43EC39F0E552E552B6EF3BF0D9CF47
:10564000E6FFDACFE6FFE1CFD9FFE2CFDAFFFA0ECD
:10565000DB500AC2E9FF0BC2EAFFEF6EFB0EDBCFA5
:10566000E6FFFC0EDBCFE6FFFD0EDBCFE6FF010E13
:105670000201156A0A25146E0B51152214C0E6FFAB
:1056800015C0E6FFF4EC6EF0166E050EE15C02E26A
:10569000E16AE552E16E1650E66AE668E6680AC21B
:1056A000E6FF0BC2E6FF0FC2E6FF10C2E6FFAEEC5C
:1056B00043F0146E070EE15C02E2E16AE552E16E2E
:1056C0001450E552E5CFDAFFE7CFD9FF1200D9CF6A
:1056D000E6FFDACFE6FFE1CFD9FFE2CFDAFF0F0E28
:1056E000E12402E3E168E652E16E010EF36E070E7B
:1056F000F3CFDBFF090EDB6A0A0EDB6A7E0E176E44
:10570000E30E186E000E196E1FC31AF01B6A1C6A96
:105710001AAE02D01B681C68050E0C6E0D6A0E6A6C
:105720001AC007F01BC008F01CC009F076EC71F03D
:1057300004C01AF005C01BF006C01CF0175004246A
:10574000146E18500520156E19500620166E0B0E9B
:1057500014C0DBFF0C0E15C0DBFF0D0E16C0DBFF07
:10576000140EE66EE66A6CEC72F0E552E552F3CF89
:105770000AF2F4CF0BF20201F350F41001E1B4D0BD
:10578000230E0AC2E9FF0BC2EAFFEF6EE66AE66883
:10579000E6680AC2E6FF0BC2E6FF0FC2E6FF10C2D0
:1057A000E6FFAEEC43F0146E070EE15C02E2E16A44
:1057B000E552E16E1450240E0AC2E9FF0BC2EAFF63
:1057C000EF6EE66AE668E6680AC2E6FF0BC2E6FF2D
:1057D0000FC2E6FF10C2E6FFAEEC43F0146E070EF8
:1057E000E15C02E2E16AE552E16E1450210EE66EE0
:1057F000660EE66EDC0EE66E000EE66E20DFE5520B
:10580000E552E552E552400EE66E5A0EE66EDC0EAB
:10581000E66E000EE66E13DFE552E552E552E55204
:10582000E7EC3CF0F3CFDEFFF4CFDDFFD00EE66E09
:10583000070EE66ED9CFE6FFDACFE6FF56EC38F07A
:10584000E552E552E552E552230E0AC2E9FF0BC2CA
:10585000EAFFEF6EE66AE668E6680AC2E6FF0BC298
:10586000E6FF0FC2E6FF10C2E6FFAEEC43F0146E97
:10587000070EE15C02E2E16AE552E16E1450240E8B
:105880000AC2E9FF0BC2EAFFEF6EE66AE668E66865
:105890000AC2E6FF0BC2E6FF0FC2E6FF10C2E6FF38
:1058A000AEEC43F0146E070EE15C02E2E16AE552F1
:1058B000E16E1450210EE66E4E0EE66EDC0EE66EC4
:1058C000000EE66EBCDEE552E552E552E552400EB2
:1058D000E66E3E0EE66EDC0EE66E000EE66EAFDEA7
:1058E000E552E552E552E552030150510BE02E0E10
:1058F000E66EDC0EE66E000EE66ECFEC70F0E55262
:10590000E552E5521D0EE66EDC0EE66E000EE66E0A
:10591000CFEC70F0E552E552E5520C0EE66EDC0E6F
:10592000E66E000EE66ECFEC70F0E552E552E55201
:10593000F60EE66EDB0EE66E000EE66ECFEC70F055
:10594000E552E552E552E20EE66EDB0EE66E000E23
:10595000E66ECFEC70F0E552E552E5520B0EDBCF70
:10596000F6FF0C0EDBCFF7FF0D0EDBCFF8FF040EBA
:10597000F626000EF722F8220800F5CF14F0156A7B
:1059800014BE156814C0E6FF15C0E6FF0B0EDBCF92
:10599000F6FF0C0EDBCFF7FF0D0EDBCFF8FF030E8B
:1059A000F626000EF722F8220800F5CF16F0176A47
:1059B00016BE176816C0E6FF17C0E6FF8AEC1CF09B
:1059C000E552E552E552E552D10EE66EDB0EE66E8B
:1059D000000EE66ECFEC70F0E552E552E552D10EC6
:1059E000E66EDB0EE66E000EE66ECFEC70F0E55272
:1059F000E552E552E7EC3CF0F3CFDEFFF4CFDDFFFC
:105A0000D00EE66E070EE66ED9CFE6FFDACFE6FFE0
:105A100056EC38F0E552E552E552E55204C2E6FF95
:105A200005C2E6FF4EEC3AF0E552E55208C2E6FF49
:105A300009C2E6FF4EEC3AF0E552E552020EDB6A8F
:105A40009D8A23EC59F0020EDB6A1EEC65F0030E12
:105A5000F3CFDBFF040EF4CFDBFFD950030FE96E69
:105A6000000EDA20EA6EEE50ED1062E0010EF36EE9
:105A7000020EF3CFDBFF010EE76E030EDBCF14F057
:105A8000040EDBCF15F0E7501426000E152214C0CB
:105A9000E6FF15C0E6FFDAEC23F0E552E552010A15
:105AA00047E1020E146EE66E070EE76E030EDBCFC3
:105AB00015F0040EDBCF16F0E7501526000E162267
:105AC00015C0E6FF16C0E6FF06EC22F0E552E552EF
:105AD000E552E7CF14F0145C2BE1070EE76E030EDE
:105AE000DBCF14F0040EDBCF15F0E7501426000EC8
:105AF000152214C0E6FF15C0E6FF35EC1DF0E55297
:105B0000E55202010E6BE66AE668E6680E0EE66E86
:105B1000020EE66E13C2E6FF14C2E6FFAEEC43F0DF
:105B2000146E070EE15C02E2E16AE552E16E145088
:105B3000200E0F01E76E0019E8AE02D0E73402D064
:105B4000E750005D03E36550020B02E08A8279D7DB
:105B50008A920401E05110E1070EDB500DE0C90EFE
:105B6000E66EDB0EE66E000EE66EA7EC69F0E5521F
:105B7000E552E552070EDB6A270EE66E190EE66E59
:105B8000020EE66ED8EC68F0E552E552E552E76E9B
:105B9000050EE7CFDBFFDB50000801E308D2050E5E
:105BA000DBCFE6FF190EE66E020EE66E7BEC28F008
:105BB000E552E552E552E76E0E0EE7CFDBFFDB5014
:105BC000070A01E1D2D10E0A01E1B7D1010A01E1D0
:105BD0009ED10E0A01E169D1030A01E13DD1010A1A
:105BE00001E116D1070A01E1E2D0010A01E1C7D0C3
:105BF000030A01E17CD0010A01E0BDD10201320EAD
:105C0000416F300E426FD2C214F0D3C215F00A0EAB
:105C10000D6E0E6AD2C208F0D3C209F023EC71F007
:105C2000300E08100201436FD2C214F0D3C215F037
:105C30000A0E0D6E0E6AD2C208F0D3C209F023EC30
:105C400071F0300E04100201446F2F0E456F60C0DA
:105C500014F061C015F00A0E0D6E0E6A60C008F0F7
:105C600061C009F023EC71F0300E08100201466F9C
:105C700060C014F061C015F00A0E0D6E0E6A60C0AF
:105C800008F061C009F023EC71F0300E041002013D
:105C9000476F2F0E486F62C014F063C015F00A0EF4
:105CA0000D6E0E6A62C008F063C009F023EC71F05B
:105CB000300E08100201496F62C014F063C015F085
:105CC0000A0E0D6E0E6A62C008F063C009F023EC84
:105CD00071F004C014F005C015F0300E041002017C
:105CE0004A6F0D0E4B6F0A0E4C6F0C0E3BD10A0E15
:105CF000146E0E6E64C009F009EC71F009503009A1
:105D00000201416F64C009F00A0E0E6E09EC71F0D9
:105D1000055030090201426F3A0E436F0A0E146EAD
:105D20000E6E65C009F009EC71F0095030090201EE
:105D3000446F65C009F00A0E0E6E09EC71F0055053
:105D400030090201456F3A0E466F0A0E146E0E6E50
:105D500066C009F009EC71F0095030090201476F83
:105D600066C009F00A0E0E6E09EC71F0055030099C
:105D70000201486F0D0E496F0A0E4A6FF3D00201FF
:105D8000D551EA6ACE0FE96E020EEA22EFCF41F258
:105D90000201D651EA6ACB0FE96E020EEA22EFCF7A
:105DA00042F202010D0E436F0A0E446F98D0000EAE
:105DB000E66EE66AE66EE66A23EC5DF0E552E552D1
:105DC000E552E552000912E0C40EE66EDB0EE66E07
:105DD000000EE66E410EE66E020EE66EF4EC6EF01C
:105DE000146E050EE15C01E378D075D0B00EE66E5E
:105DF000DB0EE66E000EE66E410EE66E020EE66EFD
:105E0000F4EC6EF0146E050EE15C01E37CD079D009
:105E1000D950060FE66E000EDA20E66E410EE66EF1
:105E2000020EE66E42EC24F0E552E552E552E552F0
:105E3000000901E0A2D0B00EE66EDB0EE66E000EA9
:105E4000E66E410EE66E020EE66EF4EC6EF0146E37
:105E5000050EE15C58E255D0010EE66E1AEC28F012
:105E6000E552000911E0C40EE66EDB0EE66E000E90
:105E7000E66E410EE66E020EE66EF4EC6EF0146E07
:105E8000050EE15C2AE227D0B00EE66EDB0EE66E70
:105E9000000EE66E410EE66E020EE66EF4EC6EF05B
:105EA000146E050EE15C2FE22CD0E66A1AEC28F0A5
:105EB000E552000916E0C40EE66EDB0EE66E000E3B
:105EC000E66E410EE66E020EE66EF4EC6EF0146EB7
:105ED000050EE15C02E2E16AE552E16E1450040E47
:105EE00041D0B00EE66EDB0EE66E000EE66E410EA1
:105EF000E66E020EE66EF4EC6EF0146E050EE15CDA
:105F000002E2E16AE552E16E1450130E2BD0940EBA
:105F1000E66EDB0EE66E000EE66E410EE66E020EDB
:105F2000E66EF4EC6EF0146E050EE15C02E2E16ADE
:105F3000E552E16E14501B0E15D0820EE66EDB0E9C
:105F4000E66E000EE66E410EE66E020EE66EF4ECB4
:105F50006EF0146E050EE15C02E2E16AE552E16E5C
:105F60001450110EF36E060E03D0010EF36E070EE1
:105F7000F3CFDBFF02D0060EDB6A0401E05117E12C
:105F8000060EDB50000813E2060EDBCFE6FF410EE3
:105F9000E66E020EE66E42EC69F0E552E552E5521D
:105FA000060EDB6A010EF36E070EF3CFDBFF040172
:105FB000E05123E10301455120E0020EDB501DE0DA
:105FC000030EDBCFE9FF040EDBCFEAFFEF50E66EF6
:105FD000010EE76E030EDBCF14F0040EDBCF15F0DD
:105FE000E7501426000E152214C0E6FF15C0E6FF88
:105FF00042EC69F0E552E552E552FFEC69F021D53B
:10600000D9CFE6FFDACFE6FFE1CFD9FFE2CFDAFF63
:10601000080EE12402E3E168E652E16EDF6A140E45
:10602000E66EE66A6CEC72F0E552E552F3CF0CF2E4
:10603000F4CF0DF2E66AE668E668D950020FE66E24
:10604000000EDA20E66E11C2E6FF12C2E6FF93EC04
:1060500047F0146E070EE15C02E2E16AE552E16E80
:1060600014500009E7E0DF6A010EF36E050EF3CF6E
:10607000DBFF050EDB50DEE0050EDB6A020EDB50B7
:10608000010A5FE0070A10E0020AF3E145C320F3CA
:1060900003014529010B456FE85003E18A84010E95
:1060A000F7D08A94000EF4D008EC16F00009E1E075
:1060B000010EDB6ADBCF14F0040EE76E1418E8AEB5
:1060C00002D0E73402D0E750145CD3E2010EDBCFFC
:1060D000E9FFEA6AE9BEEA68030ED890E936EA36D3
:1060E000E806FBE1FD0EE926020EEA22EE52EF5031
:1060F000020813E1010EDBCFE9FFEA6AE9BEEA68B4
:10610000030ED890E936EA36E806FBE1FD0EE926F3
:10611000020EEA22EE52010EEF6E010EDB50030A70
:106120000CE0010A08E0030A04E0010A07E18D908F
:1061300005D08D9203D08D9401D08D96010EDB2A6F
:10614000B9D7010E146EE66ED9CFE6FFDACFE6FFBF
:1061500034EC1BF0E552E552E552E7CF14F0145C45
:1061600001E087D7010EF36E050EF3CFDBFFDF50A2
:10617000020A01E17CD0020A68E0010A01E079D755
:10618000010EF36E060EF3CFDBFF060EDB505AE076
:106190006EEC13F0E76E040EE7CFDBFFDB50060A70
:1061A0004EE0040A06E0010A04E0070A02E0010AE0
:1061B000ECE1040EDB50FE0FE76E010EE7CFDBFFD4
:1061C000F36E070EF3CFDBFF070EDB50DEE0010EB0
:1061D000DBCF14F0156A14BE156814C0E6FF15C0B5
:1061E000E6FF6DEC12F0E552E552E76E040EE7CFE4
:1061F000DBFFDB50060A20E0050A0FE0010AE4E1BC
:10620000010EDBCF14F0156A14BE156814C0E6FF4A
:1062100015C0E6FF7DEC08F00CD0010EDBCF14F0CA
:10622000156A14BE156814C0E6FF15C0E6FF9AECA7
:106230000EF0E552E552C8D7070EDB6AC5D7060E49
:10624000DB6AA3D767EC1AF014D7010E146EE66E62
:106250001F0EE66E030EE66EB1EC17F0E552E55246
:10626000E552E7CF14F0145C01E003D711D0010E22
:10627000146EE66E1D0EE66E030EE66E55EC14F01F
:10628000E552E552E552E7CF14F0145C01E0F1D697
:106290008FEC36F0EED6D9CFE6FFDACFE6FFE1CFCE
:1062A000D9FFE2CFDAFF0F0EE12402E3E168E65204
:1062B000E16E050EDB6A080EDB6A090EDB6AE66A30
:1062C000000EE66EE66AD950070FE66E000EDA2081
:1062D000E66E15C2E6FF16C2E6FF93EC47F0146EB9
:1062E000070EE15C02E2E16AE552E16E145000093A
:1062F00013E00201D65103E0020ED65D0DE1070E58
:10630000DBCFE6FFE00E8C14E552E7108C6E640ED6
:10631000F36E080EF3CFDBFFE66A010EE66EE66A67
:10632000D950060FE66E000EDA20E66E13C2E6FFC5
:1063300014C2E6FF93EC47F0146E070EE15C02E234
:10634000E16AE552E16E145000090DE1050EDB2A09
:10635000080EDB5000080CE2080EDB0609E1E00E37
:106360008C148C6E05D0010EF36E060EF3CFDBFF9E
:10637000140EF36E050EDBCFF4FFF350F45C01E274
:10638000DFD0050EDB6A821C3F0BDF6EDF5003019E
:106390005D19E76E010EE7CFDBFFDB50DF14E76E20
:1063A000020EE7CFDBFF010EDB505D15E76E030E3B
:1063B000E7CFDBFF020EDB5041E0040EDB6A060E86
:1063C000F36E040EDBCFF4FFF350F45C01E3B6D0C0
:1063D000020EDBA029D0E66AE668E668040EDB5010
:1063E000156A490F146E030E152214C0E6FF15C07E
:1063F000E6FF11C2E6FF12C2E6FFAEEC43F0166EF6
:10640000070EE15C02E2E16AE552E16E1650040E0D
:10641000EA6ADB34FE0BEA36E96E510EE926030E1A
:10642000EA22640EEE6EED6A020EDBCFF3FFF3900C
:10643000F342F3CFDBFF040EDB2AC1D7030EDB50A0
:1064400023E0040EDB6A060EF36E040EDBCFF4FFCE
:10645000F350F45C73E2030EDBA00CD0040EEA6A86
:10646000DB34FE0BEA36E96E510EE926030EEA2212
:10647000EE6AED6A030EDBCFF3FFF390F342F3CF46
:10648000DBFF040EDB2ADFD7040EDB6A060EF36E99
:10649000040EDBCFF4FFF350F45C50E2040EEA6A22
:1064A000DB34FE0BEA36E96E510EE926030EEA22D2
:1064B000000ED880EE54000EED543DE2040EEA6A60
:1064C000DB34FE0BEA36E96E510EE926030EEA22B2
:1064D000EE06000EED5AEECF14F0EDCF15F014508D
:1064E000151029E1E66AE668E668040EDB50156AD5
:1064F000490F146E030E152214C0E6FF15C0E6FF07
:1065000011C2E6FF12C2E6FFAEEC43F0166E070EB4
:10651000E15C02E2E16AE552E16E1650040EEA6ABD
:10652000DB34FE0BEA36E96E510EE926030EEA2251
:10653000060EEE6EED6A040EDB2AA8D7DFCF5DF300
:10654000060EDB5001E1BBD60201D60501E1B7D64C
:10655000D65105E1020E0301215D01E0B0D60A0E1D
:10656000DB6ADBCF14F0040EE76E1418E8AE02D03D
:10657000E73402D0E750145C01E3A1D60A0EDBCF6A
:10658000E9FFEA6AE9BEEA68030ED890E936EA361E
:10659000E806FBE1FD0EE926020EEA22020EE926DC
:1065A000000EEA220B0EE9CFDBFF0C0EEACFDBFF79
:1065B0000A0EDBCFE9FFEA6AE9BEEA68030ED8906B
:1065C000E936EA36E806FBE1FD0EE926020EEA228C
:1065D000050EE926000EEA22E9CF14F0EACF15F005
:1065E0000D0EE9CFDBFF0E0EEACFDBFF0A0EDBCF8D
:1065F000E9FFEA6AE9BEEA68030ED890E936EA36AE
:10660000E806FBE1FD0EE926020EEA22EF5001E169
:1066100066D1020A01E1BCD0030A01E060D10A0E92
:10662000DBCFE9FFEA6AE9BEEA68030ED890E936F3
:10663000EA36E806FBE1FD0EE926020EEA22EE52FA
:10664000EF50020A4EE0030A01E0A2D00B0EDBCFAE
:10665000E9FF0C0EDBCFEAFFEF500001645D01E0C3
:1066600097D00B0EDBCFE9FF0C0EDBCFEAFFEE522B
:10667000EF500001655D01E08BD00B0EDBCFE9FF31
:106680000C0EDBCFEAFF020EE926000EEA22EF50E5
:106690000001665D01E07CD00A0EDB50030A0CE0CD
:1066A000010A08E0030A04E0010A07E18D8005D031
:1066B0008D8203D08D8401D08D860A0EDBCFE9FF59
:1066C000EA6AE9BEEA68030ED890E936EA36E806D7
:1066D000FBE1FD0EE926020EEA22EE52020EEF6EFB
:1066E00057D00D0EDBCFE9FF0E0EDBCFEAFFEF50E8
:1066F0000001645D4DE10D0EDBCFE9FF0E0EDBCF37
:10670000EAFFEE52EF500001655D42E10D0EDBCF76
:10671000E9FF0E0EDBCFEAFF020EE926000EEA22A9
:10672000EF500001665D34E10A0EDB50030A0CE015
:10673000010A08E0030A04E0010A07E18D9005D090
:106740008D9203D08D9401D08D960A0EDBCFE9FF98
:10675000EA6AE9BEEA68030ED890E936EA36E80646
:10676000FBE1FD0EE926020EEA22EF6A0A0EDBCFFC
:10677000E9FFEA6AE9BEEA68030ED890E936EA362C
:10678000E806FBE1FD0EE926020EEA22EE52EF6A70
:106790000A0EDBCFE9FFEA6AE9BEEA68030ED89089
:1067A000E936EA36E806FBE1FD0EE926020EEA22AA
:1067B000EE52EF50020A4CE0030A01E090D00B0EBB
:1067C000DBCFE9FF0C0EDBCFEAFFEF500001645D89
:1067D00001E085D00B0EDBCFE9FF0C0EDBCFEAFF2B
:1067E000EE52EF500001655D01E079D00B0EDBCF7A
:1067F000E9FF0C0EDBCFEAFF020EE926000EEA22CB
:10680000EF500001665D6BE10A0EDB50030A0CE0FD
:10681000010A08E0030A04E0010A07E18D8005D0BF
:106820008D8203D08D8401D08D860A0EDBCFE9FFE7
:10683000EA6AE9BEEA68030ED890E936EA36E80665
:10684000FBE1FD0EE926020EEA22EE52020E46D0D0
:106850000D0EDBCFE9FF0E0EDBCFEAFFEF5000019C
:10686000645D3DE10D0EDBCFE9FF0E0EDBCFEAFFED
:10687000EE52EF500001655D32E10D0EDBCFE9FF16
:106880000E0EDBCFEAFF020EE926000EEA22EF50E1
:106890000001665D24E10A0EDB50030A0CE0010AE8
:1068A00008E0030A04E0010A07E18D9005D08D920B
:1068B00003D08D9401D08D960A0EDBCFE9FFEA6AF2
:1068C000E9BEEA68030ED890E936EA36E806FBE14D
:1068D000FD0EE926020EEA22EE52010EEF6E23ECC7
:1068E00059F00A0EDB2A3DD6D9CFE6FFDACFE6FF14
:1068F000E1CFD9FFE2CFDAFFE66AE668E6686B0E21
:10690000E66E020EE66E0FC2E6FF10C2E6FF93ECE3
:1069100047F0146E070EE15C02E2E16AE552E16EB7
:1069200014500009E9E002016B51250A3CE0010A1C
:1069300030E0070A2CE0630A14E0610ADDE1100E82
:10694000E66EE66A6C0EE66E020EE66E240EE66EEB
:10695000030EE66E5AEC6EF0146E060EE15C14E265
:1069600011D0100EE66EE66A6C0EE66E020EE66E52
:10697000340EE66E030EE66E5AEC6EF0146E060EE2
:10698000E15C02E2E16AE552E16E145009D0000ECA
:1069900001D0010EE66EE66AF3EC60F0E552E552D6
:1069A00006EC60F0A9D76CC2E6FF64EC61F0E5523A
:1069B000A3D7DBEF34F08C9E959EF00EE66E41EC93
:1069C00074F0E5528C8E8A928A948C908C928C947E
:1069D0008C968C988D908D928D948D9693929394A5
:1069E0009590959295949596959896909692969462
:1069F00096964FEC5FF09480948294849486948869
:106A0000948A9380400E9B6EF19EF186F1929F9442
:106A1000D08E270EE66EE66AE66AFD0EE66E020E80
:106A2000E66EA8EC6EF0146E050EE15C02E2E16A1F
:106A3000E552E16E14500301100E1F6FD0EC6AF0A6
:106A400074D820C345F303014529010B456FE85075
:106A500002E18A84010C8A94000CD9CFE6FFDACFD8
:106A6000E6FFE1CFD9FFE2CFDAFFE652DF6AD95085
:106A7000FA0FE96EFF0EDA20EA6E000ED880EE54AF
:106A8000000EED5411E2FC0EDBCFE9FFDB2AFD0E18
:106A9000DBCFEAFF01E3DB2AEF50DF1AFA0EDB0659
:106AA000FB0EE5E2DB06E3D7F90EDB501AE0FC0E45
:106AB000DBCFE9FFFD0EDBCFEAFFDFCFEFFFDF1C0F
:106AC000E66E010EE76EFC0EDBCFE9FFFD0EDBCFBD
:106AD000EAFFE750E926000EEA22E552E750EF6EA2
:106AE0001AD0FC0EDBCFE9FFFD0EDBCFEAFFEF5043
:106AF000DF5C13E1DF1C146E010EE76EFC0EDBCFD2
:106B0000E9FFFD0EDBCFEAFFE750E926000EEA229F
:106B1000EF50145C02E1010E01D0000EE552E55287
:106B2000E5CFDAFFE7CFD9FF1200D9CFE6FFDACF02
:106B3000E6FFE1CFD9FFE2CFDAFF280EE12402E33E
:106B4000E168E652E16E270EE66EE66AD9CFE6FF0F
:106B5000DACFE6FFE66AE66AE66AE66A22EC6CF0FD
:106B6000146E080EE15C02E2E16AE552E16E145037
:106B7000E66A250EE66EE66AD9CFE6FFDACFE6FFD3
:106B80006CDF146E050EE15C02E2E16AE552E16E33
:106B90001450000902E1C3D8ADD0D9CFE9FFDACF54
:106BA000EAFFEECFFDF2EECFFEF2EECFFFF2EECF38
:106BB00000F3EECF01F3EECF02F3EECF03F3EECF0F
:106BC00004F3EECF05F3EECF06F3EECF07F3EECFEF
:106BD00008F3EECF09F3EECF0AF3EECF0BF3EECFCF
:106BE0000CF3EECF0DF3EECF0EF3EECF0FF3EECFAF
:106BF00010F3EECF11F3EECF12F3EECF13F3EECF8F
:106C000014F3EECF15F3EECF16F3EECF17F3EECF6E
:106C100018F3EECF19F3EECF1AF3EECF1BF3EECF4E
:106C20001CF3EECF1DF3EECF1EF3EECF1FF3EECF2E
:106C300020F3EECF21F3EECF22F3EFCF23F3270E95
:106C4000DB6ADBCF14F0040EE76E1418E8AE02D056
:106C5000E73402D0E750145C4DE2270EDBCFE9FFAA
:106C6000EA6AE9BEEA68030ED890E936EA36E80631
:106C7000FBE1FD0EE926020EEA22EF50020814E1C4
:106C8000270EDBCFE9FFEA6AE9BEEA68030ED89077
:106C9000E936EA36E806FBE1FD0EE926020EEA22B5
:106CA000EE52010EEF6E23D0270EDBCFE9FFEA6A2A
:106CB000E9BEEA68030ED890E936EA36E806FBE159
:106CC000FD0EE926020EEA22EF6A270EDBCFE9FF6E
:106CD000EA6AE9BEEA68030ED890E936EA36E806C1
:106CE000FBE1FD0EE926020EEA22EE52EF6A270EC4
:106CF000DB2AA7D782BA07D00301010E506F030128
:106D0000206B216B0CD8280EE15C02E2E16AE552AF
:106D1000E16EE552E5CFDAFFE7CFD9FF1200010EB1
:106D2000E66E250EE66EE66AFD0EE66E020EE66E75
:106D300094DE146E050EE15C02E2E16AE552E16E5A
:106D40001450E66AE66AE66AE66A90EC6BF0E55291
:106D5000E552E552E552270EE66EE66AFD0EE66E56
:106D6000020EE66ED8EC6BF0E552E552E552E552C4
:106D70001200D880000E04015055C20E5155010E6C
:106D80005255000E535501E2120050C4D8F451C4BC
:0C6D9000D9F452C4DAF453C4DBF412004E
:046D9C00D9CFE6FF66
:106DA000DACFE6FFE1CFD9FFE2CFDAFFE652E652D3
:106DB000E652E652E652F00EDBCFE6FFF10EDBCFF5
:106DC000E6FFF70EDBCFE6FFF80EDBCFE6FF03ECC6
:106DD00042F0E552E552E552E552DE52F3CFDEFFD6
:106DE000F4CFDDFFDD52D950010FE96E000EDA203D
:106DF000EA6EEE50ED1001E121D1010EDBCFE9FF8B
:106E0000020EDBCFEAFF170EE926000EEA22030E80
:106E1000EECFDBFF040EEDCFDBFFF70EDBCF16F07E
:106E2000F80EDBCF17F01606000E175A010EDBCF57
:106E3000E9FF020EDBCFEAFF170EE926000EEA2279
:106E40001650EE24146E1750EE20156E010EDBCF97
:106E5000E9FF020EDBCFEAFF1E0EE926000EEA2252
:106E600014C0EEFF15C0EDFFF70EDBCFE6FFF80E06
:106E7000DBCFE6FFEE0EDBCFE6FFEF0EDBCFE6FF6C
:106E8000F40EDBCFE6FFF90EDBCFE6FFFA0EDBCF29
:106E9000E6FF010EDBCFE6FF020EDBCFE6FFEAECFA
:106EA00040F0146E090EE15C02E2E16AE552E16E27
:106EB0001450F50EDBCFE6FFF60EDBCFE6FFFB0E40
:106EC000DBCFE6FFFC0EDBCFE6FFFD0EDBCFE6FF00
:106ED000030EDBCFE6FF040EDBCFE6FF76EC56F0C9
:106EE000166E070EE15C02E2E16AE552E16E1650B1
:106EF000F3CF14F0F4CF15F0010EDBCFE9FF020E53
:106F0000DBCFEAFF14C0EEFF15C0EDFFF250E66ED6
:106F1000F29E0E01F22B0E01F20509E1010EDBCF0C
:106F2000F0FE020EDBCFF1FEB1EC41F015D00E0108
:106F3000F75112E1F0CEE9FFF1CEEAFF160EEB5069
:106F4000146EF40EDB50D880145406E3010EDBCF30
:106F5000F0FE020EDBCFF1FE010EDBCFE9FF020EE9
:106F6000DBCFEAFF160EE926000EEA22EFCF14F07F
:106F70000E01F551D88014540CE2010EDBCFE9FF6D
:106F8000020EDBCFEAFF160EE926000EEA22EFCF53
:106F9000F5FE0E01FC2B010EDBCFE9FF020EDBCF6D
:106FA000EAFF160EE926000EEA22EFCF14F00E01DA
:106FB000F651D88014540CE2010EDBCFE9FF020E2B
:106FC000DBCFEAFF160EE926000EEA22EFCFF6FE2F
:106FD000010EDBCFE9FF020EDBCFEAFF020EE9264E
:106FE000000EEA22E9CF14F0EACF15F014C0E6FF54
:106FF00015C0E6FF010EDBCFE9FF020EDBCFEAFF93
:10700000160EE926000EEA22EF50090DF3CF16F016
:10701000F4CF17F07F0E1626020E172216C0E6FFD9
:1070200017C0E6FF3AEC66F0E552E552E552E5524C
:10703000010EDF6EE552E7BEF28E01D0DF68DF049D
:1070400025E1D950F20FE96EFF0EDA20EA6EEE501C
:10705000ED100CE0F20EDBCFE9FFF30EDBCFEAFF21
:10706000010EDBCFEEFF020EDBCFEDFF0E01F7517D
:107070000DE0F0CEE9FFF1CEEAFF160EEB50146EF4
:10708000F40EDB50145C02E223EC59F0DF5000D028
:10709000146E050EE15C02E2E16AE552E16E145005
:1070A000E552E5CFDAFFE7CFD9FF1200D9CFE6FFEF
:1070B000DACFE6FFE1CFD9FFE2CFDAFFE652E652C0
:1070C000E652E652030EDB6A93DBFA0EDBCF16F0D4
:1070D000FB0EDBCF17F0FC0EDBCFE9FFFD0EDBCFA5
:1070E000EAFF1650EE24146E1750EE20156E14C0F1
:1070F000DEFFDD6EFC0EDBCFE9FFFD0EDBCFEAFF2E
:10710000EECF14F0EFCF15F00E011450F35D1550D3
:10711000F4591DE2DECF14F0DDCF15F0FC0EDBCF0D
:10712000E9FFFD0EDBCFEAFFEECF16F0EFCF17F051
:107130001650145C175015582BE2DECF18F0DDCF37
:1071400019F01850F35D1950F45922E21CD0DECF2B
:1071500014F0DDCF15F0FC0EDBCFE9FFFD0EDBCF29
:10716000EAFFEECF16F0EFCF17F01650145C175071
:10717000155809E3DECF18F0DDCF19F01850F35D94
:107180001950F45905E2010EF36E030EF3CFDBFF45
:10719000FC0EDBCFE9FFFD0EDBCFEAFFDECFEEFF1B
:1071A000DDCFEDFF030EDB5059E0F0CEE9FFF1CE6D
:1071B000EAFF020EE926000EEA22E9CF14F0EACF38
:1071C00015F0E9CFE6FFEACFE6FFB0EC67F0E55255
:1071D000E552F0CEE9FFF1CEEAFF020EE926000EFD
:1071E000EA22DECFEEFFDDCFEDFFDECF14F0DDCF04
:1071F00015F00E01F351145CF451155815E2F0CE60
:10720000E9FFF1CEEAFF020EE926000EEA22E9CFFD
:1072100014F0EACF15F0E9CFE6FFEACFE6FFB7C2F8
:10722000E6FFB8C2E6FF14D0F0CEE9FFF1CEEAFFE8
:10723000020EE926000EEA22E9CF14F0EACF15F09B
:10724000E9CFE6FFEACFE6FFB5C2E6FFB6C2E6FF4A
:10725000D2EC66F0E552E552E552E552CCDAE76E43
:10726000020EE7CFDBFFDB5002E123EC59F0040E06
:10727000E15C02E2E16AE552E16EE552E5CFDAFF58
:10728000E7CFD9FF1200D9CFE6FFDACFE6FFE1CF93
:10729000D9FFE2CFDAFFE652E652F250E66EF29EF6
:1072A000FC0EDBCF14F0FD0EDBCF15F00E01F0511C
:1072B000141802E1F151151804E1FC0EDB6AFD0E11
:1072C000DB6AD950FC0FE96EFF0EDA20EA6EEE5051
:1072D000ED1005E1F0CE14F0F1CE15F006D0FC0E65
:1072E000DBCF14F0FD0EDBCF15F014C0DEFF15C0B0
:1072F000DDFFDECFE9FFDDCFEAFF020EE926000E5B
:10730000EA22E9CF14F0EACF15F014C0E6FF15C069
:10731000E6FFB0EC67F0E552E552DECFE9FFDDCFE6
:10732000EAFF0C0EE926000EEA22080EE926000EFE
:10733000EA22EE50ED1014E0DECFE9FFDDCFEAFFE8
:107340000C0EE926000EEA22E9CF14F0EACF15F080
:1073500014C0E6FF15C0E6FFB0EC67F0E552E55259
:10736000DECFE9FFDDCFEAFF020EE926000EEA22BA
:10737000E9CF14F0EACF15F014C0E6FF15C0E6FF20
:10738000C20EE66E020EE66E3AEC66F0E552E5528B
:10739000E552E552E552E7BEF28ED950FC0FE96E98
:1073A000FF0EDA20EA6EEE50ED1002E123EC59F008
:1073B000E552E552E552E5CFDAFFE7CFD9FF1200FB
:1073C000D9CFE6FFDACFE6FFE1CFD9FFE2CFDAFF90
:1073D000E652E652E652DF6AFC0EDBCF08F0FD0E05
:1073E000DBCF09F0DE5208C0DEFF09C0DDFFDD5251
:1073F000010EDBCFE9FF020EDBCFEAFFE926000E2C
:10740000EA22080EE926000EEA22EECF14F0EFCFB2
:1074100015F0C20E141838E1020E151835E1010EF0
:10742000DBCFE9FF020EDBCFEAFF0C0EE926000EF0
:10743000EA22080EE926000EEA22EECF14F0EFCF82
:1074400015F0B90E141802E1020E151802E0000E34
:1074500001D0010E010818E0010EDBCFE9FF020E9A
:10746000DBCFEAFF0C0EE926000EEA22080EE92621
:10747000000EEA22EE50ED1002E0000E01D0010EE7
:10748000010802E1010EDF6EDF50E552E552E552E0
:10749000E552E5CFDAFFE7CFD9FF1200D9CFE6FFFB
:1074A000DACFE6FFE1CFD9FFE2CFDAFFE652E652CC
:1074B000FC0EDBCFDEFFDBCFDDFFD9CFE9FFDACF7C
:1074C000EAFFEE50ED1001E188D0DECF14F0DDCF01
:1074D00015F00E01F051141802E1F151151801E1F7
:1074E0007CD0F250E66EF29EDECFE6FFDDCFE6FF07
:1074F00067DFE552E55201086DE1DECFE9FFDDCF40
:10750000EAFF020EE926000EEA22E9CF14F0EACFE4
:1075100015F014C0E6FF15C0E6FFB0EC67F0E552C9
:10752000E552DECFE9FFDDCFEAFF160EE926000EB9
:10753000EA22EFCF14F00E01F651D88014540AE27B
:10754000DECFE9FFDDCFEAFF160EE926000EEA22C4
:10755000EFCFF6FEDECFE9FFDDCFEAFF020EE92630
:10756000000EEA22E9CF14F0EACF15F014C0E6FFCE
:1075700015C0E6FFDECFE9FFDDCFEAFF160EE926F4
:10758000000EEA22EF50090DF3CF16F0F4CF17F0FA
:107590007F0E1626020E172216C0E6FF17C0E6FF62
:1075A0003AEC66F0E552E552E552E552DECFE9FFEE
:1075B000DDCFEAFF160EE926000EEA22EFCF14F027
:1075C000F0CEE9FFF1CEEAFF160EEB50145C02E3B9
:1075D00023EC59F0E552E7BEF28EE552E552E55252
:1075E000E5CFDAFFE7CFD9FF1200D9CFE6FFDACF38
:1075F000E6FFE1CFD9FFE2CFDAFFE652E652E652EC
:10760000DF6AFC0EDBCF08F0FD0EDBCF09F0DE52A7
:1076100008C0DEFF09C0DDFFDD52010EDBCFE6FF53
:10762000020EDBCFE6FFCCDEE552E552010801E0B9
:1076300093D00E01F85174E1010EDBCFE9FF020E89
:10764000DBCFEAFF160EE926000EEA22EFCF14F098
:10765000F0CEE9FFF1CEEAFF160EEB50145C02E229
:10766000000E01D0010EDF6E010EDBCFE9FF020E2E
:10767000DBCFEAFFE926000EEA22E9CF14F0EACFD9
:1076800015F0E9CFE6FFEACFE6FFB0EC67F0E55290
:10769000E552010EDBCFE9FF020EDBCFEAFF160E4B
:1076A000E926000EEA22EFCF14F00E01F651D88041
:1076B00014540CE2010EDBCFE9FF020EDBCFEAFF30
:1076C000160EE926000EEA22EFCFF6FE010EDBCF02
:1076D000E9FF020EDBCFEAFFE926000EEA22E9CF3E
:1076E00014F0EACF15F0E9CFE6FFEACFE6FF010E8E
:1076F000DBCFE9FF020EDBCFEAFF160EE926000E14
:10770000EA22EF50090DF3CF16F0F4CF17F07F0EF9
:107710001626020E172216C0E6FF17C0E6FF16D087
:10772000010EDBCFE9FF020EDBCFEAFF0C0EE926EC
:10773000000EEA22E9CF14F0EACF15F0E9CFE6FF18
:10774000EACFE6FFB90EE66E020EE66E3AEC66F0A0
:10775000E552E552E552E552DF50E552E552E55279
:10776000E552E5CFDAFFE7CFD9FF1200D9CFE6FF28
:10777000DACFE6FFE1CFD9FFE2CFDAFFE652000E23
:10778000E66EE66AE66EE66AE66EE66AE66AE66E69
:10779000E66A960EE66EE66A7D0EE66EDB0EE66E35
:1077A000BC0EE66E810EE66E000EE66ECEEC36F096
:1077B000146E100EE15C02E2E16AE552E16E1450D3
:1077C000DF6EDF0409E1F29E0E01010EF76FF36B2D
:1077D000F46BB1EC58F00009E552E552E5CFDAFF61
:1077E000E7CFD9FF1200F29E0E01F76B22EF59F09E
:1077F0000E01F82B1200D9CFE6FFDACFE6FFE1CF7A
:10780000D9FFE2CFDAFFE652E652E652E652020E26
:10781000DB6AF250E66EF29E0E01F8070E01F85197
:1078200001E0C1D00E01F251000801E3BCD0030E0B
:10783000DB6A0201B9510DE0BEC2E9FFBFC2EAFF37
:10784000060EE926000EEA22EECF14F0EFCF15F077
:1078500002D0146A156A14C0DEFF15C0DDFF145093
:10786000151001E185D0DECFE9FFDDCFEAFF0C0E78
:10787000E926000EEA22E9CF14F0EACF15F014C091
:10788000E6FF15C0E6FFB0EC67F0E552E552DECF4B
:10789000E9FFDDCFEAFF020EE926000EEA22E9CF7A
:1078A00014F0EACF15F014C0E6FF15C0E6FFB0EC07
:1078B00067F0E552E552DECFE9FFDDCFEAFF160EB5
:1078C000E926000EEA22EFCF14F00E01F651D8801F
:1078D00014540AE2DECFE9FFDDCFEAFF160EE926F7
:1078E000000EEA22EFCFF6FEDECFE9FFDDCFEAFFA2
:1078F000020EE926000EEA22E9CF14F0EACF15F0D5
:1079000014C0E6FF15C0E6FFDECFE9FFDDCFEAFFDA
:10791000160EE926000EEA22EF50090DF3CF16F0FD
:10792000F4CF17F07F0E1626020E172216C0E6FFC0
:1079300017C0E6FF3AEC66F0E552E552E552E55233
:10794000DECFE9FFDDCFEAFF160EE926000EEA22C0
:10795000EFCF14F0F0CEE9FFF1CEEAFF160EEB50B8
:10796000145C05E3010EF36E030EF3CFDBFF61D76A
:107970000E01F951000808E20E01F951000804E275
:107980004ED80E01F907F8D7030EDB0403E00E0111
:10799000FA0509E1010EF36E020EF3CFDBFF0E01D3
:1079A000FA6B23EC59F0E552E7BEF28E020EDB5083
:1079B00000D0146E040EE15C02E2E16AE552E16E71
:1079C0001450E552E5CFDAFFE7CFD9FF1200D9CF47
:1079D000E6FFDACFE6FFE1CFD9FFE2CFDAFFE652EA
:1079E000E652F250E66EF29EF3CEDEFFF4CEDDFFFD
:1079F000E552E7BEF28EDECF14F0DDCF15F014C0F5
:107A0000F3FF15C0F4FF00D0E552E552E552E5CF93
:107A1000DAFFE7CFD9FF12000E01F2511200D9CFE1
:107A2000E6FFDACFE6FFE1CFD9FFE2CFDAFFE65299
:107A3000E652E652E6520E01F85101E0DFD0F32B98
:107A4000000EF423F351F4110DE1B5C2DEFFB6C20E
:107A5000DDFFB7C2B5F2B8C2B6F2DECFB7F2DDCF06
:107A6000B8F2FB2BB5C2E9FFB6C2EAFFEF5000093E
:107A700019E0B5C2E9FFB6C2EAFF030EE926000E1F
:107A8000EA22020EE926000EEA22EE50EFCFEAFFCC
:107A9000E96E060EE926000EEA22EECF14F0EFCFD3
:107AA00015F002D0146A156A020E14C0DBFF030E33
:107AB00015C0DBFF1450151001E1A1D0020EDBCF81
:107AC000E9FF030EDBCFEAFF020EE926000EEA22F1
:107AD000EECF14F0EFCF15F00E011450F35D1550FA
:107AE000F45901E28CD0020EDBCFE9FF030EDBCFAD
:107AF000EAFF020EE926000EEA22E9CF14F0EACFEF
:107B000015F0E9CFE6FFEACFE6FFB0EC67F0E5520B
:107B1000E552020EDBCFE9FF030EDBCFEAFF0C0ECE
:107B2000E926000EEA22080EE926000EEA22EE50AF
:107B3000ED1016E0020EDBCFE9FF030EDBCFEAFF0C
:107B40000C0EE926000EEA22E9CF14F0EACF15F078
:107B5000E9CFE6FFEACFE6FFB0EC67F0E552E55289
:107B6000020EDBCFE9FF030EDBCFEAFF160EE9269C
:107B7000000EEA22EFCF14F00E01F651D880145413
:107B80000CE2020EDBCFE9FF030EDBCFEAFF160E9D
:107B9000E926000EEA22EFCFF6FE020EDBCFE9FF68
:107BA000030EDBCFEAFF020EE926000EEA22E9CF40
:107BB00014F0EACF15F0E9CFE6FFEACFE6FF020EB8
:107BC000DBCFE9FF030EDBCFEAFF160EE926000E3E
:107BD000EA22EF50090DF3CF16F0F4CF17F07F0E25
:107BE0001626020E172216C0E6FF17C0E6FF3AEC73
:107BF00066F0E552E552E552E55234D7F92B040E12
:107C0000E15C02E2E16AE552E16EE552E5CFDAFFBE
:107C1000E7CFD9FF1200D9CFE6FFDACFE6FFE1CFF9
:107C2000D9FFE2CFDAFFE652E6520E01F85103E047
:107C3000010EFA6F7AD0F651090DF3CFE9FFF4CFB8
:107C4000EAFF7F0EE926020EEA22EF5002E1F60774
:107C5000F2D7F651090DF3CF14F0F4CF15F07F0EE3
:107C60001426020E152214C0DEFF15C0DDFFDECF84
:107C7000E9FFDDCFEAFFEE52EE50EFCFEAFFE96E0B
:107C8000020EE926000EEA22EECF14F0EFCF15F037
:107C9000DECFE9FFDDCFEAFFEE5214C0EEFF15C0E4
:107CA000EDFFDECFE9FFDDCFEAFFEE52EECF14F0BD
:107CB000EFCF15F0DECFE9FFDDCFEAFF030EE926B7
:107CC000000EEA22EACF17F0E95014181DE1175010
:107CD00015181AE1DECFE9FFDDCFEAFFEE52EE50D4
:107CE000EFCFEAFFE96E020EE926000EEA22EECFA0
:107CF00014F0EFCF15F0DECFE9FFDDCFEAFFEE5253
:107D000014C0EEFF15C0EDFFDECFE9FFDDCFEAFFC7
:107D1000EE52EE50EFCFEAFFE96E060EE926000EB6
:107D2000EA22EECFF0FEEDCFF1FEE552E552E5524C
:107D3000E5CFDAFFE7CFD9FF1200D9CFE6FFDACFE0
:107D4000E6FFE1CFD9FFE2CFDAFFE652E652F0CE0E
:107D5000E9FFF1CEEAFF0C0EE926000EEA22E9CF98
:107D600014F0EACF15F0E9CFE6FFEACFE6FFFC0E0C
:107D7000DBCFE6FFFD0EDBCFE6FFD2EC66F0E5528F
:107D8000E552E552E552F0CEE9FFF1CEEAFF020EF0
:107D9000E926000EEA22E9CF14F0EACF15F0E9CF88
:107DA000E6FFEACFE6FFB0EC67F0E552E552D950C6
:107DB000FA0FE96EFF0EDA20EA6EFF0EEE181AE1F6
:107DC000FF0EED1817E1F0CEE9FFF1CEEAFF020E4B
:107DD000E926000EEA22E9CF14F0EACF15F0E9CF48
:107DE000E6FFEACFE6FFC20EE66E020EE66E3AEC62
:107DF00066F050D0FA0EDB500E01F3250001146E30
:107E0000FB0EDB500E01F4210001156E14C0DEFFE5
:107E1000DD6EF0CEE9FFF1CEEAFF020EE926000E9C
:107E2000EA22DECFEEFFDDCFEDFFDECF14F0DDCFB7
:107E300015F00E01F351145CF451155815E2F0CE13
:107E4000E9FFF1CEEAFF020EE926000EEA22E9CFB1
:107E500014F0EACF15F0E9CFE6FFEACFE6FFB7C2AC
:107E6000E6FFB8C2E6FF14D0F0CEE9FFF1CEEAFF9C
:107E7000020EE926000EEA22E9CF14F0EACF15F04F
:107E8000E9CFE6FFEACFE6FFB5C2E6FFB6C2E6FFFE
:107E9000D2EC66F0E552E552E552E552E552E55284
:107EA000E552E5CFDAFFE7CFD9FF1200D9CFE6FFE1
:107EB000DACFE6FFE1CFD9FFE2CFDAFFE652E652B2
:107EC000E652FC0EDBCFE9FFFD0EDBCFEAFFEF5001
:107ED0001BE0FC0EDBCFE9FFFD0EDBCFEAFF030E5C
:107EE000E926000EEA22020EE926000EEA22EE50F2
:107EF000EFCFEAFFE96E060EE926000EEA22EECF8A
:107F000014F0EFCF15F002D0146A156A14C0DEFF2A
:107F100015C0DDFFDECFE9FFDDCFEAFF0C0EE9265D
:107F2000000EEA22E9CF14F0EACF15F0E9CFE6FF20
:107F3000EACFE6FFB0EC67F0E552E5520E01F851EA
:107F400054E1DECFE9FFDDCFEAFF020EE926000EA5
:107F5000EA22E9CF14F0EACF15F0E9CFE6FFEACF45
:107F6000E6FFB0EC67F0E552E552DECFE9FFDDCF8A
:107F7000EAFF160EE926000EEA22EFCF14F00E01FA
:107F8000F651D88014540AE2DECFE9FFDDCFEAFFD4
:107F9000160EE926000EEA22EFCFF6FEDECFE9FF4D
:107FA000DDCFEAFF020EE926000EEA22E9CF14F047
:107FB000EACF15F0E9CFE6FFEACFE6FFDECFE9FF33
:107FC000DDCFEAFF160EE926000EEA22EF50090D7A
:107FD000F3CF16F0F4CF17F07F0E1626020E1722FD
:107FE00016C0E6FF17C0E6FF14D0DECFE9FFDDCFF5
:107FF000EAFF0C0EE926000EEA22E9CF14F0EACFE0
:1080000015F0E9CFE6FFEACFE6FFB90EE66E020E05
:10801000E66E3AEC66F0E552E552E552E552DECF07
:10802000E9FFDDCFEAFF160EE926000EEA22EFCFC8
:1080300014F0F0CEE9FFF1CEEAFF160EEB50145C1F
:1080400006E3010EF36E020EF3CFDBFF02D0020E49
:10805000DB6ADB50E552E552E552E552E5CFDAFF47
:10806000E7CFD9FF1200D9CFE6FFDACFE6FFE1CFA5
:10807000D9FFE2CFDAFFFC0EDBCFE9FFFD0EDBCF4D
:10808000EAFFFBCEEFFFFC0EDBCFE9FFFD0EDBCFFF
:10809000EAFFEE52F3CEEEFFF4CEEDFFE552E5CF70
:1080A000DAFFE7CFD9FF1200D9CFE6FFDACFE6FF3C
:1080B000E1CFD9FFE2CFDAFFE652F250E66EF29E50
:1080C000FA0EDBCFE9FFFB0EDBCFEAFFFF0EEE1867
:1080D00002E1FF0EED1802E1DF6A60D0FC0EDBCF9B
:1080E000E9FFFD0EDBCFEAFFEF500E01FB5D14E070
:1080F000FC0EDBCFE9FFFD0EDBCFEAFFEE52EECF49
:1081000014F0EFCF15F00E011450F35D1550F45933
:1081100003E3010EDF6E42D0FC0EDBCFE9FFFD0E64
:10812000DBCFEAFFEE520E01EE50F35D146EEE501F
:10813000F459156EFA0EDBCFE9FFFB0EDBCFEAFF39
:10814000EECF16F0EFCF17F01650145C17501558FD
:1081500023E2FC0EDBCFE9FFFD0EDBCFEAFFEE52A0
:108160000E01EE50F35D146EEE50F459156EFA0EDA
:10817000DBCFE9FFFB0EDBCFEAFF1450EE5E1550BC
:10818000ED5AFC0EDBCFE6FFFD0EDBCFE6FF6BDF2B
:10819000E552E552DF6A02D0010EDF6EE552E7BE1E
:1081A000F28EDF5000D0E552E552E5CFDAFFE7CF9F
:1081B000D9FF12000E01010EFA6F1200D9CFE6FFAF
:1081C000DACFE6FFE1CFD9FFE2CFDAFF1BD923EC0C
:1081D00059F0FCD7D9CFE6FFDACFE6FFE1CFD9FFE0
:1081E000E2CFDAFF050EE66EE66AFA0EDBCFE6FFB7
:1081F000FB0EDBCFE6FFFC0EDBCFE9FFFD0EDBCF96
:10820000EAFF190EE926000EEA22E9CF14F0EACFC0
:1082100015F0E9CFE6FFEACFE6FF40EC6FF0166E0F
:10822000060EE15C02E2E16AE552E16E1650FC0ED8
:10823000DBCFE9FFFD0EDBCFEAFF190EE926000ECA
:10824000EA22040EE926000EEA22EF6A040EF36E1B
:10825000F90EDBCFF4FFF350F45C05E3030EF36E8D
:10826000F90EF3CFDBFFFC0EDBCFE9FFFD0EDBCF1A
:10827000EAFF160EE926000EEA22F90EDBCFEFFF29
:10828000FC0EDBCFE9FFFD0EDBCFEAFF020EE92695
:10829000000EEA22E9CF14F0EACF15F0E9CFE6FFAD
:1082A000EACFE6FF22EC66F0E552E552FC0EDBCFAA
:1082B000E9FFFD0EDBCFEAFF0C0EE926000EEA22F5
:1082C000E9CF14F0EACF15F0E9CFE6FFEACFE6FFF9
:1082D00022EC66F0E552E552FC0EDBCFE9FFFD0E25
:1082E000DBCFEAFF020EE926000EEA22060EE9269F
:1082F000000EEA22FC0EDBCFEEFFFD0EDBCFEDFF22
:10830000F90EDB50146E156A040ED8801456000E58
:108310001556FC0EDBCFE9FFFD0EDBCFEAFF0C0E9E
:10832000E926000EEA2214C0EEFF15C0EDFFFC0E98
:10833000DBCFE9FFFD0EDBCFEAFF0C0EE926000ED6
:10834000EA22060EE926000EEA22FC0EDBCFEEFF43
:10835000FD0EDBCFEDFFE552E5CFDAFFE7CFD9FF2A
:108360001200D9CFE6FFDACFE6FFE1CFD9FFE2CFA7
:10837000DAFFE652DF6A040EDF5C14E2DF50090D1B
:10838000F3CF14F0F4CF15F07F0E1426020E152251
:1083900014C0E6FF15C0E6FFA8EC65F0E552E55213
:1083A000DF2AE9D7A30EE66E020EE66EA8EC65F0B2
:1083B000E552E552AC0EE66E020EE66EA8EC65F0F4
:1083C000E552E552B90EE66E020EE66EA8EC65F0D7
:1083D000E552E552C20EE66E020EE66EA8EC65F0BE
:1083E000E552E5520201A30EB56F020EB66FAC0E58
:1083F000B76F020EB86FE552E552E5CFDAFFE7CF6F
:10840000D9FF12001200D9CFE6FFDACFE6FFE1CFA5
:10841000D9FFE2CFDAFFE652E652200EE66EE66AB8
:108420006CEC72F0E552E552F3CFDEFFF4CFDDFFE6
:10843000D9CFE9FFDACFEAFFEE50ED105EE0D95078
:10844000FA0FE96EFF0EDA20EA6EEE50ED100FE142
:10845000FC0EDBCFE6FFFD0EDBCFE6FF6CEC72F02F
:10846000E552E552F3CF14F0F4CF15F006D0FA0E32
:10847000DBCF14F0FB0EDBCF15F0DECFE9FFDDCF55
:10848000EAFF170EE926000EEA2214C0EEFF15C01F
:10849000EDFFDECFE9FFDDCFEAFF170EE926000E84
:1084A000EA22EE50ED100BE1DECFE6FFDDCFE6FF76
:1084B000C2EC72F0E552E552DE6ADD6A1ED0FC0EB7
:1084C000DBCFE6FFFD0EDBCFE6FFA50EE66EDECFCF
:1084D000E9FFDDCFEAFF170EE926000EEA22EECF14
:1084E000E6FFEFCFE6FFA8EC6EF0146E050EE15C40
:1084F00002E2E16AE552E16E1450DECF14F0DDCF06
:1085000015F014C0F3FF15C0F4FFE552E552E55233
:0A851000E5CFDAFFE7CFD9FF120034
:06851A00D9CFE6FFDACF25
:10852000E6FFE1CFD9FFE2CFDAFFE652E652E652AC
:10853000E652FD0EDB50000801E302D11F0EE66E8D
:10854000E66A6CEC72F0E552E552F3CFDEFFF4CF51
:10855000DDFFD9CFE9FFDACFEAFFEE50ED1001E100
:10856000EFD0FC0EDBCFE6FFFD0EDB50E552E7025D
:10857000F350146E156A010E1426000E1522020E19
:1085800014C0DBFF030E15C0DBFF020EDBCFE6FFDE
:10859000030EDBCFE6FF6CEC72F0E552E552F3CF51
:1085A00014F0F4CF15F0DECFE9FFDDCFEAFFF3CF13
:1085B000EEFF15C0EDFFDECFE9FFDDCFEAFFEE50A5
:1085C000ED1001E1B5D0FC0EDBCFE6FFFD0EDB5078
:1085D000E552E702F350176ADECFE9FFDDCFEAFF8D
:1085E000F350EE24146E1750EE20156EDECFE9FF27
:1085F000DDCFEAFF020EE926000EEA2214C0EEFFEC
:1086000015C0EDFFDECFE9FFDDCFEAFF1A0EE92648
:10861000000EEA22EF6ADECFE9FFDDCFEAFFEECF00
:1086200014F0EFCF15F0DECFE9FFDDCFEAFF040E47
:10863000E926000EEA2214C0EEFF15C0EDFFFC0E85
:10864000DBCFE6FFFD0EDB04E552E702F350166ECA
:10865000176ADECFE9FFDDCFEAFFF350EE24146E98
:108660001750EE20156EDECFE9FFDDCFEAFF060ED4
:10867000E926000EEA2214C0EEFF15C0EDFFDECFA2
:10868000E9FFDDCFEAFF1B0EE926000EEA22FD0E10
:10869000DBCFEFFFDECFE9FFDDCFEAFF1C0EE926DF
:1086A000000EEA22FC0EDBCFEFFFDECFE9FFDDCFCD
:1086B000EAFF1D0EE926000EEA22EF68DECFE9FF91
:1086C000DDCFEAFF1E0EE926000EEA22EF68DECFBC
:1086D000E9FFDDCFEAFF080EE926000EEA22E9CF26
:1086E00014F0EACF15F0E9CFE6FFEACFE6FFA8ECF9
:1086F00065F0E552E552DECFE9FFDDCFEAFF110E6E
:10870000E926000EEA22E9CF14F0EACF15F0E9CF0E
:10871000E6FFEACFE6FFA8EC65F0E552E552DECFD2
:1087200014F0DDCF15F014C0F3FF15C0F4FF0AD02C
:10873000DECFE6FFDDCFE6FFC2EC72F0E552E55298
:10874000F36AF46A040EE15C02E2E16AE552E16E6A
:10875000E552E5CFDAFFE7CFD9FF1200D9CFE6FF28
:10876000DACFE6FFE1CFD9FFE2CFDAFFE652E652F9
:10877000E652E652DF6AF250E66EF29EFC0EDBCF66
:10878000E9FFFD0EDBCFEAFF1A0EE926000EEA2212
:10879000EFCF14F0FC0EDBCFE9FFFD0EDBCFEAFFDD
:1087A0001B0EE926000EEA22EF50145C45E2F70E9C
:1087B000DBCFE6FFFA0EDBCFE6FFFB0EDBCFE6FFFB
:1087C000FC0EDBCFE6FFFD0EDBCFE6FF00EC4AF050
:1087D000146E050EE15C02E2E16AE552E16E1450AE
:1087E000FC0EDBCFE9FFFD0EDBCFEAFF110EE92621
:1087F000000EEA22EF501AE0FC0EDBCFE9FFFD0E7F
:10880000DBCFEAFF110EE926000EEA22E9CF14F0D1
:10881000EACF15F014C0E6FF15C0E6FF56EC3FF0B6
:10882000E552E552010802E123EC59F0E552E7BEBA
:10883000F28E010EC4D01DD0D950F80FE96EFF0E94
:10884000DA20EA6EEE50ED1006E1E552E7BEF28E58
:10885000000EB5D00ED0DF500CE1D950010FE66EFE
:10886000000EDA20E66E33EC40F0E552E552010EE0
:10887000DF6EE552E7BEF28EF8EC3BF0F250E66EAA
:10888000F29EFC0EDBCFE9FFFD0EDBCFEAFF1D0EF3
:10889000E926000EEA22EF50FF080BE1FC0EDBCFC9
:1088A000E9FFFD0EDBCFEAFF1D0EE926000EEA22EE
:1088B000EF6AFC0EDBCFE9FFFD0EDBCFEAFF1E0EF9
:1088C000E926000EEA22EF50FF080BE1FC0EDBCF99
:1088D000E9FFFD0EDBCFEAFF1E0EE926000EEA22BD
:1088E000EF6AE552E7BEF28ED950F80FE66EFF0E42
:1088F000DA20E66ED950010FE66E000EDA20E66E41
:1089000054EC40F0E552E552E552E552000948E1E9
:10891000FC0EDBCFE6FFFD0EDBCFE6FFD8EC4CF024
:10892000E552E55200092FE0F80EDBCFE6FFF90E25
:10893000DBCFE6FFFC0EDBCFE9FFFD0EDBCFEAFF6E
:10894000080EE926000EEA22E9CF14F0EACF15F06E
:1089500014C0E6FF15C0E6FF9DEC3EF0E552E5527F
:10896000E552E552FC0EDBCFE6FFFD0EDBCFE6FF66
:10897000C9EC4BF0E552E552FBEC3BF0000902E19B
:1089800023EC59F00CD0FC0EDBCFE6FFFD0EDBCF65
:10899000E6FFC9EC4BF0E552E552FBEC3BF00ED0A4
:1089A000FC0EDBCFE6FFFD0EDBCFE6FFC9EC4BF0A4
:1089B000E552E552FBEC3BF0000E01D0DCD6146E24
:1089C000040EE15C02E2E16AE552E16E1450E55208
:1089D000E5CFDAFFE7CFD9FF1200D9CFE6FFDACF34
:1089E000E6FFE1CFD9FFE2CFDAFFE652E652E652E8
:1089F000E652DF6AF250E66EF29EFC0EDBCFE9FF34
:108A0000FD0EDBCFEAFF1A0EE926000EEA22EFCFB9
:108A100014F0FC0EDBCFE9FFFD0EDBCFEAFF1B0EEF
:108A2000E926000EEA22EF50145C45E2F70EDBCF98
:108A3000E6FFFA0EDBCFE6FFFB0EDBCFE6FFFC0E18
:108A4000DBCFE6FFFD0EDBCFE6FF00EC4AF0146E55
:108A5000050EE15C02E2E16AE552E16E1450FC0EA3
:108A6000DBCFE9FFFD0EDBCFEAFF110EE926000E9A
:108A7000EA22EF501AE0FC0EDBCFE9FFFD0EDBCF60
:108A8000EAFF110EE926000EEA22E9CF14F0EACF40
:108A900015F014C0E6FF15C0E6FF56EC3FF0E552B6
:108AA000E552010802E123EC59F0E552E7BEF28EEF
:108AB000010E6ED01DD0D950F80FE96EFF0EDA20EE
:108AC000EA6EEE50ED1006E1E552E7BEF28E000EC2
:108AD0005FD00ED0DF500CE1D950010FE66E000ED2
:108AE000DA20E66E33EC40F0E552E552010EDF6E1F
:108AF000E552E7BEF28EF250E66EF29ED950F80FC4
:108B0000E66EFF0EDA20E66ED950010FE66E000E1B
:108B1000DA20E66E54EC40F0E552E552E552E552BB
:108B200000092DE1FC0EDBCFE6FFFD0EDBCFE6FFFB
:108B3000D8EC4CF0E552E552000920E0F80EDBCF0E
:108B4000E6FFF90EDBCFE6FFFC0EDBCFE9FFFD0E03
:108B5000DBCFEAFF080EE926000EEA22E9CF14F087
:108B6000EACF15F014C0E6FF15C0E6FF9DEC3EF01D
:108B7000E552E552E552E55223EC59F005D0E552B5
:108B8000E7BEF28E000E04D0E552E7BEF28E32D779
:108B9000146E040EE15C02E2E16AE552E16E1450EB
:108BA000E552E5CFDAFFE7CFD9FF1200D9CFE6FFD4
:108BB000DACFE6FFE1CFD9FFE2CFDAFF060EE124FC
:108BC00002E3E168E652E16EDF6AF250E66EF29E81
:108BD000FC0EDBCFE9FFFD0EDBCFEAFF1A0EE92624
:108BE000000EEA22EF50000801E393D0FC0EDBCF29
:108BF000E9FFFD0EDBCFEAFF060EE926000EEA22B2
:108C0000040EEECFDBFF050EEDCFDBFFFA0EDBCF60
:108C1000E6FFFB0EDBCFE6FFFC0EDBCFE6FFFD0E33
:108C2000DBCFE6FF32EC4BF0E552E552E552E55280
:108C3000F70EDB5032E1FC0EDBCFE9FFFD0EDBCFA0
:108C4000EAFF1A0EE926000EEA22EF06FC0EDBCF41
:108C5000E9FFFD0EDBCFEAFF080EE926000EEA224F
:108C6000EF501AE0FC0EDBCFE9FFFD0EDBCFEAFF91
:108C7000080EE926000EEA22E9CF14F0EACF15F03B
:108C800014C0E6FF15C0E6FF56EC3FF0E552E55292
:108C9000010802E123EC59F036D0FC0EDBCFE9FFEE
:108CA000FD0EDBCFEAFF060EE926000EEA22040ED7
:108CB000DBCFEEFF050EDBCFEDFFFC0EDBCFE9FFD8
:108CC000FD0EDBCFEAFF110EE926000EEA22EF507F
:108CD0001AE0FC0EDBCFE9FFFD0EDBCFEAFF110E41
:108CE000E926000EEA22E9CF14F0EACF15F014C00D
:108CF000E6FF15C0E6FF56EC3FF0E552E5520009ED
:108D000002E023EC59F0E552E7BEF28E010E6ED080
:108D10001DD0D950F80FE96EFF0EDA20EA6EEE5042
:108D2000ED1006E1E552E7BEF28E000E5FD00ED0E8
:108D3000DF500CE1D950010FE66E000EDA20E66E2E
:108D400033EC40F0E552E552010EDF6EE552E7BE2E
:108D5000F28EF250E66EF29ED950F80FE66EFF0EDC
:108D6000DA20E66ED950010FE66E000EDA20E66ECC
:108D700054EC40F0E552E552E552E55200092DE190
:108D8000FC0EDBCFE6FFFD0EDBCFE6FF8FEC4CF0F9
:108D9000E552E552000920E0F80EDBCFE6FFF90EC0
:108DA000DBCFE6FFFC0EDBCFE9FFFD0EDBCFEAFFFA
:108DB000110EE926000EEA22E9CF14F0EACF15F0F1
:108DC00014C0E6FF15C0E6FF9DEC3EF0E552E5520B
:108DD000E552E55223EC59F005D0E552E7BEF28E9C
:108DE000000E04D0E552E7BEF28EEFD6146E060EEA
:108DF000E15C02E2E16AE552E16E1450E552E5CF32
:108E0000DAFFE7CFD9FF1200D9CFE6FFDACFE6FFCE
:108E1000E1CFD9FFE2CFDAFFE652E652010EDB6A7C
:108E2000FC0EDBCFE9FFFD0EDBCFEAFF1A0EE926D1
:108E3000000EEA22EFCF14F0FC0EDBCFE9FFFD0EAF
:108E4000DBCFEAFF1B0EE926000EEA22EF50145C8E
:108E500060E2F70EDBCFE6FFFA0EDBCFE6FFFB0E9C
:108E6000DBCFE6FFFC0EDBCFE6FFFD0EDBCFE6FF40
:108E7000C7DA146E050EE15C02E2E16AE552E16ECA
:108E80001450FC0EDBCFE9FFFD0EDBCFEAFF1E0E18
:108E9000E926000EEA22EF50FF082DE1FC0EDBCFA1
:108EA000E9FFFD0EDBCFEAFF110EE926000EEA22F4
:108EB000EF502CE0FC0EDBCFE9FFFD0EDBCFEAFF2D
:108EC000110EE926000EEA22E9CF14F0EACF15F0E0
:108ED000E9CFE6FFEACFE6FF56EC3FF0E552E55278
:108EE000000914E0F80EDBCFE9FFF90EDBCFEAFF53
:108EF000010EEF6E0BD0FC0EDBCFE9FFFD0EDBCFDA
:108F0000EAFF1E0EE926000EEA22EF2A010EDF6EAE
:108F100001D0DF6ADF50E552E552E552E5CFDAFFD6
:108F2000E7CFD9FF1200D9CFE6FFDACFE6FFE1CFD6
:108F3000D9FFE2CFDAFF060EE12402E3E168E65250
:108F4000E16EDF6AF250E66EF29EFC0EDBCFE9FFC7
:108F5000FD0EDBCFEAFF1A0EE926000EEA22EF50E3
:108F6000000801E392D0FC0EDBCFE9FFFD0EDBCF62
:108F7000EAFF060EE926000EEA22040EEECFDBFF22
:108F8000050EEDCFDBFFFA0EDBCFE6FFFB0EDBCFEE
:108F9000E6FFFC0EDBCFE6FFFD0EDBCFE6FF62DB7C
:108FA000E552E552E552E552F70EDB5032E1FC0E98
:108FB000DBCFE9FFFD0EDBCFEAFF1A0EE926000E3C
:108FC000EA22EF06FC0EDBCFE9FFFD0EDBCFEAFF66
:108FD000080EE926000EEA22EF501AE0FC0EDBCF65
:108FE000E9FFFD0EDBCFEAFF080EE926000EEA22BC
:108FF000E9CF14F0EACF15F014C0E6FF15C0E6FF84
:1090000056EC3FF0E552E552010802E123EC59F03D
:1090100036D0FC0EDBCFE9FFFD0EDBCFEAFF060EFC
:10902000E926000EEA22040EDBCFEEFF050EDBCFB1
:10903000EDFFFC0EDBCFE9FFFD0EDBCFEAFF110EEB
:10904000E926000EEA22EF501AE0FC0EDBCFE9FF22
:10905000FD0EDBCFEAFF110EE926000EEA22E9CF72
:1090600014F0EACF15F014C0E6FF15C0E6FF56EC89
:109070003FF0E552E552000902E023EC59F0E552D9
:10908000E7BEF28E010EC0D01DD0D950F80FE96EA8
:10909000FF0EDA20EA6EEE50ED1006E1E552E7BE73
:1090A000F28E000EB1D00ED0DF500CE1D950010F7E
:1090B000E66E000EDA20E66E33EC40F0E552E55243
:1090C000010EDF6EE552E7BEF28EF8EC3BF0F25097
:1090D000E66EF29EFC0EDBCFE9FFFD0EDBCFEAFF72
:1090E0001D0EE926000EEA22EF50FF080BE1FC0EF0
:1090F000DBCFE9FFFD0EDBCFEAFF1D0EE926000EF8
:10910000EA22EF6AFC0EDBCFE9FFFD0EDBCFEAFFC0
:109110001E0EE926000EEA22EF50FF080BE1FC0EBE
:10912000DBCFE9FFFD0EDBCFEAFF1E0EE926000EC6
:10913000EA22EF6AE552E7BEF28ED950F80FE66EEA
:10914000FF0EDA20E66ED950010FE66E000EDA202F
:10915000E66E54EC40F0E552E552E552E552000966
:1091600045E1FC0EDBCFE6FFFD0EDBCFE6FFD7DBF4
:10917000E552E55200092EE0F80EDBCFE6FFF90ECE
:10918000DBCFE6FFFC0EDBCFE9FFFD0EDBCFEAFF16
:10919000110EE926000EEA22E9CF14F0EACF15F00D
:1091A00014C0E6FF15C0E6FF9DEC3EF0E552E55227
:1091B000E552E552FC0EDBCFE6FFFD0EDBCFE6FF0E
:1091C000E8DAE552E552FBEC3BF0000902E123EC62
:1091D00059F00BD0FC0EDBCFE6FFFD0EDBCFE6FF38
:1091E000D8DAE552E552FBEC3BF00DD0FC0EDBCFBC
:1091F000E6FFFD0EDBCFE6FFCCDAE552E552FBECF5
:109200003BF0000E01D09ED6146E060EE15C02E229
:10921000E16AE552E16E1450E552E5CFDAFFE7CF9F
:10922000D9FF1200D9CFE6FFDACFE6FFE1CFD9FFB1
:10923000E2CFDAFFE652E652010EDB6AFC0EDBCF2C
:10924000E9FFFD0EDBCFEAFF1A0EE926000EEA2247
:10925000EF50000864E2FA0EDBCFE6FFFB0EDBCF37
:10926000E6FFFC0EDBCFE6FFFD0EDBCFE6FFFAD913
:10927000E552E552E552E552FC0EDBCFE9FFFD0E6B
:10928000DBCFEAFF1A0EE926000EEA22EF06FC0EFB
:10929000DBCFE9FFFD0EDBCFEAFF1D0EE926000E56
:1092A000EA22EF50FF082DE1FC0EDBCFE9FFFD0EB7
:1092B000DBCFEAFF080EE926000EEA22EF502CE091
:1092C000FC0EDBCFE9FFFD0EDBCFEAFF080EE9263F
:1092D000000EEA22E9CF14F0EACF15F0E9CFE6FF5D
:1092E000EACFE6FF56EC3FF0E552E552000914E004
:1092F000F80EDBCFE9FFF90EDBCFEAFF010EEF6ED0
:109300000BD0FC0EDBCFE9FFFD0EDBCFEAFF1D0E1D
:10931000E926000EEA22EF2A010EDF6E01D0DF6A95
:10932000DF50E552E552E552E5CFDAFFE7CFD9FF4E
:109330001200D9CFE6FFDACFE6FFE1CFD9FFE2CFC7
:10934000DAFFE652F250E66EF29EFC0EDBCFE9FF4A
:10935000FD0EDBCFEAFF1A0EE926000EEA22EFCF60
:10936000DFFFE552E7BEF28EDF5000D0E552E55256
:10937000E5CFDAFFE7CFD9FF1200D9CFE6FFDACF8A
:10938000E6FFE1CFD9FFE2CFDAFFE652FC0EDBCFFA
:10939000E9FFFD0EDBCFEAFF1A0EE926000EEA22F6
:1093A000EFCFDFFFDF50E552E552E5CFDAFFE7CF41
:1093B000D9FF1200D9CFE6FFDACFE6FFE1CFD9FF20
:1093C000E2CFDAFFFC0EDBCFE9FFFD0EDBCFEAFFD9
:1093D000EECFE6FFEFCFE6FFC2EC72F0E552E552CA
:1093E000FC0EDBCFE6FFFD0EDBCFE6FFC2EC72F03A
:1093F000E552E552E552E5CFDAFFE7CFD9FF12009B
:10940000D9CFE6FFDACFE6FFE1CFD9FFE2CFDAFF2F
:10941000FC0EDBCFE9FFFD0EDBCFEAFF1C0EE926D9
:10942000000EEA22EF5001E10CD1F90EDB5001E011
:109430007AD0FC0EDBCFE9FFFD0EDBCFEAFF1C0E7E
:10944000E926000EEA22EF50E66EE66AFA0EDBCF5E
:10945000E6FFFB0EDBCFE6FFFC0EDBCFE9FFFD0EE8
:10946000DBCFEAFF040EE926000EEA22EECFE6FF8C
:10947000EFCFE6FF5AEC6EF0146E060EE15C02E2EE
:10948000E16AE552E16E1450FC0EDBCFE9FFFD0E00
:10949000DBCFEAFF1C0EE926000EEA22EF50146E25
:1094A000156AFC0EDBCFE9FFFD0EDBCFEAFF040EF1
:1094B000E926000EEA221450EE261550ED22FC0E8D
:1094C000DBCFE9FFFD0EDBCFEAFF040EE926000E3D
:1094D000EA22EECF14F0EFCF15F0FC0EDBCFE9FF60
:1094E000FD0EDBCFEAFF020EE926000EEA22EECFE8
:1094F00016F0EFCF17F01650145C1750155801E214
:10950000A0D0FC0EDBCFE9FFFD0EDBCFEAFFEECFF4
:1095100014F0EFCF15F0FC0EDBCFE9FFFD0EDBCF33
:10952000EAFF040E87D0FC0EDBCFE9FFFD0EDBCF98
:10953000EAFF1C0EE926000EEA22EF50E66EE66A0C
:10954000FA0EDBCFE6FFFB0EDBCFE6FFFC0EDBCF38
:10955000E9FFFD0EDBCFEAFF060EE926000EEA2248
:10956000EECFE6FFEFCFE6FF5AEC6EF0146E060E7C
:10957000E15C02E2E16AE552E16E1450FC0EDBCFE1
:10958000E9FFFD0EDBCFEAFF1C0EE926000EEA2202
:10959000EF50146E156AFC0EDBCFE9FFFD0EDBCF3A
:1095A000EAFF060EE926000EEA221450EE5E155080
:1095B000ED5AFC0EDBCFE9FFFD0EDBCFEAFF060E16
:1095C000E926000EEA22EECF14F0EFCF15F0FC0EE4
:1095D000DBCFE9FFFD0EDBCFEAFFEECF16F0EFCFDA
:1095E00017F01650145C175015582BE2FC0EDBCF09
:1095F000E9FFFD0EDBCFEAFF1C0EE926000EEA2292
:10960000EF50166E176AFC0EDBCFE9FFFD0EDBCFC5
:10961000EAFF020EE926000EEA221650EE5C146EF6
:109620001750EE58156EFC0EDBCFE9FFFD0EDBCFB9
:10963000EAFF060EE926000EEA2214C0EEFF15C06E
:10964000EDFFFC0EDBCFE9FFFD0EDBCFEAFF1A0ECC
:10965000E926000EEA22EF2AE552E5CFDAFFE7CF4E
:10966000D9FF1200D9CFE6FFDACFE6FFE1CFD9FF6D
:10967000E2CFDAFFFC0EDBCFE9FFFD0EDBCFEAFF26
:10968000EE50ED1001E17FD0FC0EDBCFE9FFFD0EC7
:10969000DBCFEAFF1C0EE926000EEA22EF50146E23
:1096A000156AFC0EDBCFE9FFFD0EDBCFEAFF060EED
:1096B000E926000EEA221450EE261550ED22FC0E8B
:1096C000DBCFE9FFFD0EDBCFEAFF060EE926000E39
:1096D000EA22EECF14F0EFCF15F0FC0EDBCFE9FF5E
:1096E000FD0EDBCFEAFF020EE926000EEA22EECFE6
:1096F00016F0EFCF17F01650145C1750155818E3FA
:10970000FC0EDBCFE9FFFD0EDBCFEAFFEECF14F05E
:10971000EFCF15F0FC0EDBCFE9FFFD0EDBCFEAFF4C
:10972000060EE926000EEA2214C0EEFF15C0EDFF7A
:10973000FC0EDBCFE9FFFD0EDBCFEAFF1C0EE926B6
:10974000000EEA22EF50E66EE66AFC0EDBCFE9FF80
:10975000FD0EDBCFEAFF060EE926000EEA22EECF71
:10976000E6FFEFCFE6FFFA0EDBCFE6FFFB0EDBCF27
:10977000E6FF5AEC6EF0146E060EE15C02E2E16A5E
:10978000E552E16E1450E552E5CFDAFFE7CFD9FF9D
:109790001200D9CFE6FFDACFE6FFE1CFD9FFE2CF63
:1097A000DAFFF250E66EF29EFC0EDBCFE9FFFD0E13
:1097B000DBCFEAFF1E0EE926000EEA22EFCF14F0FF
:1097C000000EE76E1418E8AE02D0143403D0E75050
:1097D000D880145434E2FC0EDBCFE9FFFD0EDBCF62
:1097E000EAFF110EE926000EEA22EF5026E0FC0EF9
:1097F000DBCFE9FFFD0EDBCFEAFF110EE926000EFD
:10980000EA22E9CF14F0EACF15F014C0E6FF15C044
:10981000E6FF56EC3FF0E552E552000902E0DAECD3
:1098200040F0FC0EDBCFE9FFFD0EDBCFEAFF1E0EA2
:10983000E926000EEA22EF0601D001D0B5D7FC0ED2
:10984000DBCFE9FFFD0EDBCFEAFF1E0EE926000E9F
:10985000EA22EF68E552E7BEF28EF250E66EF29E23
:10986000FC0EDBCFE9FFFD0EDBCFEAFF1D0EE92684
:10987000000EEA22EFCF14F0000EE76E1418E8AEE7
:1098800002D0143403D0E750D880145434E2FC0ED4
:10989000DBCFE9FFFD0EDBCFEAFF080EE926000E65
:1098A000EA22EF5026E0FC0EDBCFE9FFFD0EDBCF16
:1098B000EAFF080EE926000EEA22E9CF14F0EACF0B
:1098C00015F014C0E6FF15C0E6FF56EC3FF0E55278
:1098D000E552000902E0DAEC40F0FC0EDBCFE9FFD4
:1098E000FD0EDBCFEAFF1D0EE926000EEA22EF0691
:1098F00001D001D0B5D7FC0EDBCFE9FFFD0EDBCFE9
:10990000EAFF1D0EE926000EEA22EF68E552E7BEE7
:10991000F28EE552E5CFDAFFE7CFD9FF1200D9CFBB
:10992000E6FFDACFE6FFE1CFD9FFE2CFDAFFE6527A
:10993000F250E66EF29EFC0EDBCFE9FFFD0EDBCFB0
:10994000EAFF1A0EE926000EEA22EF5002E0000EAE
:1099500001D0010EDF6EE552E7BEF28EDF5000D07F
:10996000E552E552E5CFDAFFE7CFD9FF1200D9CFB4
:10997000E6FFDACFE6FFE1CFD9FFE2CFDAFFE6522A
:10998000FC0EDBCFE9FFFD0EDBCFEAFF1A0EE92666
:10999000000EEA22EF5002E0000E01D0010EDF6E51
:1099A000DF50E552E552E5CFDAFFE7CFD9FF1200ED
:1099B000D9CFE6FFDACFE6FFE1CFD9FFE2CFDAFF7A
:1099C000E652F250E66EF29EFC0EDBCFE9FFFD0E92
:1099D000DBCFEAFF1A0EE926000EEA22EFCF14F0E1
:1099E000FC0EDBCFE9FFFD0EDBCFEAFF1B0EE92605
:1099F000000EEA22EF50145C02E0000E01D0010ECE
:109A0000DF6EE552E7BEF28EDF5000D0E552E55240
:109A1000E5CFDAFFE7CFD9FF1200D9CFE6FFDACFE3
:109A2000E6FFE1CFD9FFE2CFDAFFE652FC0EDBCF53
:109A3000E9FFFD0EDBCFEAFF1A0EE926000EEA224F
:109A4000EFCF14F0FC0EDBCFE9FFFD0EDBCFEAFF1A
:109A50001B0EE926000EEA22EF50145C02E0000E15
:109A600001D0010EDF6EDF50E552E552E5CFDAFF9F
:069A7000E7CFD9FF120050
:0A9A7600D9CFE6FFDACFE6FFE1CF1B
:109A8000D9FFE2CFDAFFE652A098636A626A0F015B
:109A9000160E5F6F9F0E5D6F7B0E5C6F658C5E6B4D
:109AA000030EE66EE66AE66A4D0EE66E0F0EE66E91
:109AB000A8EC6EF0146E050EE15C02E2E16AE5527C
:109AC000E16E1450659CDF6ADF50146E156A100E4B
:109AD000145C000E155810E2DF50040DF3CFE9FFBF
:109AE000F4CFEAFF000EE926040EEA22EE6AEE6ADF
:109AF000EE6AEE6ADF2AE8D70F01160E4C6F62A6F7
:109B000002D06296FCD70F011C6B216B226B236B7A
:109B10006598DF6A040EDF5C18E2EA6ADF34FE0B48
:109B2000EA36E96E0F0EE9260F0EEA22EE6AED6ABA
:109B3000EA6ADF34FE0BEA36E96E070EE9260F0EFD
:109B4000EA22EE6AED6ADF2AE5D70F01080E0F6FF1
:109B5000040E106F016B006BE552E552E5CFDAFFA2
:109B6000E7CFD9FF1200D9CFE6FFDACFE6FFE1CF8A
:109B7000D9FFE2CFDAFFE6520F01000509E165BA2D
:109B800007D0626A0F015C815C890F01020E006FD1
:109B90006250040B06E00F015C51040B02E062947A
:109BA000D0D865B26BD06250010B17E00F015C5149
:109BB000010B13E060DFD08EA288A088F28E0F0127
:109BC000040E006F0401400E026F040E036F080EB6
:109BD000016F006B8C0E001362906250100B05E059
:109BE0000F015C51100B01E095D86250400B18E05A
:109BF0000F015C51400B14E0010EE66EE66A000EA8
:109C0000E66EE66A730EE66EE66AFAEC6FF0146EC4
:109C1000060EE15C02E2E16AE552E16E1450629CDC
:109C20006250200B05E00F015C51200B01E058D879
:109C30006250020B18E00F015C51020B14E0010EA0
:109C4000E66EE66A000EE66EE66AE6687F0EE66E8F
:109C5000FAEC6FF0146E060EE15C02E2E16AE55286
:109C6000E16E1450636A040E0F01E76E0019E8AE4E
:109C700002D0E73402D0E750005D02E2A19829D07B
:109C80000F015CA725D0DF6A040EDF5C21E262A62B
:109C90001FD064CF2AFF6296780E0F012A1502E1C9
:109CA0006AD814D0000EE66EE66A2A0EE66E0F0E33
:109CB000E66E720EE66EE66AFAEC6FF0146E060E51
:109CC000E15C02E2E16AE552E16E1450DF2ADCD782
:109CD000A198E552E552E5CFDAFFE7CFD9FF1200B0
:109CE0000F014CA115D003CFE9FF04CFEAFFEF50DD
:109CF00080080DE10FCFE9FF10CFEAFFEF50840895
:109D000006E103CFE9FF04CFEAFF8C0EEF6E4C9122
:109D1000629A12000F015C8562986582000EE66E01
:109D2000E66AE66EE66A750EE66EE66AFAEC6FF0D3
:109D3000146E060EE15C02E2E16AE552E16E145037
:109D40001200000EE66EE66AE66EE66A740EE66ED5
:109D5000E66AFAEC6FF0146E060EE15C02E2E16A6C
:109D6000E552E16E145065920F015C9562A402D039
:109D70006294FCD71200D9CFE6FFDACFE6FFE1CF3D
:109D8000D9FFE2CFDAFFE652FD0E0F012A155AE1A4
:109D90007E0E2A15E8407F0B040DF3CF03FFF4CFAE
:109DA00004FF000E0327040E042303CF05FF04CF96
:109DB00006FF057503CFE9FF04CFEAFFEF503C0B28
:109DC000E842E8420D083CE103CFE9FF04CFEAFF97
:109DD000020EE926000EEA22EECF14F0EFCF15F0C6
:109DE000480E14182BE1040E151828E103CFE9FFE3
:109DF00004CFEAFF020EE926000EEA22400EEE6EC4
:109E0000040EED6EDF6ADF50146E156A080E145CE6
:109E1000000E155813E2DF50EA6A480FE96E040E8F
:109E2000EA22EF50E66EDF50EA6A400FE96E040E58
:109E3000EA22E552E750EF6EDF2AE5D70FD807D0C8
:109E400034D805D0FD0E2A15040801E154D8E55296
:109E5000E552E5CFDAFFE7CFD9FF12000FCFE9FFD8
:109E600010CFEAFFEF50800B05E00FCFE9FF10CFD6
:109E7000EAFFEF6A0F01176B186B1D6B1E6B1C6BF3
:109E8000C4D8000EE66EE66AE66EE66A030EE66E7B
:109E9000E66AFAEC6FF0146E060EE15C02E2E16A2B
:109EA000E552E16E1450F5EF51F0020E0F01185D0E
:109EB00002E155EF53F072D80F012B511AE105CF93
:109EC000E9FF06CFEAFFEE52080EEF6E05CFE9FF7D
:109ED00006CFEAFF020EE926000EEA22400EEE6EE1
:109EE000040EED6E05CFE9FF06CFEAFF8C0EEF6E94
:109EF00012002B6B1200D9CFE6FFDACFE6FFE1CFDD
:109F0000D9FFE2CFDAFFE6520FCFE9FF10CFEAFF29
:109F1000EF50400B01E0010EDF6E0F010F75080ED0
:109F2000005D0CE142C45EFF0F015E51000803E2D8
:109F30000F01100E02D00F01040E006F180526E16C
:109F40000FCFE9FF10CFEAFF020EE926000EEA224A
:109F5000480EEE6E040EED6E1ADB020E0F01175D59
:109F600006E10FCFE9FF10CFEAFF840E0DD0DF50DE
:109F700006E10FCFE9FF10CFEAFFC80E05D00FCFE3
:109F8000E9FF10CFEAFF880EEF6E01D007D8E55247
:109F9000E552E5CFDAFFE7CFD9FF1200D9CFE6FFD0
:109FA000DACFE6FFE1CFD9FFE2CFDAFFE652E652A1
:109FB0000F01186B0FCFE9FF10CFEAFFEF6A040E15
:109FC0000F19146E10CF15F0DE6E10CFDDFFDECF4F
:109FD000E9FFDDCFEAFFEF6A21AF0FD02451251151
:109FE000261109E007D026CFFBFF25CFFAFF0F018E
:109FF0002451F96EF8DF0F01219FE552E552E55239
:10A00000E5CFDAFFE7CFD9FF120004014051600B22
:10A01000E842E842E842E842E842000901E0120072
:10A0200041510C0A54E00B0A3FE00C0A31E0010AEE
:10A0300022E00B0A1EE0020A1CE0030A18E0080AEC
:10A0400010E0010A0CE00F0A08E0030A01E0120028
:10A050000F011C8F080E006F1200F5EF50F0F6EFA5
:10A0600053F00F01010E196F0F0E1A6F0CD099EFFC
:10A0700051F068EF50F044510F01196F1A6B020E46
:10A0800019270F0E1A231C81010E1D6F1C8F120041
:10A090000F011C8F04014451EA6A020FE96E0F0E92
:10A0A000EA2242C4EFFF1200000EE66EE66AE66E98
:10A0B000E66A020EE66EE66AFAEC6FF0146E060EC1
:10A0C000E15C02E2E16AE552E16E14501200120016
:10A0D000D9CFE6FFDACFE6FFE1CFD9FFE2CFDAFF53
:10A0E000E652E652E652E6520401420510E14051C2
:10A0F0001F0B00090CE10F011C8F030E0401415DD1
:10A1000004E10F01010E296F02D00F01296B040138
:10A1100042515FE140511F0B02085BE144510F0BBC
:10A12000000957E00F011C8F040144BF0BD04451BC
:10A130000F0BE96EEA6AD890E936EA36070EE9268F
:10A140000F0E0AD044510F0BE96EEA6AD890E93637
:10A15000EA360F0EE9260F0EEA22EECFDEFFEDCF34
:10A16000DDFF030E415D06E1DECFE9FFDDCFEAFF53
:10A17000840E2ED044510F0B156A4C0F146E0F0E27
:10A180001522020E14C0DBFF030E15C0DBFF020E0A
:10A19000DBCFE9FF030EDBCFEAFFEF9044AF0CD03B
:10A1A000DECFE9FFDDCFEAFFEF6ADF74DECFE9FF44
:10A1B000DDCFEAFF400E0CD0DECFE9FFDDCFEAFFB6
:10A1C000880EEF6EDF74DECFE9FFDDCFEAFFC80E49
:10A1D000EF6E040EE15C02E2E16AE552E16EE552E7
:10A1E000E5CFDAFFE7CFD9FF1200800E0401405D12
:10A1F00001E09ED00F01C00E1C6F04014351030A01
:10A2000057E0010A0CE0030A01E090D00F01BC0EF8
:10A21000196FE50E1A6F000E1B6F120E81D07D0EA6
:10A22000146EE60E156E000E166E42C417F0186A14
:10A23000196A030E0C6E0D6A0E6A17C007F018C07B
:10A2400008F019C009F076EC71F014500424F36E94
:10A2500015500520F46E16500620F86EF4CFF7FF67
:10A26000F3CFF6FF0900F5CF19FF0900F5CF1AFF6C
:10A270000800F5CF1BFF19CFF6FF1ACFF7FF1BCF52
:10A28000F8FF020EF626000EF722F8220800F5CF9E
:10A290001DFF19CFF6FF1ACFF7FF1BCFF8FF030EF4
:10A2A000F626000EF722F8220800F5CF1EFF120056
:10A2B000030E425D38E2800E146EE60E156E000E3F
:10A2C000166E42C417F0186A196A030E0C6E0D6AF6
:10A2D0000E6A17C007F018C008F019C009F076EC34
:10A2E00071F014500424F36E15500520F46E1650CE
:10A2F0000620F86EF4CFF7FFF3CFF6FF0900F5CF95
:10A3000019FF0900F5CF1AFF0800F5CF1BFF19CF81
:10A31000F6FF1ACFF7FF1BCFF8FF0800F5500F012B
:10A320001D6F1E6B12000F011C6B12000F011C6BC6
:10A330001200D9CFE6FFDACFE6FFE1CFD9FFE2CFB7
:10A34000DAFFE652E6520401486B496B40511F0B9D
:10A35000020A11E0030A0CE0010A35E10F011C8F2B
:10A36000040148810F0129052EE1040148832BD007
:10A370000F011C8F28D00F011C8F040144BF0BD08C
:10A3800044510F0BE96EEA6AD890E936EA36070EB7
:10A39000E9260F0E0AD044510F0BE96EEA6AD890F5
:10A3A000E936EA360F0EE9260F0EEA22EECFDEFF7F
:10A3B000EDCFDDFFDECFE9FFDDCFEAFFEF50040B8D
:10A3C00002E0010E486F0F011CAF07D0480E196F55
:10A3D000040E1A6F1C81020E1D6FE552E552E55204
:10A3E000E5CFDAFFE7CFD9FF120065980F011CBF58
:10A3F00047D021AF26D0020E186F0FCFE9FF10CF44
:10A40000EAFFEE52EF6A0FCFE9FF10CFEAFFC80E66
:10A41000EF6E05CFE9FF06CFEAFFEE52080EEF6EB2
:10A4200005CFE9FF06CFEAFF020EE926000EEA2279
:10A43000480EEE6E040EED6E05CFE9FF06CFEAFF83
:10A440007AD005CFE9FF06CFEAFFEE52080EEF6E95
:10A4500005CFE9FF06CFEAFF020EE926000EEA2249
:10A46000400EEE6E040EED6E05CFE9FF06CFEAFF5B
:10A470008C0EEF6E0FCFE9FF10CFEAFF840E5CD099
:10A4800021BF84D0040140AF59D00F011D510401F8
:10A49000465D0F011E510401475904E246C41DFFE9
:10A4A00047C41EFF74D80F01010E186F05CFE9FFD6
:10A4B00006CFEAFFEE52080EEF6E05CFE9FF06CF9A
:10A4C000EAFF020EE926000EEA22400EEE6E040EAE
:10A4D000ED6E05CFE9FF06CFEAFF800EEF6E2B6B26
:10A4E00003CFE9FF04CFEAFFEE52080EEF6E03CF71
:10A4F000E9FF04CFEAFF020EE926000EEA22400E31
:10A50000EE6E040EED6E03CFE9FF04CFEAFF840E7A
:10A51000EF6E010E2B6F0FCFE9FF10CFEAFF020E97
:10A52000E926000EEA22480EEE6E040EED6E0FCF05
:10A53000E9FF10CFEAFFC80EEF6E12000F01020E06
:10A54000186F0FCFE9FF10CFEAFFEE52EF6A0FCF7F
:10A55000E9FF10CFEAFFC80EEF6E05CFE9FF06CF87
:10A56000EAFFEE52080EEF6E05CFE9FF06CFEAFFD5
:10A57000020EE926000EEA22480EEE6E040EED6E83
:10A5800005CFE9FF06CFEAFFC80EEF6E1200D9CF64
:10A59000E6FFDACFE6FFE1CFD9FFE2CFDAFFE652FE
:10A5A000E6520F01080E1D5D000E1E590DE21DCF73
:10A5B000DEFF1ECFDDFF175102E1010E03D01705AC
:10A5C00006E1020E176F03D0080EDE6EDD6A0FCFB4
:10A5D000E9FF10CFEAFFEF920FCFE9FF10CFEAFFBC
:10A5E000EF900FCFE9FF10CFEAFF010EDB50EF1223
:10A5F0000FCFE9FF10CFEAFFEE52DFCFEFFF000EE3
:10A60000DB501D5F010EDB501E5B480E276F040EF2
:10A61000286F1CB123D0D9CFE9FFDACFEAFFEE5083
:10A62000ED103BE019CFF6FF192B1ACFF7FF000E04
:10A630001A231BCFF8FF1B230800F550E66E27CF27
:10A64000E9FF28CFEAFF272B000E2823E552E75029
:10A65000EF6EDF06010EDFE2DB06DDD7D9CFE9FFC3
:10A66000DACFEAFFEE50ED1018E019CFE9FF1ACF6C
:10A67000EAFF192B000E1A23EF50E66E27CFE9FFF1
:10A6800028CFEAFF272B000E2823E552E750EF6E74
:10A69000DF06010EE3E2DB06E1D7E552E552E552C3
:10A6A000E5CFDAFFE7CFD9FF1200D9CFE6FFDACF47
:10A6B000E6FFE1CFD9FFE2CFDAFFE652E65203CF61
:10A6C000E9FF04CFEAFFEE52EFCFDFFFDFCF14F058
:10A6D00014500F01225D000E235902E222CFDFFF4A
:10A6E000DF50146E156AE850225D226F1550235911
:10A6F000236F010EDB6ADF50F36E010EDBCFF4FF38
:10A70000F350F45C16E2010EDB50EA6A480FE96E82
:10A71000040EEA22EF50E66E1FCFE9FF20CFEAFFDA
:10A720001F2B000E2023E552E750EF6E010EDB2AAF
:10A73000E2D7000ED8802255000E235527E205CF20
:10A74000E9FF06CFEAFFEE52080EEF6E05CFE9FFF4
:10A7500006CFEAFF020EE926000EEA22480EEE6E50
:10A76000040EED6E03CFE9FF04CFEAFFEF50400B7C
:10A7700006E105CFE9FF06CFEAFFC80E05D005CFF9
:10A78000E9FF06CFEAFF880EEF6E28D005CFE9FF7C
:10A7900006CFEAFFEE52080EEF6E05CFE9FF06CFB7
:10A7A000EAFF020EE926000EEA22400EEE6E040ECB
:10A7B000ED6E05CFE9FF06CFEAFF840EEF6E245160
:10A7C0002511261109E007D026CFFBFF25CFFAFF80
:10A7D0000F012451F96EF8DF0F01219FE552E55278
:10A7E000E552E5CFDAFFE7CFD9FF1200D9CFE6FF78
:10A7F000DACFE6FFE1CFD9FFE2CFDAFFE6520F0171
:10A800001C8F030EE66EE66AE66A4D0EE66E0F0ECC
:10A81000E66EA8EC6EF0146E050EE15C02E2E16AF1
:10A82000E552E16E1450DF6ADF50146E156A100EA7
:10A83000145C000E155810E2DF50040DF3CFE9FF51
:10A84000F4CFEAFF000EE926040EEA22EE6AEE6A71
:10A85000EE6AEE6ADF2AE8D7658C010EE66EE66ADC
:10A86000E66A020EE66E0F0EE66EA8EC6EF0146E4F
:10A87000050EE15C02E2E16AE552E16E1450659C6E
:10A880000F01080E0F6F040E106F000E036F040E01
:10A89000046F03CF05FF066F42C401FF015102E1BF
:10A8A000100E16D0010EE66EE66A010EE66E0F0E71
:10A8B000E66E010EE66EE66AFAEC6FF0146E060EB6
:10A8C000E15C02E2E16AE552E16E14500F01200EF4
:10A8D000006FE552E552E5CFDAFFE7CFD9FF12006E
:10A8E000D9CFE6FFDACFE6FFE1CFD9FFE2CFDAFF3B
:10A8F000E652E652000EDE6E040EDD6EFC0EDB50FC
:10A90000E824166EFD0EDB50040DF3501624040DE2
:10A91000F350146E156A020E0F0B05E0D890153235
:10A920001432E806FBE1D89014361536D890143668
:10A930001536D9CFE9FFDACFEAFF1450EE261550CD
:10A94000ED22DECFE9FFDDCFEAFFEF9EFC0EDB500C
:10A950000AE1FD0EEA6ADB34FE0BEA36E96E070E09
:10A96000E9260F0E09D0FD0EEA6ADB34FE0BEA364B
:10A97000E96E0F0EE9260F0EEA22DECFEEFFDDCFE5
:10A98000EDFFDECFE9FFDDCFEAFFEF9CDECFE9FF91
:10A99000DDCFEAFF040EE926000EEA22EF8CE55235
:10A9A000E552E552E5CFDAFFE7CFD9FF1200D9CF64
:10A9B000E6FFDACFE6FFE1CFD9FFE2CFDAFFE652DA
:10A9C000E652FD0EDB50156A4C0F146E0F0E152269
:10A9D00014C0DEFF15C0DDFFDECFE9FFDDCFEAFFEB
:10A9E000FC0EDBCFEFFFDBA407D0E66AFD0EDBCF6A
:10A9F000E6FF76DFE552E552FC0EDBA208D0010E41
:10AA0000E66EFD0EDBCFE6FF6BDFE552E552E55269
:10AA1000E552E552E5CFDAFFE7CFD9FF1200D9CFF3
:10AA2000E6FFDACFE6FFE1CFD9FFE2CFDAFFE65269
:10AA3000E652FD0EDB5020E105CFE9FF06CFEAFF2D
:10AA4000EE52080EEF6E05CFE9FF06CFEAFF020EC9
:10AA5000E926000EEA22400EEE6E040EED6E05CFE2
:10AA6000E9FF06CFEAFF8C0EEF6E0FCFE9FF10CFA4
:10AA7000EAFF840EEF6E3BD0FC0EDB50E824166E2E
:10AA8000FD0EDB50040DF3501624040DF3CF14F02B
:10AA9000F4CF15F0000E1426040E152214C0DEFFAC
:10AAA00015C0DDFF840EDECFE9FFDDCFEAFFE85001
:10AAB000EF12FC0EDB50E824166EFD0EDB50040D89
:10AAC000F3501624010F040DF3CF14F0F4CF15F05A
:10AAD000000E1426040E152214C0DEFF15C0DDFF83
:10AAE000840EDECFE9FFDDCFEAFFE850EF12E5523A
:10AAF000E552E552E5CFDAFFE7CFD9FF1200D9CF13
:10AB0000E6FFDACFE6FFE1CFD9FFE2CFDAFFE65288
:10AB1000E652FC0EDB500AE0FD0EEA6ADB34FE0B67
:10AB2000EA36E96E0F0EE9260F0E09D0FD0EEA6A2D
:10AB3000DB34FE0BEA36E96E070EE9260F0EEA2239
:10AB4000EECFDEFFEDCFDDFFD9CFE9FFDACFEAFFB1
:10AB5000EE50ED1003E1F36AF46A44D0DECFE9FF72
:10AB6000DDCFEAFF020EE926000EEA22FA0EDBCF65
:10AB7000EEFFFB0EDBCFEDFFDECFE9FFDDCFEAFF1F
:10AB8000EE52F90EDBCFEFFF400EDECFE9FFDDCF57
:10AB9000EAFFE850EF16880EDECFE9FFDDCFEAFFCF
:10ABA000E850EF12FC0EDB500AE0FD0EEA6ADB34DF
:10ABB000FE0BEA36E96E0F0EE9260F0E09D0FD0EE8
:10ABC000EA6ADB34FE0BEA36E96E070EE9260F0E61
:10ABD000EA22EF74DECF14F0DDCF15F014C0F3FFDE
:10ABE00015C0F4FFE552E552E552E5CFDAFFE7CFB5
:10ABF000D9FF1200D9CFE6FFDACFE6FFE1CFD9FFC8
:10AC0000E2CFDAFF65A84ED0FD0EEA6ADB34FE0B18
:10AC1000EA36E96E0F0EE9260F0EEA22EE50EFCF6C
:10AC2000EAFFE96E400EEE16EE6AEE6AEE6AFD0E7F
:10AC3000EA6ADB34FE0BEA36E96E0F0EE9260F0EE8
:10AC4000EA22EE50EFCFEAFFE96EEE7CFD0EEA6AF3
:10AC5000DB34FE0BEA36E96E0F0EE9260F0EEA2210
:10AC6000EF74400E146EFD0EEA6ADB34FE0BEA361A
:10AC7000E96E0F0EE9260F0EEA22EE50EFCFEAFF43
:10AC8000E96E1450EF16FD0EEA6ADB34FE0BEA366D
:10AC9000E96E0F0EE9260F0EEA22EE50EFCFEAFF23
:10ACA000E96EEF7CE552E5CFDAFFE7CFD9FF12007E
:10ACB000656A0F015C6B0F01006B12000F01005100
:10ACC00014E1656A0F015C6B160E5F6F9F0E5D6F7E
:10ACD0007B0E5C6FD08EA288A088F28E65B602D003
:0CACE0006586FCD70F01010E006F12000A
:04ACEC00D9CFE6FFD7
:10ACF000DACFE6FFE1CFD9FFE2CFDAFFE652E65244
:10AD0000E652E652E652FC0EDBCFE9FFFD0EDBCF4A
:10AD1000EAFF110EEF6EFC0EDB2AFD0E01E3DB2ACB
:10AD2000FC0EDBCFE9FFFD0EDBCFEAFF220EEF6E5C
:10AD3000FC0EDB2AFD0E01E3DB2AFC0EDBCFE9FF74
:10AD4000FD0EDBCFEAFF330EEF6EFC0EDB2AFD0EAD
:10AD500001E3DB2AF70EDBCF14F0F80EDBCF15F0A2
:10AD6000000E14C0DFFF010E15C0DBFF020EDB6A10
:10AD7000030EDB6AD9CFE9FFDACFEAFFEECF14F09A
:10AD8000EECF15F0EECF16F01450E66EFC0EDBCFD2
:10AD9000E9FFFD0EDBCFEAFFE552E750EF6EFC0E58
:10ADA000DB2AFD0E01E3DB2AD9CFE9FFDACFEAFF88
:10ADB000080EE76ED890030EEB32020EEB32010E56
:10ADC000EB32EF32E706F6E1D9CFE9FFDACFEAFF5F
:10ADD000EECF14F0EECF15F0EECF16F01450E66E75
:10ADE000FC0EDBCFE9FFFD0EDBCFEAFFE552E750BB
:10ADF000EF6EFC0EDB2AFD0E01E3DB2AFC0EDBCF3F
:10AE0000E9FFFD0EDBCFEAFF440EEF6EFC0EDB2AFE
:10AE1000FD0E01E3DB2AFC0EDBCFE9FFFD0EDBCFED
:10AE2000EAFF660EEF6EFC0EDB2AFD0E01E3DB2A65
:10AE3000FC0EDBCFE9FFFD0EDBCFEAFFCC0EEF6EA1
:10AE4000FC0EDB2AFD0E01E3DB2AFC0EDBCFE9FF63
:10AE5000FD0EDBCFEAFFC00EEF6EFC0EDB2AFD0E0F
:10AE600001E3DB2AFC0EDBCFE9FFFD0EDBCFEAFFBF
:10AE7000110EEF6EFC0EDB2AFD0E01E3DB2AFC0E49
:10AE8000DBCFE9FFFD0EDBCFEAFF220EEF6EFC0EFB
:10AE9000DB2AFD0E01E3DB2AFC0EDBCFE9FFFD0E12
:10AEA000DBCFEAFF330EEF6EFC0EDB2AFD0E01E373
:10AEB000DB2AFC0EDBCFE9FFFD0EDBCFEAFF440E01
:10AEC000EF6EFC0EDB2AFD0E01E3DB2AFC0EDBCF6E
:10AED000E9FFFD0EDBCFEAFF550EEF6EFC0EDB2A1D
:10AEE000FD0E01E3DB2AFC0EDBCFE9FFFD0EDBCF1D
:10AEF000EAFF660EEF6EFC0EDB2AFD0E01E3DB2A95
:10AF0000FC0EDBCFE9FFFD0EDBCFEAFFEF6AFC0EA4
:10AF1000DB2AFD0E01E3DB2AFC0EDBCFE9FFFD0E91
:10AF2000DBCFEAFF880EEF6EFC0EDB2AFD0E01E39D
:10AF3000DB2AFC0EDBCFE9FFFD0EDBCFEAFF990E2B
:10AF4000EF6EFC0EDB2AFD0E01E3DB2AFC0EDBCFED
:10AF5000E9FFFD0EDBCFEAFFAA0EEF6EFC0EDB2A47
:10AF6000FD0E01E3DB2AFC0EDBCFE9FFFD0EDBCF9C
:10AF7000EAFFBB0EEF6EFC0EDB2AFD0E01E3DB2ABF
:10AF8000FC0EDBCFE9FFFD0EDBCFEAFFEF6AFC0E24
:10AF9000DB2AFD0E01E3DB2AFC0EDBCFE9FFFD0E11
:10AFA000DBCFEAFFEF6AFC0EDB2AFD0E01E3DB2AB2
:10AFB000040EDB6ADB50130815E3FC0EDBCFE9FF60
:10AFC000FD0EDBCFEAFF040EDBCFEFFFFC0EDBCF85
:10AFD000E9FFDB2AFD0EDBCFEAFF01E3DB2A040EEB
:10AFE000DB2AE8D7FC0EDBCFE9FFFD0EDBCFEAFF63
:10AFF000130EEF6EFC0EDB2AFD0E01E3DB2AFC0EC6
:10B00000DBCFE9FFFD0EDBCFEAFFEF6AFC0EDB2AA8
:10B01000FD0E01E3DB2AF90EDBCF14F0FA0EDBCFD5
:10B0200015F0FB0EDBCF16F0176A14C0DFFF010E20
:10B0300015C0DBFF020E16C0DBFF030E17C0DBFFDF
:10B04000D9CFE9FFDACFEAFFEECF14F0EECF15F05B
:10B05000EECF16F01450E66EFC0EDBCFE9FFFD0ECE
:10B06000DBCFEAFFE552E750EF6EFC0EDB2AFD0E68
:10B0700001E3DB2AD9CFE9FFDACFEAFF080EE76E5A
:10B08000D890030EEB32020EEB32010EEB32EF32B0
:10B09000E706F6E1D9CFE9FFDACFEAFFEECF14F009
:10B0A000EECF15F0EECF16F01450E66EFC0EDBCFAF
:10B0B000E9FFFD0EDBCFEAFFE552E750EF6EFC0E35
:10B0C000DB2AFD0E01E3DB2AD9CFE9FFDACFEAFF65
:10B0D000080EE76ED890030EEB32020EEB32010E33
:10B0E000EB32EF32E706F6E1D9CFE9FFDACFEAFF3C
:10B0F000EECF14F0EECF15F0EECF16F01450E66E52
:10B10000FC0EDBCFE9FFFD0EDBCFEAFFE552E75097
:10B11000EF6EFC0EDB2AFD0E01E3DB2AFC0EDBCF1B
:10B12000E9FFFD0EDBCFEAFF010EEF6EFC0EDB2A1E
:10B13000FD0E01E3DB2AFC0EDBCF14F0FD0EDBCFAE
:10B1400015F014C0F3FF15C0F4FF050EE15C02E238
:10B15000E16AE552E16EE552E5CFDAFFE7CFD9FFCC
:10B16000120081DAF0CEE9FFF1CEEAFFEECFE1FF87
:10B17000EECFE2FFE5CFE9FFE5CFE9FFFC6AE9505A
:10B18000FC5C08E20500E550FF6EE550FE6EE55000
:10B19000FD6EF5D7E5CFEAFFE5CFE9FFE5CFEDFF9F
:10B1A000E5CFEDFFE5CFEDFFE5CFEDFFE5CFEDFF1F
:10B1B000E5CFEDFFE5CFEDFFE5CFEDFFE5CFEDFF0F
:10B1C000E5CFEDFFE5CFEDFFE5CFEDFFE5CFEDFFFF
:10B1D000E5CFEDFFE5CFEDFFE5CFEDFFE5CFEDFFEF
:10B1E000E5CFEDFFE5CFEDFFE5CFEFFFE5CFFAFFD0
:10B1F000E5CFFBFFE5CFF3FFE5CFF4FFE5CFF6FFAB
:10B20000E5CFF7FFE5CFF8FFE5CFF5FFE5CFEAFFA4
:10B21000E5CFE9FFE5CFDAFFE5CFD9FFE5CFE0FFE6
:10B22000E5CFE8FFE8AE06D0E5CFD8FFE5CFE8FFF1
:10B23000100005D0E5CFD8FFE5CFE8FF1200010EE2
:10B2400000D012001200E8CFE4FFD8CFE4FFF2CF25
:10B25000E8FF0009E8CFE4FFF29EE0CFE4FFD9CF9A
:10B26000E4FFDACFE4FFE9CFE4FFEACFE4FFF5CF74
:10B27000E4FFF8CFE4FFF7CFE4FFF6CFE4FFF4CF2D
:10B28000E4FFF3CFE4FFFBCFE4FFFACFE4FFE96A8A
:10B29000EA6AEECFE4FFEECFE4FFEECFE4FFEECFBD
:10B2A000E4FFEECFE4FFEECFE4FFEECFE4FFEECF1E
:10B2B000E4FFEECFE4FFEECFE4FFEECFE4FFEECF0E
:10B2C000E4FFEECFE4FFEECFE4FFEECFE4FFEECFFE
:10B2D000E4FFEECFE4FFEECFE4FFEECFE4FFEFCFED
:10B2E000E4FFE9CFE4FFEACFE4FFFCCFE9FFFC5045
:10B2F000000808E2FDCFE4FFFECFE4FFFFCFE4FF4C
:10B300000600F5D7E9CFE4FFE452F0CEE9FFF1CE35
:10B31000EAFFE1CFEEFFE2CFEEFF0BEC3EF0F0CE26
:10B32000E9FFF1CEEAFFEECFE1FFEECFE2FFE5CF9E
:10B33000E9FFE5CFE9FFFC6AE950FC5C08E20500A3
:10B34000E550FF6EE550FE6EE550FD6EF5D7E5CF9A
:10B35000EAFFE5CFE9FFE5CFEDFFE5CFEDFFE5CF74
:10B36000EDFFE5CFEDFFE5CFEDFFE5CFEDFFE5CF5D
:10B37000EDFFE5CFEDFFE5CFEDFFE5CFEDFFE5CF4D
:10B38000EDFFE5CFEDFFE5CFEDFFE5CFEDFFE5CF3D
:10B39000EDFFE5CFEDFFE5CFEDFFE5CFEDFFE5CF2D
:10B3A000EDFFE5CFEFFFE5CFFAFFE5CFFBFFE5CF00
:10B3B000F3FFE5CFF4FFE5CFF6FFE5CFF7FFE5CFED
:10B3C000F8FFE5CFF5FFE5CFEAFFE5CFE9FFE5CFF1
:10B3D000DAFFE5CFD9FFE5CFE0FFE5CFE8FFE8AE44
:10B3E00006D0E5CFD8FFE5CFE8FF100005D0E5CFC8
:10B3F000D8FFE5CFE8FF12001200D8CFE4FFE0CF7E
:10B40000E4FFE46EE9CFE4FFEACFE4FFF6CFE4FF28
:10B41000F7CFE4FFF8CFE4FFF5CFE4FFF3CFE4FF8D
:10B42000F4CFE4FFFACFE4FFFBCFE4FF00EE00F03F
:10B43000140EE80403E3EECFE4FFFBD700EE14F0B4
:10B44000120EE80403E3EECFE4FFFBD7E6529EB40E
:10B450002FD8F0A402D069EC23F0E55200EE25F0DD
:10B46000120EE80403E3E5CFEDFFFBD700EE13F087
:10B47000140EE80403E3E5CFEDFFFBD7E5CFFBFFB8
:10B48000E5CFFAFFE5CFF4FFE5CFF3FFE5CFF5FF1A
:10B49000E5CFF8FFE5CFF7FFE5CFF6FFE5CFEAFF11
:10B4A000E5CFE9FFE550E5CFE0FFE5CFD8FF10009D
:10B4B000E8CFE4FFD8CFE4FFF2CFE8FF8009E8CF80
:10B4C000E4FFF29EE0CFE4FFD9CFE4FFDACFE4FF60
:10B4D000E9CFE4FFEACFE4FFF5CFE4FFF8CFE4FFE4
:10B4E000F7CFE4FFF6CFE4FFF4CFE4FFF3CFE4FFC0
:10B4F000FBCFE4FFFACFE4FFE96AEA6AEECFE4FFAC
:10B50000EECFE4FFEECFE4FFEECFE4FFEECFE4FFBB
:10B51000EECFE4FFEECFE4FFEECFE4FFEECFE4FFAB
:10B52000EECFE4FFEECFE4FFEECFE4FFEECFE4FF9B
:10B53000EECFE4FFEECFE4FFEECFE4FFEECFE4FF8B
:10B54000EECFE4FFEECFE4FFEFCFE4FFE9CFE4FF7F
:10B55000EACFE4FFFCCFE9FFFC50000808E2FDCF92
:10B56000E4FFFECFE4FFFFCFE4FF0600F5D7E9CF0D
:10B57000E4FFE452F0CEE9FFF1CEEAFFE1CFEEFFC7
:10B58000E2CFEEFF9E940FEC3DF0F0CEE9FFF1CE5E
:10B59000EAFFEECFE1FFEECFE2FFE5CFE9FFE5CF37
:10B5A000E9FFFC6AE950FC5C08E20500E550FF6E2B
:10B5B000E550FE6EE550FD6EF5D7E5CFEAFFE5CF2D
:10B5C000E9FFE5CFEDFFE5CFEDFFE5CFEDFFE5CFFF
:10B5D000EDFFE5CFEDFFE5CFEDFFE5CFEDFFE5CFEB
:10B5E000EDFFE5CFEDFFE5CFEDFFE5CFEDFFE5CFDB
:10B5F000EDFFE5CFEDFFE5CFEDFFE5CFEDFFE5CFCB
:10B60000EDFFE5CFEDFFE5CFEDFFE5CFEDFFE5CFBA
:10B61000EFFFE5CFFAFFE5CFFBFFE5CFF3FFE5CF87
:10B62000F4FFE5CFF6FFE5CFF7FFE5CFF8FFE5CF75
:10B63000F5FFE5CFEAFFE5CFE9FFE5CFDAFFE5CF9C
:10B64000D9FFE5CFE0FFE5CFE8FFE8AE06D0E5CFD4
:10B65000D8FFE5CFE8FF100005D0E5CFD8FFE5CF54
:10B66000E8FF12001200D9CFE6FFDACFE6FFE1CF04
:10B67000D9FFE2CFDAFF090EE12402E3E168E652E6
:10B68000E16EE00EDE6E2E0EDE6EDE6ADD6ADD52EB
:10B69000DD52CF6ACE6AD9CFE9FFDACFEAFF040ED6
:10B6A000EECFDBFF050EEECFDBFF060EEECFDBFFAE
:10B6B000070EEECFDBFF040EDBCF14F0050E060EF7
:10B6C000070E1450BC6ED950040FE96E000EDA203C
:10B6D000EA6E080EE76ED890030EEB32020EEB32E4
:10B6E000010EEB32EF32E706F6E1040EDBCF14F089
:10B6F000050EDBCF15F0060EDBCF16F0070EDBCF05
:10B7000017F01450BD6EBB80BB82BB94BB869D847A
:10B71000F28CC50EE66EDEEC73F0E552090EE15CCC
:10B7200002E2E16AE552E16EE552E5CFDAFFE7CFEA
:04B73000D9FF12002B
:0CB73400D9CFE6FFDACFE6FFE1CFD9FF66
:10B74000E2CFDAFF0E01FD6BFE6BFD0EDBCFFFFEDD
:10B75000E552E5CFDAFFE7CFD9FF1200D9CFE6FFF8
:10B76000DACFE6FFE1CFD9FFE2CFDAFFE652E652C9
:10B77000DE52010EDD6ED950FC0FE96EFF0EDA20AD
:10B78000EA6EEE50ED105FE0010EDB505CE00E0162
:10B79000FD51146E156A2C0E141802E1155053E079
:10B7A000FE51E76EFC0EDBCFE9FFFD0EDBCFEAFFBB
:10B7B000E750E926000EEA22EF5026E00D0A11E0DC
:10B7C000370A0BE0150A04E0030A23E1DF6A1ED002
:10B7D000FF051FE1010EDF6E1AD0FF051AE1020E10
:10B7E00014D00A0E146EFE29E76EFC0EDBCFE9FFC3
:10B7F000FD0EDBCFEAFFE750E926000EEA22EF500C
:10B80000145C1FE1030E01D0030EDF6E010EDB6A34
:10B8100018D0FE51E76EFC0EDBCFE9FFFD0EDBCF4B
:10B82000EAFFE750E926000EEA22EF50E66EFD51EE
:10B83000FD2BEA6AB80FE96E0E0EEA22E552E750D8
:10B84000EF6EFE2BA1D70E01FD51EA6AB80FE96E2B
:10B850000E0EEA22EF6AFD6BDF50E552E552E5522B
:10B86000E5CFDAFFE7CFD9FF1200D9CFE6FFDACF75
:10B87000E6FFE1CFD9FFE2CFDAFFB80EE66E0E0E9B
:10B88000E66E0DEC6FF0E552E552F3CF14F0F4CF15
:10B8900015F0010EF3184AE1000E151847E1B8CE75
:10B8A00018F0196A18BE196818C0E6FF19C0E6FF3B
:10B8B00094EC73F0E552E552F3CF16F0F4CF17F0A5
:10B8C000F350F41033E00F0E0E01B815E66EFC0EC7
:10B8D000DBCFE9FFFD0EDBCFEAFFE552E750EF6E6D
:10B8E000FC0EDBCFE9FFFD0EDBCFEAFFEFCF14F05C
:10B8F000FB0EDB50E76E1418E8AE02D0E73402D03E
:10B90000E750145C13E3FA0EDBCF15F0FC0EDBCF2F
:10B91000E9FFFD0EDBCFEAFFEF50E76E1518E8AE4A
:10B9200002D0E73402D0E750155C02E2000E01D0ED
:10B93000010EE552E5CFDAFFE7CFD9FF1200D9CFEC
:10B94000E6FFDACFE6FFE1CFD9FFE2CFDAFFB80EAC
:10B95000E66E0E0EE66E0DEC6FF0E552E552F3CF9B
:10B9600014F0F4CF15F0020EF31864E1000E151870
:10B9700061E1B8CE18F0196A18BE196818C0E6FF60
:10B9800019C0E6FF94EC73F0E552E552F3CF16F0E0
:10B99000F4CF17F0F350F4104DE0B9CE1CF01D6A4F
:10B9A0001CBE1D681CC0E6FF1DC0E6FF94EC73F0D2
:10B9B000E552E552F3CF1AF0F4CF1BF0F350F41038
:10B9C00039E00F0E0E01B915146E0F0EB8150A0DE1
:10B9D000F3501424E66EFC0EDBCFE9FFFD0EDBCF47
:10B9E000EAFFE552E750EF6EFC0EDBCFE9FFFD0EFC
:10B9F000DBCFEAFFEFCF14F0FB0EDB50E76E14183D
:10BA0000E8AE02D0E73402D0E750145C13E3FA0E3C
:10BA1000DBCF15F0FC0EDBCFE9FFFD0EDBCFEAFF3D
:10BA2000EF50E76E1518E8AE02D0E73402D0E750C9
:10BA3000155C02E2000E01D0010EE552E5CFDAFFFF
:10BA4000E7CFD9FF1200D9CFE6FFDACFE6FFE1CF8B
:10BA5000D9FFE2CFDAFF3BEC24F0F3CFEEFEF4CFD8
:10BA6000EFFE010EE66E66DEE5520E01E56BEECEF0
:10BA7000E6FFEFCEE6FF72DEE552E552030A01E192
:10BA8000A7D0010A5AE0030A44E0010A01E0B2D05B
:10BA90000E01E551020A19E0030A04E0010A01E17E
:10BAA000B6D1A8D0040EE66E010EE66EE60EE66E86
:10BAB0000E0EE66EDADEE552E552E552E552000979
:10BAC00001E198D00E01E607A2D1B80EE66E0E0E87
:10BAD000E66E0DEC6FF0E552E552F3CF14F0F4CFC3
:10BAE00015F0010EF31801E085D0000E151801E0E5
:10BAF00081D00E01B851530A09E01C0A05E00C0A76
:10BB000001E078D0020E03D0E76B81D1010EE76F20
:10BB10007ED1050E0E01E55D6DE13B0EE66EE66A37
:10BB2000EC0EE66E0E0EE66E0ADFE552E552E552C9
:10BB3000E552000901E06BD15DD00E01E551070A25
:10BB400037E0010A25E0020A13E0070A01E05FD1AD
:10BB5000170EE66EE66AE80EE66E0E0EE66EEFDE95
:10BB6000E552E552E552E552000901E050D142D0DC
:10BB70003B0EE66EE66AEA0EE66E0E0EE66EDFDE5F
:10BB8000E552E552E552E552000901E040D132D0DC
:10BB9000170EE66EE66AE90EE66E0E0EE66ECFDE74
:10BBA000E552E552E552E552000901E030D122D0DC
:10BBB0003B0EE66EE66AEB0EE66E0E0EE66EBFDE3E
:10BBC000E552E552E552E552000901E020D112D0DC
:10BBD000080E0E01E55D0EE13B0EE66EE66AED0E27
:10BBE000E66E0E0EE66EABDEE552E552E552E5522C
:10BBF000000902E1000E0ED10E01E75134E0010A06
:10BC000002E0030A65E1E6CEE9FFEA6AE9BEEA6816
:10BC1000030ED890E936EA36E806FBE1FD0EE92688
:10BC2000020EEA22EE52EFCF14F0010EE76E141866
:10BC3000E8AE02D0143403D0E750D880145448E35F
:10BC4000E6CEE9FFEA6AE9BEEA68030ED890E93673
:10BC5000EA36E806FBE1FD0EE926020EEA22EE5284
:10BC6000010EEF6E35D0E6CEE9FFEA6AE9BEEA687A
:10BC7000030ED890E936EA36E806FBE1FD0EE92628
:10BC8000020EEA22EE52EF50020822E00E01E651C7
:10BC9000030A0CE0010A08E0030A04E0010A07E1D4
:10BCA0008D9005D08D9203D08D9401D08D96E6CEE7
:10BCB000E9FFEA6AE9BEEA68030ED890E936EA3697
:10BCC000E806FBE1FD0EE926020EEA22EE52EF6ADB
:10BCD000E6CEE9FFEA6AE9BEEA68030ED890E936E3
:10BCE000EA36E806FBE1FD0EE926020EEA22E7CE7F
:10BCF000EFFFE6CEE9FFEA6AE9BEEA68030ED890F4
:10BD0000E936EA36E806FBE1FD0EE926020EEA22F4
:10BD1000020EE926000EEA22E8CEEFFFE6CEE9FFAA
:10BD2000EA6AE9BEEA68030ED890E936EA36E80620
:10BD3000FBE1FD0EE926020EEA22020EE926000EC4
:10BD4000EA22EE52EACEEFFFE6CEE9FFEA6AE9BE6A
:10BD5000EA68030ED890E936EA36E806FBE1FD0E04
:10BD6000E926020EEA22020EE926000EEA22020E5F
:10BD7000E926000EEA22ECCEEFFFE6CEE9FFEA6A02
:10BD8000E9BEEA68030ED890E936EA36E806FBE138
:10BD9000FD0EE926020EEA22050EE926000EEA2231
:10BDA000E9CEEFFFE6CEE9FFEA6AE9BEEA68030EF4
:10BDB000D890E936EA36E806FBE1FD0EE926020EE8
:10BDC000EA22050EE926000EEA22EE52EBCEEFFF44
:10BDD000E6CEE9FFEA6AE9BEEA68030ED890E936E2
:10BDE000EA36E806FBE1FD0EE926020EEA22050E20
:10BDF000E926000EEA22020EE926000EEA22EDCE26
:10BE0000EFFF8FEC36F023EC59F0010E03D00E015A
:10BE1000E52B2DD6E552E5CFDAFFE7CFD9FF1200AB
:10BE2000D9CFE6FFDACFE6FFE1CFD9FFE2CFDAFFE5
:10BE3000E652966A9892FD0EDB50E8B08F82E8A039
:10BE40008F920F0E8D14DF6EFC0EDB50F00BDF10A7
:10BE50008D6E000000008F800000000000000000D8
:10BE6000000000000000000000008F90FC0EDB3896
:10BE7000F00BDF108D6E000000008F8000000000CE
:10BE800000000000000000000000000000008F9093
:10BE9000E552E552E5CFDAFFE7CFD9FF1200D9CF5F
:10BEA000E6FFDACFE6FFE1CFD9FFE2CFDAFF070EF8
:10BEB000E12402E3E168E652E16E200EE66EE66AF6
:10BEC000200EE66E240EE66E030EE66EA8EC6EF013
:10BED000146E050EE15C02E2E16AE552E16E145077
:10BEE0000301446B8F90966A98929890280EF36E97
:10BEF000010EF3CFDBFF020EDB6A010EDBCF14F085
:10BF0000DB06020EDBCF15F001E2DB061450151044
:10BF100006E00C0EE66E15EC74F0E552EED78F924B
:10BF2000300E8D6E00000000DF6A030EDF5C22E23F
:10BF30008F800C0EE66E41EC74F0E5528F90020E8D
:10BF4000F36E030EF3CFDBFF040EDB6A030EDBCFD1
:10BF500014F0DB06040EDBCF15F001E2DB06145013
:10BF6000151006E00C0EE66E15EC74F0E552EED7F7
:10BF7000DF2ADBD7280EE66EE66A52DFE552E5528D
:10BF80003C0EE66E41EC74F0E552060EE66EE66A93
:10BF900047DFE552E5523C0EE66E41EC74F0E552A7
:10BFA0000C0EE66EE66A3CDFE552E5523C0EE66EAC
:10BFB00041EC74F0E552010EE66EE66A31DFE552BF
:10BFC000E552020EF36E050EF3CFDBFF060EDB6AC1
:10BFD000050EDBCF14F0DB06060EDBCF15F001E219
:10BFE000DB061450151006E00C0EE66E15EC74F02E
:10BFF000E552EED7070EE15C02E2E16AE552E16E3E
:10C00000E552E5CFDAFFE7CFD9FF1200D9CFE6FF3F
:10C01000DACFE6FFE1CFD9FFE2CFDAFFE652E65210
:10C02000E652E652020EE66EE66AFADEE552E552A6
:10C03000020EF36EDB6E030EDB6A020EDBCF14F032
:10C04000DB06030EDBCF15F001E2DB061450151002
:10C0500006E00C0EE66E15EC74F0E552EED7DF6AE2
:10C06000100EDF5C33E2DF50EA6A240FE96E030E44
:10C07000EA22EF5017E1010EDFCFDBFF100EF36E67
:10C08000010EDBCFF4FFF350F45C0CE2010EDB5049
:10C09000EA6A240FE96E030EEA22200EEF6E010E0B
:10C0A000DB2AECD7DF50EA6A240FE96E030EEA229E
:10C0B000EF50E66E010EE66EB3DEE552E5523C0E41
:10C0C000E66E41EC74F0E552DF2ACAD7C00EE66E88
:10C0D000E66AA6DEE552E5523C0EE66E41EC74F0EF
:10C0E000E552100EDF6E200EDF5C33E2DF50EA6AAD
:10C0F000240FE96E030EEA22EF5017E1010EDFCFA5
:10C10000DBFF200EF36E010EDBCFF4FFF350F45C87
:10C110000CE2010EDB50EA6A240FE96E030EEA22FC
:10C12000200EEF6E010EDB2AECD7DF50EA6A240FF7
:10C13000E96E030EEA22EF50E66E010EE66E70DE47
:10C14000E552E5523C0EE66E41EC74F0E552DF2A12
:10C15000CAD7040EE15C02E2E16AE552E16EE55203
:10C16000E5CFDAFFE7CFD9FF1200D9CFE6FFDACF6C
:10C17000E6FFE1CFD9FFE2CFDAFFE652E652010E49
:10C18000E66EE66A4DDEE552E552020EDE6EDD6ACF
:10C19000DFCF14F0DF06010EDBCF15F001E2DB0686
:10C1A0001450151006E00C0EE66E15EC74F0E55216
:10C1B000EFD7200EE66EE66AE66E240EE66E030EFC
:10C1C000E66EA8EC6EF0146E050EE15C02E2E16A28
:10C1D000E552E16E1450E552E552E552E5CFDAFF43
:10C1E000E7CFD9FF1200D9CFE6FFDACFE6FFE1CFE4
:10C1F000D9FFE2CFDAFFE150FC0FE96EFF0EE2203B
:10C20000EA6EEE50ED1010E1100EE66EE66A200EBA
:10C21000E66E240EE66E030EE66EA8EC6EF0146E6B
:10C22000050EE15C1DE21AD0010E146E156AFC0EBB
:10C23000DB50141817E1FD0EDB50151813E1100E3A
:10C24000E66EE66A200EE66E340EE66E030EE66ECD
:10C25000A8EC6EF0146E050EE15C02E2E16AE552B4
:10C26000E16E1450E552E5CFDAFFE7CFD9FF1200B7
:10C27000D9CFE6FFDACFE6FFE1CFD9FFE2CFDAFF91
:10C28000E652E652020EE66EE66ACADDE552E55275
:10C29000020EDE6EDD6ADFCF14F0DF06010EDBCFAB
:10C2A00015F001E2DB061450151006E00C0EE66EE8
:10C2B00015EC74F0E552EFD7E552E552E552E5CFC3
:10C2C000DAFFE7CFD9FF1200D9CFE6FFDACFE6FFDA
:10C2D000E1CFD9FFE2CFDAFFE652E652FD0EDBCF27
:10C2E000E6FFE66A9DDDE552E552020EDE6EDD6A8E
:10C2F000DFCF14F0DF06010EDBCF15F001E2DB0625
:10C300001450151006E00C0EE66E15EC74F0E552B4
:10C31000EFD7E552E552E552E5CFDAFFE7CFD9FF97
:10C320001200D9CFE6FFDACFE6FFE1CFD9FFE2CFA7
:10C33000DAFFFD0EDBCFE6FF010EE66E71DDE552A2
:10C34000E5523C0EE66E41EC74F0E552E552E5CF65
:10C35000DAFFE7CFD9FF1200D9CFE6FFDACFE6FF49
:10C36000E1CFD9FFE2CFDAFFE652E652E652E652DB
:10C37000020EE66EE66A54DDE552E552020EF36EF9
:10C38000DB6E030EDB6A020EDBCF14F0DB06030E5E
:10C39000DBCF15F001E2DB061450151006E00C0EA1
:10C3A000E66E15EC74F0E552EED7DF6A100EDF5C36
:10C3B00033E2DF50EA6A240FE96E030EEA22EF50FF
:10C3C00017E1010EDFCFDBFF100EF36E010EDBCFA6
:10C3D000F4FFF350F45C0CE2010EDB50EA6A240F28
:10C3E000E96E030EEA22200EEF6E010EDB2AECD777
:10C3F000DF50EA6A240FE96E030EEA22EF50E66E80
:10C40000010EE66E0DDDE552E5523C0EE66E41ECA6
:10C4100074F0E552DF2ACAD7040EE15C02E2E16A59
:10C42000E552E16EE552E5CFDAFFE7CFD9FF120022
:10C43000D9CFE6FFDACFE6FFE1CFD9FFE2CFDAFFCF
:10C44000E652E652C00EE66EE66AEADCE552E552D6
:10C450003C0EE66E41EC74F0E552100EDF6E200EDD
:10C46000DF5C33E2DF50EA6A240FE96E030EEA2252
:10C47000EF5017E1010EDFCFDBFF200EF36E010E50
:10C48000DBCFF4FFF350F45C0CE2010EDB50EA6A00
:10C49000240FE96E030EEA22200EEF6E010EDB2A56
:10C4A000ECD7DF50EA6A240FE96E030EEA22EF5060
:10C4B000E66E010EE66EB4DCE552E5523C0EE66E29
:10C4C00041EC74F0E552DF2ACAD7E552E552E55255
:0AC4D000E5CFDAFFE7CFD9FF120035
:06C4DA00D9CFE6FFDACF26
:10C4E000E6FFE1CFD9FFE2CFDAFFF250E66EF29E2F
:10C4F000AD6AAC6A949C948E9F889F8AFA0EDBCFBB
:10C5000018F0FB0EDBCF19F0FC0EDBCF1AF0FD0E9E
:10C51000DBCF1BF0D890183619361A361B361B0E97
:10C520001926B70E1A22000E1B2218C006F019C0D9
:10C5300007F01AC008F01BC009F0FA0EDBCF0BF0B1
:10C54000FB0EDBCF0CF0FC0EDBCF0DF0FD0EDBCFD6
:10C550000EF0BAEC73F006C014F007C015F008C076
:10C5600016F009C017F0020ED890173216321532A5
:10C570001432E806F9E11406000E155A000E165A98
:10C58000000E175AD880FF0E1454000E1554000EDA
:10C590001654000E175448E3FA0EDBCF18F0FB0ECA
:10C5A000DBCF19F0FC0EDBCF1AF0FD0EDBCF1BF05A
:10C5B000D890183619361A361B361B0E1926B70EA8
:10C5C0001A22000E1B2218C006F019C007F01AC06C
:10C5D00008F01BC009F0FA0EDBCF0BF0FB0EDBCF2F
:10C5E0000CF0FC0EDBCF0DF0FD0EDBCF0EF0BAEC45
:10C5F00073F006C014F007C015F008C016F009C0AB
:10C6000017F0020ED8901732163215321432E8069F
:10C61000F9E11406000E155A000E165A000E175AAC
:10C620001450B06EAD844AD0FA0EDBCF18F0FB0E7A
:10C63000DBCF19F0FC0EDBCF1AF0FD0EDBCF1BF0C9
:10C64000030ED890183619361A361B36E806F9E16B
:10C650001B0E1926B70E1A22000E1B2218C006F058
:10C6600019C007F01AC008F01BC009F0FA0EDBCFA2
:10C670000BF0FB0EDBCF0CF0FC0EDBCF0DF0FD0E54
:10C68000DBCF0EF0BAEC73F006C014F007C015F063
:10C6900008C016F009C017F0040ED89017321632F1
:10C6A00015321432E806F9E11406000E155A000E90
:10C6B000165A000E175A1450B06EAD94AD8AAC8E57
:10C6C000AC88E552E7BEF28EF36AF46A00D0E55218
:10C6D000E5CFDAFFE7CFD9FF1200D9CFE6FFDACFF7
:10C6E000E6FFE552E5CFDAFFE7CFD9FF1200D9CF59
:10C6F000E6FFDACFE6FFE552E5CFDAFFE7CFD9FF75
:10C700001200D9CFE6FFDACFE6FFE1CFD9FFE2CFC3
:10C71000DAFFE66AF90EDBCFE6FFFA0EDBCFE6FFC3
:10C72000D950FB0FE66EFF0EDA20E66E58CEE6FF1C
:10C7300059CEE6FFAEEC43F0146E070EE15C02E268
:10C74000E16AE552E16E1450010802E0000E02D0E9
:10C750009D88010EE552E5CFDAFFE7CFD9FF120041
:10C76000D9CFE6FFDACFE6FFE552E5CFDAFFE7CF34
:10C77000D9FF1200D9CFE6FFDACFE6FFE1CFD9FF2C
:10C78000E2CFDAFFE652AF50DF6EACA202D0AC9837
:10C79000AC88C00E0F013DAF02D0D89003D03C5DF5
:10C7A000000E3D591BE238CFE9FF39CFEAFF382BA5
:10C7B000000E3923980EE9260D0EEA22DFCFEFFF97
:10C7C000C00E39AF02D0D89003D0385D000E395971
:10C7D00002E3386B396B3C2B000E3D23E552E552EA
:10C7E000E5CFDAFFE7CFD9FF1200E9CFE4FFEACFC8
:10C7F000E4FFF6CFE4FFF7CFE4FFF8CFE4FFF5CF97
:10C80000E4FFF3CFE4FFF4CFE4FFFACFE4FFFBCF84
:10C81000E4FF00EE00F0140EE80403E3EECFE4FFC3
:10C82000FBD700EE14F0120EE80403E3EECFE4FFB2
:10C83000FBD7E652A050100B06E0A150100B03E00E
:10C84000B3EC4DF002D09EBA95DFE55200EE25F034
:10C85000120EE80403E3E5CFEDFFFBD700EE13F083
:10C86000140EE80403E3E5CFEDFFFBD7E5CFFBFFB4
:10C87000E5CFFAFFE5CFF4FFE5CFF3FFE5CFF5FF16
:10C88000E5CFF8FFE5CFF7FFE5CFF6FFE5CFEAFF0D
:10C89000E5CFE9FF1100D8CFE4FFE0CFE4FFE46E7D
:10C8A000E9CFE4FFEACFE4FFF6CFE4FFF7CFE4FF00
:10C8B000F8CFE4FFF5CFE4FFF3CFE4FFF4CFE4FFDC
:10C8C000FACFE4FFFBCFE4FF00EE00F0140EE80423
:10C8D00003E3EECFE4FFFBD700EE14F0120EE80402
:10C8E00003E3EECFE4FFFBD7E652D9CFE6FFDACF82
:10C8F000E6FFE1CFD9FFE2CFDAFFE652E652010EC2
:10C90000DB6AD950010FE66E000EDA20E66ED9CF51
:10C91000E6FFDACFE6FF58CEE6FF59CEE6FF12EC8F
:10C9200049F0266E060EE15C02E2E16AE552E16E34
:10C930002650010803E1DF50AE6E01D09D98E5520C
:10C94000E552E552E5CFDAFFE7CFD9FFE55200EE39
:10C9500025F0120EE80403E3E5CFEDFFFBD700EE70
:10C9600013F0140EE80403E3E5CFEDFFFBD7E5CFAA
:10C97000FBFFE5CFFAFFE5CFF4FFE5CFF3FFE5CF0F
:10C98000F5FFE5CFF8FFE5CFF7FFE5CFF6FFE5CF01
:10C99000EAFFE5CFE9FFE550E5CFE0FFE5CFD8FFBF
:10C9A0001000D9CFE6FFDACFE6FFE1CFD9FFE2CF23
:10C9B000DAFFE652F250E66EF29EACA203D08C741F
:10C9C000AC98AC889EBA04D0E552E7BEF28E2ED069
:10C9D000AF50DF6EE552E7BEF28EC00E0F013DAFE5
:10C9E00002D0D89003D03C5D000E3D591FE20F01EC
:10C9F00038CFE9FF39CFEAFF382B000E3923980EE4
:10CA0000E9260D0EEA22DFCFEFFFC00E0F0139AF8E
:10CA100002D0D89003D0385D000E395903E30F01DE
:10CA2000386B396B0F013C2B000E3D23C3D7E55209
:10CA3000E552E5CFDAFFE7CFD9FF1200D9CFE6FF05
:10CA4000DACFE6FFE1CFD9FFE2CFDAFFE6520F01FE
:10CA50003C513D1121E03C07000E3D5B3ACFE9FF20
:10CA60003BCFEAFF3A2B3B23980EE9260D0EEA2234
:10CA7000EFCFDFFFC00E3BAF02D0D89003D03A5DBE
:10CA8000000E3B5902E33A6B3B6B3F510BE1240E26
:10CA9000146EDF50145C03E0F36AF46A52D0010EA6
:10CAA0003F6F3E6F3E513E2BE96EEA6AE9BEEA688F
:10CAB0005C0EE9260E0EEA22DFCFEFFF3ECF14F028
:10CAC000156A14BE1568580E141821E115501FE19F
:10CAD0003E513E2BE96EEA6AE9BEEA685C0EE92641
:10CAE0000E0EEA220D0EEF6E3E513E2BE96EEA6A03
:10CAF000E9BEEA685C0EE9260E0EEA220A0EEF6E27
:10CB00003ECFE9FFEA6AE9AE0CD0EA680AD00A0E25
:10CB1000146EDF50145C9BE13ECFE9FFEA6AE9BE88
:10CB2000EA685C0EE9260E0EEA22EF6A3E050E0167
:10CB30005C6F0F013F6B5C0E146E0E0E14C0F3FFA2
:10CB4000F46EE552E552E5CFDAFFE7CFD9FF1200E8
:10CB5000D9CFE6FFDACFE6FFE1CFD9FFE2CFDAFFA8
:10CB6000FC0EDBCFE9FFFD0EDBCFEAFF030EE9266B
:10CB7000000EEA22E9CF14F0EACF15F0FC0EDBCF6D
:10CB8000E9FFFD0EDBCFEAFFEE5214C0EEFF15C049
:10CB9000EDFFFC0EDBCFE9FFFD0EDBCFEAFF030E5E
:10CBA000E926000EEA22EE68ED68FC0EDBCFE9FF15
:10CBB000FD0EDBCFEAFF030EE926000EEA22E9CFE5
:10CBC00014F0EACF15F0FC0EDBCFE9FFFD0EDBCF52
:10CBD000EAFF030EE926000EEA22020EE926000E05
:10CBE000EA2214C0EEFF15C0EDFFFC0EDBCFE9FF1B
:10CBF000FD0EDBCFEAFF030EE926000EEA22E9CFA5
:10CC000014F0EACF15F0FC0EDBCFE9FFFD0EDBCF11
:10CC1000EAFF030EE926000EEA22040EE926000EC2
:10CC2000EA2214C0EEFF15C0EDFFFC0EDBCFE9FFDA
:10CC3000FD0EDBCFEAFFEF6AE552E5CFDAFFE7CF83
:10CC4000D9FF1200D9CFE6FFDACFE6FFE1CFD9FF57
:10CC5000E2CFDAFFFC0EDBCFE9FFFD0EDBCFEAFF10
:10CC6000080EEB6A090EEB6AE552E5CFDAFFE7CF73
:10CC7000D9FF1200D9CFE6FFDACFE6FFE1CFD9FF27
:10CC8000E2CFDAFFE652E652FC0EDBCFE9FFFD0E03
:10CC9000DBCFEAFFEE52EECFDEFFEDCFDDFFDECFE2
:10CCA000E9FFDDCFEAFF020EE926000EEA22EECF11
:10CCB00014F0EFCF15F0FA0EDBCFE9FFFB0EDBCF60
:10CCC000EAFF020EE926000EEA2214C0EEFF15C0AC
:10CCD000EDFFFC0EDBCFE9FFFD0EDBCFEAFFEE52EE
:10CCE000EECF14F0EFCF15F0FA0EDBCFE9FFFB0E1D
:10CCF000DBCFEAFF040EE926000EEA2214C0EEFFA5
:10CD000015C0EDFFDECFE9FFDDCFEAFF020EE92619
:10CD1000000EEA22EE50EFCFEAFFE96E040EE9269C
:10CD2000000EEA22FA0EDBCFEEFFFB0EDBCFEDFFAB
:10CD3000DECFE9FFDDCFEAFF020EE926000EEA2290
:10CD4000FA0EDBCFEEFFFB0EDBCFEDFFFC0EDBCFF1
:10CD5000E9FFFD0EDBCFEAFFEE52FA0EDBCFEEFF6E
:10CD6000FB0EDBCFEDFFFA0EDBCFE9FFFB0EDBCFD7
:10CD7000EAFF080EE926000EEA22FC0EDBCFEEFFEA
:10CD8000FD0EDBCFEDFFFC0EDBCFE9FFFD0EDBCFB1
:10CD9000EAFFEF2AE552E552E552E5CFDAFFE7CFA9
:10CDA000D9FF1200D9CFE6FFDACFE6FFE1CFD9FFF6
:10CDB000E2CFDAFFE652E652E652E652FA0EDBCF57
:10CDC000E9FFFB0EDBCFEAFF020EEECFDBFF030E27
:10CDD000EDCFDBFFD950020FE96E000EDA20EA6ECC
:10CDE000FF0EEE1816E1FF0EED1813E1FC0EDBCF7F
:10CDF000E9FFFD0EDBCFEAFF030EE926000EEA2273
:10CE0000040EE926000EEA22EECFDEFFEDCFDDFFB5
:10CE100036D0FC0EDBCFE9FFFD0EDBCFEAFF030EC1
:10CE2000E926000EEA22E9CFDEFFEACFDDFFDECF02
:10CE3000E9FFDDCFEAFF020EE926000EEA22EE50FE
:10CE4000EFCFEAFFE96EEECF14F0EFCF15F0020E50
:10CE5000DBCF16F0030EDBCF17F01450165C155025
:10CE600017580DE3DECFE9FFDDCFEAFF020EE9261A
:10CE7000000EEA22EECFDEFFEDCFDDFFD8D7DECF0A
:10CE8000E9FFDDCFEAFF020EE926000EEA22EECF2F
:10CE900014F0EFCF15F0FA0EDBCFE9FFFB0EDBCF7E
:10CEA000EAFF020EE926000EEA2214C0EEFF15C0CA
:10CEB000EDFFFA0EDBCFE9FFFB0EDBCFEAFF020E40
:10CEC000E926000EEA22EE50EFCFEAFFE96E040EEB
:10CED000E926000EEA22FA0EDBCFEEFFFB0EDBCFD7
:10CEE000EDFFFA0EDBCFE9FFFB0EDBCFEAFF040E0E
:10CEF000E926000EEA22DECFEEFFDDCFEDFFDECF2A
:10CF0000E9FFDDCFEAFF020EE926000EEA22FA0E63
:10CF1000DBCFEEFFFB0EDBCFEDFFFA0EDBCFE9FF41
:10CF2000FB0EDBCFEAFF080EE926000EEA22FC0E1C
:10CF3000DBCFEEFFFD0EDBCFEDFFFC0EDBCFE9FF1D
:10CF4000FD0EDBCFEAFFEF2A040EE15C02E2E16AAC
:10CF5000E552E16EE552E5CFDAFFE7CFD9FF1200E7
:10CF6000D9CFE6FFDACFE6FFE1CFD9FFE2CFDAFF94
:10CF7000E652E652FC0EDBCFE9FFFD0EDBCFEAFF07
:10CF8000040EE926000EEA22EECF14F0EFCF15F0E2
:10CF9000FC0EDBCFE9FFFD0EDBCFEAFF020EE92638
:10CFA000000EEA22EE50EFCFEAFFE96E040EE9260A
:10CFB000000EEA2214C0EEFF15C0EDFFFC0EDBCF21
:10CFC000E9FFFD0EDBCFEAFF020EE926000EEA22A2
:10CFD000EECF14F0EFCF15F0FC0EDBCFE9FFFD0E26
:10CFE000DBCFEAFF040EE926000EEA22EE50EFCF77
:10CFF000EAFFE96E020EE926000EEA2214C0EEFFF7
:10D0000015C0EDFFFC0EDBCFE9FFFD0EDBCFEAFF25
:10D01000080EE926000EEA22EECFDEFFEDCFDDFF9F
:10D02000DECFE9FFDDCFEAFFEE52EECF14F0EFCF17
:10D0300015F0FC0EDB5014181BE1FD0EDB5015182B
:10D0400017E1FC0EDBCFE9FFFD0EDBCFEAFF040E9C
:10D05000E926000EEA22EECF14F0EFCF15F0DECF76
:10D06000E9FFDDCFEAFFEE5214C0EEFF15C0EDFF81
:10D07000FC0EDBCFE9FFFD0EDBCFEAFF080EEB6A0B
:10D08000090EEB6ADECFE9FFDDCFEAFFEF06E552DE
:0ED09000E552E552E5CFDAFFE7CFD9FF1200F7
:02D09E0004018B
:10D0A00040511F0B010801E012004051600BE842A3
:10D0B000E842E842E842E842010801E01200445137
:10D0C00003E0440501E012004151220A35E0030A61
:10D0D00028E0010A15E0210A0DE0010A01E0120032
:10D0E0000F01F20E196F040E1A6F080E1D6F1E6BE2
:10D0F0001C8125D00F01F20E196F040E1A6F1FD07C
:10D1000046C422FF47C423FF0F01500E1F6F040EB9
:10D11000206F720E246F6D0E256F000E266F218F0B
:10D1200012000F01D80E196F040E1A6F070E1D6F33
:10D130001E6BC10E1C6F120042C4EDF40F011C8F58
:10D1400012000401D86B4B0ED96FDA6BDB6BDC6B12
:10D15000DD6B080EDE6FE06BDF6B1A0EE66E020E03
:10D16000E66ED7EC54F0E552E5521E0EE66E030E65
:10D17000E66ED7EC54F0E552E552400EE66E580EDE
:10D18000E66E040EE66EE66A030EE66E7FEC55F080
:10D19000146E050EE15C02E2E16AE552E16E1450A4
:10D1A000F3CFE9F4F4CFEAF40401EB6BEC6B12007B
:10D1B000D9CFE6FFDACFE6FFE1CFD9FFE2CFDAFF42
:10D1C0000401DF6BE951EA1102E1000E08D0E9C465
:10D1D000E9FFEAC4EAFFEF50800B01E0010E00090D
:10D1E00049E1FB0EDBCF14F0E9C4E9FFEAC4EAFF32
:10D1F000EE52EF50D880145408E2E9C4E9FFEAC4C3
:10D20000EAFFEE52FB0EEFCFDBFFDF6BFB0EDB50D6
:10D21000DF5D19E2DF51EA6A580FE96E040EEA2277
:10D22000EF50E66EDF51E76EFC0EDBCFE9FFFD0E3F
:10D23000DBCFEAFFE750E926000EEA22E552E7508D
:10D24000EF6EDF2BE3D7400EE66E580EE66E040E4F
:10D25000E66EE66A030EE66E7FEC55F0146E050E80
:10D26000E15C02E2E16AE552E16E1450F3CFE9F4C9
:10D27000F4CFEAF40401DF51E552E5CFDAFFE7CF5E
:10D28000D9FF1200D9CFE6FFDACFE6FFE1CFD9FF11
:10D29000E2CFDAFFA0980401E0510CE1FC0EDBCFF5
:10D2A000E1F4FD0EDBCFE2F4FB0EDBCFE7F4010E81
:10D2B000E86FE06FA088E552E5CFDAFFE7CFD9FF4E
:10D2C0001200D9CFE6FFDACFE6FFE1CFD9FFE2CFF8
:10D2D000DAFFE652E652E652A0980401E0512DE151
:10D2E000DF6AFC0EDBCF08F0FD0EDBCF09F0DE526B
:10D2F00008C0DEFF09C0DDFFDD52DF2ADF50146EFB
:10D30000156AFF0E141802E115500BE0010EDBCF79
:10D31000E9FFDB2A020EDBCFEAFF01E3DB2AEF5055
:10D32000ECE1FC0EDBCFE1F4FD0EDBCFE2F4DFCF6E
:10D33000E7F40401010EE86FE06FA088E552E552C2
:10D34000E552E552E5CFDAFFE7CFD9FF1200D9CF9A
:10D35000E6FFDACFE6FFE1CFD9FFE2CFDAFFE65210
:10D36000E652E652E652A0980401E0513BE1DF6A42
:10D37000D950FB0FE96EFF0EDA20EA6E010EEECFF8
:10D38000DBFF020EEECFDBFF030EEECFDBFFDF2A6B
:10D39000DF50146E156AFF0E141802E1155013E0E9
:10D3A000D950010FE96E000EDA20EA6EEFCFF6FFDA
:10D3B000EE2AEFCFF7FF000EEE22EFCFF8FFEE22BE
:10D3C0000800F550E4E1FB0EDBCFE1F4FC0EDBCF0F
:10D3D000E2F4FD0EDBCFE3F4DFCFE7F40401E86B0A
:10D3E000010EE06FA088040EE15C02E2E16AE55202
:10D3F000E16EE552E5CFDAFFE7CFD9FF1200D9CFD2
:10D40000E6FFDACFE6FFE1CFD9FFE2CFDAFFE6525F
:10D41000E652A0980401EB51EC1102E1000E08D095
:10D42000EBC4E9FFECC4EAFFEF50800B01E0010E12
:10D43000000906E1030EE05D01E1E06BE05102E16D
:10D44000A08889D0020EE05D1AE1E66A000EE66E61
:10D45000E66A010EE66E030EE66E7FEC55F0146E82
:10D46000050EE15C02E2E16AE552E16E1450F3CF91
:10D47000EBF4F4CFECF40401030EE06F6BD0E005A5
:10D4800069E1400E146E156AE751145C000E1558E0
:10D4900003E2400EDF6E02D0E7C4DFFFDF50E75D3E
:10D4A000E76F980EE46F040EE56F010EDFCFDBFF30
:10D4B000E85119E1010EDB502BE0E1C4F6FFE2C4B4
:10D4C000F7FFE3C4F8FF0800F550E4C4E9FFE5C442
:10D4D000EAFFEF6EE42B000EE523E12BE223E323CA
:10D4E000010EDB06E7D7010EDB5012E0E1C4E9FFD5
:10D4F000E2C4EAFFEF50E4C4E9FFE5C4EAFFEF6EDF
:10D50000E42B000EE523E12BE223010EDB06EBD733
:10D510000401E75107E1400EDF5C02E1020E01D099
:10D52000030EE06FDFCFE6FF980EE66E040EE66EA8
:10D53000010EE66E030EE66E7FEC55F0146E050EDE
:10D54000E15C02E2E16AE552E16E1450F3CFEBF4E4
:10D55000F4CFECF4A088E552E552E552E5CFDAFFCE
:06D56000E7CFD9FF120025
:0AD56600D9CFE6FFDACFE6FFE1CFF0
:10D57000D9FFE2CFDAFFFD0EDB506F6E6CAE02D04A
:10D58000FF0E03D06DB0FED7000EE552E5CFDAFFF7
:10D59000E7CFD9FF12006B866DA0FED76F50120047
:10D5A0003F0E6D166C6A6B6A6C86958C958A6C8AD8
:10D5B0000B0E6E6E12006D50040B01E0010E146E26
:10D5C0001F0E6B141410F7E16B846BB4FED7A1B679
:10D5D000010C000CD9CFE6FFDACFE6FFE1CFD9FF8F
:10D5E000E2CFDAFFE652E652FB0EDBCFDEFFDBCF07
:10D5F000DDFF6D50040B01E0010E146E1F0E6B1465
:10D600001410F7E16B806BB0FED7A1B635D0FD0EDC
:10D61000DBCFE6FFA8DFE55200092EE16D50040BD9
:10D6200001E0010E146E1F0E6B141410F7E16BBCB9
:10D6300025D0010EDBCFE6FF96DFE55200091CE1A5
:10D640006D50040B01E0010E146E1F0E6B141410CC
:10D65000F7E1DFCFE6FF87DFE55200090DE16D500E
:10D66000040B01E0010E146E1F0E6B141410F7E191
:10D670006BBC02D0000E03D0010E01D0010EE552AA
:10D68000E552E552E5CFDAFFE7CFD9FF1200D9CF57
:10D69000E6FFDACFE6FFE1CFD9FFE2CFDAFFE652CD
:10D6A000FA0EDBCFE6FFFB0EDBCFE6FFA00EE66E49
:10D6B00091DFE552E552E552DF6EDF5004E17BDF9A
:10D6C000DF6EDF5002E0DF5024D06D50040B01E02C
:10D6D000010E146E1F0E6B141410F7E16B806BB00B
:10D6E000FED7A1B606D0A10EE66E3DDFE5520009D9
:10D6F00002E0010E0ED06D50040B01E0010E146E1D
:10D700001F0E6B141410F7E16BBC02D0000E01D099
:10D71000010EE552E552E5CFDAFFE7CFD9FF12005F
:10D72000D9CFE6FFDACFE6FFE1CFD9FFE2CFDAFFCC
:10D73000FA0EDBCFE6FFFB0EDBCFE6FFA00EE66EB8
:10D7400049DFE552E552E552E552E5CFDAFFE7CF92
:10D75000D9FF1200D9CFE6FFDACFE6FFE1CFD9FF3C
:10D76000E2CFDAFF6D50040B01E0010E146E1F0EC4
:10D770006B141410F7E1FD0EDBCFE6FFF4DEE5528B
:10D78000000902E0010E0ED06D50040B01E0010E05
:10D79000146E1F0E6B141410F7E16BBC02D0000E58
:10D7A00001D0010EE552E5CFDAFFE7CFD9FF120035
:10D7B000D9CFE6FFDACFE6FFE1CFD9FFE2CFDAFF3C
:10D7C000FA0EDBCF14F0DB06FB0EDBCF15F001E227
:10D7D000DB06145015100EE0FC0EDBCFE9FFDB2A50
:10D7E000FD0EDBCFEAFF01E3DB2AEF50E66EB2DF8E
:10D7F000E552E6D706D8E552E5CFDAFFE7CFD9FF05
:10D8000012006D50040B01E0010E146E1F0E6B141C
:10D810001410F7E16B846BB4FED7000CBCDE6BB662
:10D82000FED76B9A6B886BB8FED76F501200B3DED1
:10D830006BB6FED76B8A6B886BB8FED76B846BB404
:10D84000FED7000CD9CFE6FFDACFE6FFE1CFD9FF54
:10D85000E2CFDAFFE652D950FA0FE96EFF0EDA2076
:10D86000EA6EEECFE6FFEECFE6FFEECFE6FFEFCFBC
:10D87000E6FF0DDFE552E552E552E552DF6EDF507F
:10D880001DE1F60EDBCF14F0DB06F70EDBCF15F053
:10D8900001E2DB06145015100FE0C0DFE66EF80E53
:10D8A000DBCFE9FFDB2AF90EDBCFEAFF01E3DB2A5E
:10D8B000E552E750EF6EE5D7BADFDF6EDF50E55295
:10D8C000E552E5CFDAFFE7CFD9FF1200D9CFE6FF67
:10D8D000DACFE6FFE1CFD9FFE2CFDAFFE6526D50B3
:10D8E000040B01E0010E146E1F0E6B141410F7E10F
:10D8F0006B806BB0FED7A1B61BD0E66A34DEE55272
:10D90000000916E16D50040B01E0010E146E1F0EAC
:10D910006B141410F7E1A1B60BD06BBC02D0DF6A18
:10D9200002D0010EDF6E6B846BB4FED7A1A602D0CD
:10D93000010E01D0DF50E552E552E5CFDAFFE7CF27
:04D94000D9FF1200F9
:0CD944000D0A00544D4F4600544D4F4E4C
:10D950000047544D520053544D52005354555300F8
:10D9600054494D450044415445004F464600434EFE
:10D97000540053474C0024504645430030003300C8
:10D980003200310047506173740047507470730067
:10D99000205554432054696D652041646A75737441
:10D9A000004E6F7720496E697469616C697A696E9F
:10D9B00067002447505A44412C2C2C2C2C2B3030FF
:10D9C0002C30300D0A00534154004652490054484F
:10D9D000550057454400545545004D4F4E00535592
:10D9E0004E0053656C656374204D656E75204974F7
:10D9F000656D002B30303A30300059657320204E71
:10DA00006F200054696D657220416C6C204F666612
:10DA1000203F00313248203234482000544D31201C
:10DA2000544D3220544D3320544D34200053545221
:10DA300020205354500053657475702054494D454F
:10DA4000522D6E20200054696D65722D6E204F4658
:10DA500046004966207075736820544F4646204B37
:10DA6000657900207F2020207E20205550202044F2
:10DA7000574E00434E540053474C004F4646005407
:10DA80004D0054696D6520466F726D617400536579
:10DA9000742054696D6572004C6F63616C20546929
:10DAA0006D6500414854005954004844540059449D
:10DAB0005400505400504454004D4454004354000A
:10DAC00043445400454454004E54004E4654004EC6
:10DAD00044540057455400474D540057455444544E
:10DAE000004554004E4F52004D455A004D45575485
:10DAF00000465400444E54004345540054004D45E4
:10DB0000544454004D455400465754004545540074
:10DB1000434554445400454554445400425400493C
:10DB20005400574154004A5400575400574144543C
:10DB300000434354004D5400574454004B54004A92
:10DB400053540041575400434154004154004C4940
:10DB50004754004754004541540041445400434158
:10DB600044540041435400414554004E5A54004926
:10DB7000444C45004E5A4454005554430049444CCB
:10DB80004500496E76616C696420436F6D6D616E0E
:10DB9000640D0A0053656E642044697265637420E5
:10DBA000746F20475053204D6F64756C650D0A00EB
:10DBB000496E76616C696420506172616D6574654F
:10DBC000720D0A004F4B0D0A000D0A24436D643E8E
:10DBD0000024504645432C47507365742C5A320D2F
:10DBE0000A0024504645432C4750696E742C6173DB
:10DBF0007430310D0A0024504645432C4750727250
:10DC0000732C312C3130302C320D0A002450464513
:10DC1000432C47507365742C4D350D0A0024504633
:10DC200045432C47507365742C4B320D0A00245029
:10DC30004645432C4750636C722C310D0A004672E6
:10DC4000656552544F532076362E312E30002050C9
:10DC50006F776572656420627900202056657220B6
:10DC6000312E302E310047505320436C6F636B2FA1
:06DC700054696D657200AD
:0ADC7600FB0EE3CFF6FFFC0EE3CF38
:10DC8000F7FFFD0EE3CFF8FFFE0EE3CFE9FFFF0E37
:10DC9000E3CFEAFFF90EE35003E1FA0EE35009E0A7
:10DCA000F90EE30602E2FA0EE3060900F550EE5C17
:10DCB000F1E01200D9CFE6FFDACFE6FFFA0EE3CFAC
:10DCC000D9FFFB0EE3CFDAFFFC0EE3CFE9FFFD0E39
:10DCD000E3CFEAFFE9CFF3FFEACFF4FFF80EE3501A
:10DCE00003E1F90EE35008E0F80EE30602E2F90E54
:10DCF000E306DECFEEFFF2D7FF0EE3CFDAFFE55209
:10DD0000FF0EE3CFD9FFE5521200FB0EE3CFF6FF83
:10DD1000FC0EE3CFF7FFFD0EE3CFF8FFFE0EE3CFDF
:10DD2000E9FFFF0EE3CFEAFFE9CFF3FFEACFF4FF0D
:10DD3000F90EE35003E1FA0EE35009E0F90EE306B1
:10DD400002E2FA0EE3060900F5CFEEFFF1D712006A
:10DD5000FE0EE3CFE9FFFF0EE3CFEAFFE9CFF3FFCB
:10DD6000EACFF4FFFB0EE35003E1FC0EE35009E0C1
:10DD7000FB0EE30602E2FC0EE306FD0EE350EE6E40
:10DD8000F1D71200FB0EE3CFF6FFFC0EE3CFF7FF57
:10DD9000FD0EE3CFF8FFFE0EE3CFE9FFFF0EE3CF6A
:10DDA000EAFFE9CFF3FFEACFF4FFEE66FED7ED52CC
:10DDB0000900F5CFEFFFEE66FBD71200FB0EE3CFB5
:10DDC000F6FFFC0EE3CFF7FFFD0EE3CFF8FFFE0EEC
:10DDD000E3CFE9FFFF0EE3CFEAFF0900F550EF5C68
:10DDE00002E1EE66FAD71200FB0EE3CFF6FFFC0E5F
:10DDF000E3CFF7FFFD0EE3CFF8FFFE0EE3CFE9FF21
:10DE0000FF0EE3CFEAFFE9CFF3FFEACFF4FF09000B
:10DE1000F5CFEFFFEE66FBD71200FE0EE3CFE9FF72
:10DE2000FF0EE3CFEAFFF36AF46AEE5203E0F34A2F
:10DE3000F42AFBD71200FF0EE3CFF8FFE552FF0EE6
:10DE4000E3CFF7FFE552FF0EE3CFF6FFE552E66AB8
:10DE5000E66AE66A0900F55209E0FD0EE32A05E1EB
:10DE6000FE0EE32A02E1FF0EE32AF4D7FD0EE3CF14
:10DE700007F0FE0EE3CF08F0FF0EE3CF09F012002B
:10DE8000D9CFE6FFDACFE6FFFA0EE3CFD9FFFB0EDC
:10DE9000E3CFDAFFFC0EE3CFE9FFFD0EE3CFEAFFAD
:10DEA000E9CFF3FFEACFF4FFF80EE35003E1F90EF8
:10DEB000E3500BE0F80EE30602E2F90EE306DECFD4
:10DEC000EFFFEE66F1D7DD52EFD7FF0EE3CFDAFFBB
:0CDED000E552FF0EE3CFD9FFE55212002F
:04DEDC00D9CFE6FFB5
:10DEE000DACFE6FFE1CFD9FFE2CFDAFFE652E65222
:10DEF000B00EDE6E040EDD6E9B8CDFCF14F0DF06FD
:10DF0000010EDBCF15F001E2DB0614501510F5E130
:10DF1000C088C168C268C098D9EC34F03BEC4DF0C1
:10DF2000E552E552E552E5CFDAFFE7CFD9FF12001F
:10DF30000401FB51FC1112E165A20BD062B404D0C4
:10DF4000E20EFB6F040E08D06284100EFB6F270EEA
:10DF500003D0880EFB6F130EFC6F03D0FB07000E7F
:10DF6000FC5B65A20AD0FB51FC112CE18A728AA2EB
:10DF700002D08A8412008A9412000F01005101E13C
:10DF80001200000501E11200020E005D01E1120025
:10DF9000040E005D01E11200100E005D06E10401B7
:10DFA000FB51FC110FE18A720AD0200E005D0AE1DC
:10DFB0000401FB51FC1106E18A728AA202D08A9404
:10DFC00012008A84120012001200120012004FEF99
:10DFD00068F01200A1EF68F065840401080EFD6F7F
:10DFE000070EFE6FFD07000EFE5BFD51FE11FAE10C
:10DFF00065941200D9CFE6FFDACFE6FFE1CFD9FF73
:10E00000E2CFDAFFFC0EDBCF08F0FD0EDBCF09F02C
:10E01000720E081801E1095033E0E868081802E1BF
:10E020007F0E09182BE0740E081801E1095024E056
:10E03000750E081801E109501DE0730E081801E182
:10E04000095016E0030E081801E109500FE0020E16
:10E05000081801E1095008E0010E081801E1095013
:10E0600001E010D0B7DF0FD0B4DF0DD0B0DF0BD0A0
:10E07000ACDF09D0A8DF07D0A7DF05D0A7DF03D02A
:10E08000000001D000D0010E00D0E552E5CFDAFF4C
:06E09000E7CFD9FF1200EA
:0AE09600AD50020B020A01E0010E7A
:10E0A00012004F0EAC16AD9ACF0E9D161200ACA208
:10E0B00002D0AC98AC889E50200B01E0010E1200FB
:10E0C000AF501200D9CFE6FFDACFE6FFE1CFD9FF9C
:10E0D000E2CFDAFFFD0EDB50AE6EE552E5CFDAFFA0
:10E0E000E7CFD9FF1200D9CFE6FFDACFE6FFE1CFC5
:10E0F000D9FFE2CFDAFFE652E652DF6AFB0EDB50D1
:10E10000DF5C18E2D4DF0009FDE0DADFE76E010E24
:10E11000E7CFDBFFFC0EDBCFE9FFFD0EDBCFEAFF35
:10E12000010EDBCFEFFFFC0EDB2AFD0E01E3DB2A45
:10E13000DF2AE4D7E552E552E552E5CFDAFFE7CF33
:10E14000D9FF1200D9CFE6FFDACFE6FFE1CFD9FF42
:10E15000E2CFDAFFF250E66EF29E9DDF000901E0A9
:10E16000FCD7FC0EDBCFE9FFFD0EDBCFEAFFEF5063
:10E17000E66EA8DFE552FC0EDBCFE9FFDB2AFD0EE1
:10E18000DBCFEAFF01E3DB2AEF50E7E1E552E7BE30
:10E19000F28EE552E5CFDAFFE7CFD9FF1200D9CFF3
:10E1A000E6FFDACFE6FFE1CFD9FFE2CFDAFFF250A8
:10E1B000E66EF29E70DF000901E0FCD7FB0EDBCFBC
:10E1C000F6FFFC0EDBCFF7FFFD0EDBCFF8FF0800FC
:10E1D000F550E66E77DFE552D950FB0FE96EFF0E82
:10E1E000DA20EA6EEFCFF6FFEE2AEFCFF7FF000E50
:10E1F000EE22EFCFF8FF000EEE220800F550DAE134
:10E20000E552E7BEF28EE552E5CFDAFFE7CFD9FF60
:02E210001200FA
:0EE21200006A0EAE0FEF71F00E6C001E09AE2A
:10E2200014EF71F0096C001E33EC74F009BE1EEFA0
:10E2300071F000AE000C096C056C000C00BE1BEF09
:10E2400071F00188FF0C006A0EAE2CEF71F00D6CBE
:10E250000E1EE86A0E22001E09AE34EF71F0086C43
:10E26000091EE86A0922001EFFEC73F009BE44EFA4
:10E2700071F000AE000C086C091EE86A0922046CFB
:10E28000051EE86A0522000C00BE3BEF71F0018814
:10E29000FF0C09C013F008C012F008500D02F4CFB3
:10E2A00007F0F3CF06F009500E02F4CF09F0F3CFD8
:10E2B00008F00D02F3500726F4500822E86A0922FC
:10E2C00012500E02F3500726F4500822E86A092281
:10E2D0000EAE6FEF71F01250085E1350095A13AE74
:10E2E000000C0D50085E0E50095A000C09C013F0C6
:10E2F00008C012F007C011F007500C02F4CF05F06F
:10E30000F3CF04F008500D02F4CF07F0F3CF06F07E
:10E310000C02F3500526F4500622E86A0722115039
:10E320000D02F3500526F4500622E86A0722095030
:10E330000C02F3500626F450072209500D02086A19
:10E34000E86A0822F3500726F450082211500E0202
:10E35000F3500626F4500722096AE86A08220922C7
:10E3600012500E02F3500726F4500822E86A0922E0
:0EE3700013500E02F3500826F4500922000C40
:02E37E0079DB49
:10E3800000000074DB000D006FDB000C006BDB0095
:10E390000C0067DB000B0063DB000A1E5EDB000A7B
:10E3A0001E5ADB000A1E67DB000A0056DB000A006B
:10E3B00053DB000A004EDB000A0063DB00091E4B42
:10E3C000DB00091E47DB00091E43DB0009003FDBC1
:10E3D0000009003CDB00090038DB00090035DB00E8
:10E3E000081E43DB00080031DB0008002CDB0008BE
:10E3F0000029DB00080026DB00071E22DB000700E7
:10E400001FDB00031E1CDB00030016DB00030010F3
:10E41000DB0002000CDB00020008DB0002001FDB57
:10E4200000020004DB000200FEDA000200FCDA0059
:10E4300002001CDB000100F8DA000100F4DA000140
:10E4400000F1DA00010004DB000100ECDA00010059
:10E45000E8DA000100E4DA000100E1DA0001002955
:10E46000DB000100DBDA000100D7DA000000D3DABC
:10E4700000000022DB00FF00CFDA00FE1E5ADB00A6
:10E48000FD00CBDA00FD1EC8DA00FD1E4BDB00FCF0
:10E4900000C4DA00FC00C0DA00FB00E1DA00FB0097
:10E4A000BDDA00FA00B9DA00FA0035DB00F900B590
:10E4B000DA00F900B2DA00F800AEDA00F800AADA01
:10E4C00000F700A7DA00F700A3DA00F60047DB0048
:07E4D000F600C8DA00F500B8
:01E4D7000044
:08E4D800D9CFE6FFDACFE6FF21
:10E4E000E1CFD9FFE2CFDAFFE652E652DE6ADD6A1B
:10E4F000F8EC3BF0FC0EDB50030168250001146EC4
:10E50000FD0EDB50030169210001156E980E145CAD
:10E51000080E155825E2FC0EDB50030168250001AA
:10E52000166EFD0EDB50030169210001176E030119
:10E530001650685D1750695913E2000E6825146E75
:10E54000050E6921156E14C0DEFFDD6EFC0EDBCFFB
:10E5500008F0FD0EDBCF09F0085068270950692349
:10E56000FBEC3BF0DECF14F0DDCF15F014C0F3FF71
:10E5700015C0F4FFE552E552E552E5CFDAFFE7CFEB
:10E58000D9FF1200D9CFE6FFDACFE6FFE552E5CF9B
:10E59000DAFFE7CFD9FF12000301686B696B120045
:10E5A00068C314F069C315F0980ED8801456080E8D
:0CE5B000155614C0F3FF15C0F4FF120054
:04E5BC001201000246
:10E5C00002000008D8040A0000010102000109024B
:10E5D0004300020100C032090400000102020100F0
:10E5E000052400100104240202052406000105246C
:10E5F0000100010705820308000209040100020A64
:10E6000000000007050302400000070583024000E8
:10E61000000403090434034D006900630072006FB5
:10E62000006300680069007000200054006500630A
:10E630000068006E006F006C006F006700790020BA
:10E640000049006E0063002E00340354007200691C
:10E650000053007400610074006500200040004712
:10E6600000500053002D0043006C006F0063006BEE
:10E67000002F00540069006D0065007200CEE500B7
:09E6800011E60015E60049E60070
:01E68900454B
:06E68A00800EF66E100E7A
:10E69000F76E000EF86E00010900F550FB6F0900DF
:10E6A000F550FC6F03E1FB6701D03DD00900F55048
:10E6B000F66F0900F550F76F0900F550F86F090083
:10E6C0000900F550E96E0900F550EA6E09000900ED
:10E6D0000900F550F96F0900F550FA6F09000900BB
:10E6E000F6CFFDF0F7CFFEF0F8CFFFF0F6C0F6FF63
:10E6F000F7C0F7FFF8C0F8FF0001F95302E1FA5341
:10E7000007E00900F550EE6EF907F8E2FA07F9D7CD
:10E71000FDC0F6FFFEC0F7FFFFC0F8FF0001FB07DA
:08E72000000EFC5BBFD71200E4
:08E72800F36AF46AFF0EE1241C
:10E73000E96EFF0EE220EA6EED6607D02F0EEF6461
:10E7400004D03A0EEF6001D0F32A1200FF0EE1244C
:10E75000E96EFF0EE220EA6EEDCFF4FFEFCFF3FF9C
:10E76000F46607D0600EF36404D07B0EF36001D032
:04E77000F39A120006
:0CE77400056A046A036A026A200EE76E60
:10E78000D890063607360836093602360336043680
:10E7900005360B50025C0C5003580D5004580E50B7
:10E7A000055809E30B50025E0C50035A0D50045AF1
:0CE7B0000E50055A062AE72EE4D712008E
:04E7BC00D9CFE6FFCC
:10E7C000DACFE6FFE1CFD9FFE2CFDAFFFD0EDB5073
:10E7D0007E0BCD6EFD0EDBAC02D0CD8E01D0CD9E7A
:10E7E000CF6ACE6A9E90DBAE02D09D8001D09D9014
:0EE7F000CD80E552E5CFDAFFE7CFD9FF12006A
:02E7FE00056AAA
:10E80000046A100EE76ED8900836093604360536CD
:10E810000D50045C0E50055805E30D50045E0E507B
:0AE82000055A082AE72EF0D712006F
:06E82A00FF0EE350276E13
:10E83000480E01D04C0EE76EE72EFED7E76AE72EB2
:0AE84000FED7272EF7D700001200C4
:06E84A0011EE00F021EECA
:10E8500000F0F86A019C45EC73F053EC74F01FEC87
:06E860002AF0FBD71200B4
:0AE86600056A080EE76ED890093627
:10E8700005360E50055C02E3056E092AE72EF7D730
:02E88000120084
:0EE88200FF0EE350E84E1200000000D000D060
:08E8900000D0E82EFAD71200B7
:08E8980000EE00F00F0EEE6A25
:06E8A000EA62FDD7120040
:02E8A60012005E
:08E8A800000000000000000068
:05E8B000000000000063
:08E8B50000000000000000005B
:03E8BD0001000057
:10E8C0000001020304050600000000000000000033
:06E8D00000000000000042
:03E8D6000000013E
:07E8D90098DA008EDA0082DC
:03E8E000DA00005B
:02E8E300000033
:03E8E50000000030
:08E8E8005247552A2B000000E5
:10E8F000000000000001000000DED900DAD900D6D7
:10E90000D900D2D900CED900CAD900C6D900000A90
:0AE91000141E28323C46505A000045
:020000040001F9
:01FFF800A662
:01FFF900F710
:01FFFA000501
:01FFFB00FF06
:01FFFD00F70C
:00000001FF
